:100000000C94BC180C94ED180C94ED180C94ED188D
:100010000C94ED180C94ED180C94ED180C94ED184C
:100020000C94ED180C94ED180C94ED180C94ED183C
:100030000C94ED180C94ED180C94ED180C94ED182C
:100040000C94ED180C94DBD80C94ED180C94ED186E
:100050000C94ED180C94ED180C9439C40D945310B5
:100060000C94ED180C94E2490C94D8490C94ED18BA
:100070000C94ED180C94ED180C94ED180C94ED18EC
:100080000C94ED180C94ED180C94ED180C94ED18DC
:100090000C94ED180C94ED180C94ED180C94ED18CC
:1000A0000C94ED180C94ED180C94ED180C94ED18BC
:1000B0000C94ED180C94ED180C94ED180C94ED18AC
:1000C0000C94ED180C94ED180C94ED180C94472E2C
:1000D0000C94112E0C94ED180C94ED180C94ED1852
:1000E0000C94ED18084AD73B3BCE016E84BCBFFD93
:1000F000C12F3D6C74319ABD56833DDA3D00C77FF8
:1001000011BED9E4BB4C3E916BAAAABE0000008090
:100110003F05A84CCDB2D44EB93836A9020C50B91F
:10012000918688083CA6AAAA2ABE000000803F004B
:100130000C9482F40C94B2FC0C94744A0C94E8F382
:100140000C94D22E0C94A5F30C94A64A0D9411068F
:100150000D9495060C94C3F40C94E4F30C94C1F83C
:100160000C945E4A0C94CDF40C9466F40C9456AA4C
:100170000C94CCF30C9440F40C94DAF30C94B7F395
:100180000D9409040C94563A0C9428AC0C9450AB82
:100190000C94852E0C946BAB0C944F4A0D94FC166A
:1001A0000C94E92E0C948CF40C9473AA0C94BFF369
:1001B0000D941A170C94AFF40C946EF40C942A3A24
:1001C0000C94F2F30D9488000D945C060C9433F4B7
:1001D0000C94A5F40C9431FB0C94F12E0C949E4AD3
:1001E0000C94ECF80D9474060C94F82E0C94ABA7B8
:1001F0000C94D7F70C94DEF30C940FFF0C942EA8FC
:100200000C94884A0C946D4A0C94A0F30D94190B2D
:100210000C94D92E0C94F2AC0C944AF40C94BBF3CD
:100220000D9455000C948C4A0C94D6F30D948806CA
:100230000C943BF40C94ED2E0C949BF40C94844A97
:100240000C94C3F30C94204A0C94ADF60C94934A8E
:100250000D946A060D946E070C94032F0C94ECF326
:100260000C94804A0C942DA80C94CF3A0D9441081C
:100270000C94E9AB0C9457FA0C94B9F40C9454F424
:100280000D9441060C9462380C94973A0C940B2F01
:100290000C945E380C94E12E0C94FBAB0C945EF441
:1002A0000C94E52E0C940F380C9478F40C94D0F345
:1002B0000C94C6F30C94B42E0C947C4A0C940CABA6
:1002C0000D947E070D9438060C94F6F30C94784A3E
:1002D0000C94DD2E0D943E060C94C32E0D94590300
:1002E0000C94EBAA4E414E494E495459494E46CDC5
:1002F000CCCC3D0AD7233C17B7D13877CC2B3295DD
:1003000095E6241FB14F0A000020410000C84200BA
:10031000401C4620BCBE4CCA1B0E5AAEC59D740084
:10032000407A10F35A00A0724E18090010A5D4E8C4
:100330000000E87648170000E40B54020000CA9A57
:100340003B000000E1F505000080969800000040A9
:10035000420F000000A086010000001027000000EE
:1003600000E803000000006400000000000A000034
:100370000000000100000000002C76D888DC674FE8
:100380000823DFC1DFAE59E1B1B796E5E3E453C618
:100390003AE651997696E8E6C28426EB898C9B6210
:1003A000ED407C6FFCEFBC9C9F40F2BAA56FA5F4BA
:1003B00090055A2AF75C936B6CF9676DC11BFCE0E2
:1003C000E40D47FEF520E6B500D0ED902E03009435
:1003D0003577050080841E080000204E0A000000CA
:1003E000C80C333333330F986E12831141EF8D21D4
:1003F00014893BE65516CFFEE6DB18D1844B381B3B
:10040000F77C1D901DA4BBE424203284725E2281FF
:1004100000C9F124ECA1E53D27434F4D4D554E4910
:10042000434154494F4E0044525952554E00455293
:10043000524F525300494E464F004543484F0045E6
:1004400072726F722077726974696E6720746F20A0
:10045000454550524F4D210A0053544F505045448A
:100460002E20005072696E7465722073746F707004
:1004700065642064756520746F206572726F727395
:100480002E2046697820746865206572726F72202C
:10049000616E6420757365204D39393920746F2081
:1004A000726573746172742E202854656D70657264
:1004B00061747572652069732072657365742E208E
:1004C0005365742069742061667465722072657367
:1004D00074617274696E67290A004E6F2043686503
:1004E000636B73756D2077697468206C696E652025
:1004F0006E756D6265722C204C617374204C696E50
:10050000653A20004E6F20436865636B73756D20FC
:1005100077697468206C696E65206E756D626572AE
:100520002C204C617374204C696E653A200063681E
:1005300065636B73756D206D69736D617463682C91
:10054000204C617374204C696E653A20004C696ED2
:1005500065204E756D626572206973206E6F742020
:100560004C617374204C696E65204E756D626572C6
:100570002B312C204C617374204C696E653A20003D
:100580004D3131300053657269616C207374617450
:100590007573206D69736D617463680A00776169B2
:1005A000740A0053442072656164206572726F7230
:1005B0000A002121204B494C4C206361757365640E
:1005C00020627920746F6F206D75636820696E6199
:1005D00063746976652074696D65202D206375727A
:1005E00072656E7420636F6D6D616E643A200048B1
:1005F0006F74656E642049646C652054696D656F25
:10060000757400486F74656E642049646C6520548D
:10061000696D656F75740A002A2A2A496E697469C2
:100620006E672063617264206973204F4B2A2A2A07
:10063000004D6564696120496E736572746564007C
:100640004D656469612052656D6F766564004D315A
:100650003030305300627573793A2070617573657C
:100660006420666F7220696E7075740A006275731B
:10067000793A2070617573656420666F72207573B6
:1006800065720A00627573793A2070726F636573E0
:1006900073696E670A002A2A2A6B696C6C2A2A2AF7
:1006A00000706F7765726F6666004B494C4C45442D
:1006B0002E20005072696E7465722068616C7465DA
:1006C000642E206B696C6C28292063616C6C6564F6
:1006D000210A006563686F3A004572726F723A00D2
:1006E0000A4D6561737572656420706F696E74730D
:1006F0003A0A00357835206D6573682E205A206FD0
:1007000066667365743A20002F2F616374696F6E9B
:100710003A00656E640053656E64204D31303820B8
:10072000746F20726573756D650A00496E7365722A
:10073000742066696C616D656E7420616E642073EF
:10074000656E64204D3130380A0052656865617409
:100750002066696E69736865642E0052656865611C
:100760007420446F6E6500526568656174696E67D8
:100770002E2E2E00526568656174004865617465AF
:10078000722054696D656F75740053656E64204DF9
:1007900031303820746F2068656174206E6F7A7A0A
:1007A0006C650A004E6F7A7A6C65205061726B65D9
:1007B0006400486F74656E6420746F6F20636F6CA3
:1007C000640A00706175736564005061757365003B
:1007D00050757267654D6F72650050617573656421
:1007E0000070726F6D70745F0073686F7700627570
:1007F00074746F6E00626567696E004C6F6164208F
:1008000046696C616D656E74004C6F616420466969
:100810006C616D656E74205400496E73657274204E
:1008200066696C616D656E7420616E642073656EBF
:1008300064204D3130380A00726573756D6564004F
:10084000526573756D696E670057616974696E678B
:1008500020666F72206865617475702E0A004C65A1
:100860006176696E6720473236003F537065636971
:100870006669656420582C5920636F6F7264696ED5
:10088000617465206F7574206F6620626F756E6489
:10089000732E0A003F2852296570656174207661C5
:1008A0006C7565206E6F7420706C61757369626C15
:1008B000653B206D757374206265206174206C65E2
:1008C00061737420312E0A003F28522965706561DA
:1008D00074206D757374206265207370656369663A
:1008E000696564207768656E206E6F742075736922
:1008F0006E6720616E204C43442E0A003F537065A2
:10090000636966696564206E6F7A7A6C65207465C8
:100910006D7065726174757265206E6F7420706C95
:1009200061757369626C652E0A003F537065636977
:10093000666965642066696C616D656E74207369B3
:100940007A65206E6F7420706C61757369626C6576
:100950002E0A003F53706563696669656420707292
:10096000696D65206C656E677468206E6F742070A9
:100970006C61757369626C652E0A003F5072696D17
:1009800065206C656E677468206D75737420626590
:1009900020737065636966696564207768656E2099
:1009A0006E6F74207573696E6720616E204C4344CE
:1009B0002E0A003F537065636966696564206E6F37
:1009C0007A7A6C652073697A65206E6F7420706C1A
:1009D00061757369626C652E0A003F5265747261BD
:1009E0006374696F6E204D756C7469706C696572A3
:1009F000206D757374206265207370656369666924
:100A000065642E0A003F53706563696669656420FA
:100A100052657472616374696F6E204D756C746990
:100A2000706C696572206E6F7420706C617573698B
:100A3000626C652E0A003F53706563696669656480
:100A4000206C6179657220686569676874206E6FD3
:100A50007420706C61757369626C652E0A0043299D
:100A60002E0A003F5370656369666965642062659C
:100A7000642074656D7065726174757265206E6F47
:100A80007420706C61757369626C65202834302D38
:100A900000473236207374617274696E672E2E2E91
:100AA0000A004F46460A004661646520486569674A
:100AB00068742000426564204C6576656C696E67D9
:100AC00020004661696C656420746F20656E616208
:100AD0006C6520426564204C6576656C696E670ABA
:100AE000004D65736820426564204C6576656C2016
:100AF000646174613A0A00496E76616C6964206DC4
:100B00006573682E0A00206E6F7420656E746572BE
:100B100065642E0A0050726F62696E6720506F69BB
:100B20006E740025532025692F256900206F6620EB
:100B3000004D424C2047323920706F696E7420009E
:100B4000290A004A206F7574206F662072616E67F3
:100B5000652028302D00290A0049206F7574206F08
:100B6000662072616E67652028302D004732384C50
:100B700030004D6573682070726F62696E67206423
:100B80006F6E65004D6573682070726F62696E6785
:100B900020646F6E652E0A005374617274206D6557
:100BA00073682070726F62696E672077697468205D
:100BB00022473239205331222066697273742E0A1B
:100BC000004732395332004732384C300A47323905
:100BD000533200686173206E6F20646174612E0A65
:100BE000004D65736820426564204C6576656C69CC
:100BF0006E67200053206F7574206F662072616EDF
:100C000067652028302D35292E0A004D6573682030
:100C1000706F696E74206F7574206F662072616EDC
:100C200067650A004D34323120696E636F727265F8
:100C3000637420706172616D657465722075736193
:100C400067650A00546F6F6C6368616E67653A0090
:100C500020204D32313700205700204C0020410029
:100C60002047002046002055002052002053003D20
:100C70003D4F6E506F7765724C6F7373526573752D
:100C80006D653D3D004D32342053256C6420542564
:100C90006C64004739322E392045257300473120D6
:100CA000462564004739322E39205A2573004731D2
:100CB000205A3020463230300047312058257320EA
:100CC00059257320463330303000473132004D34DF
:100CD000323020532569205A2573004D313036209B
:100CE00050256920532569005425692053004D3251
:100CF000303020542569204430004D3230302054AB
:100D0000256920442573004732385230585900472E
:100D100039322E39204530205A300A47315A25734E
:100D2000004D31303920532569004D313930205381
:100D30002569004D343230205330205A300020498C
:100D40006E76616C69642065787472756465722072
:100D50000047322F47332062616420706172616DF9
:100D600065746572730A00536C6565702E2E2E00D3
:100D70004D65736820706F696E74206F7574206F95
:100D8000662072616E67650A004D302053746F7083
:100D9000004D312053746F7000436F6E74696E752F
:100DA0006500436C69636B20746F20526573756DC9
:100DB000652E2E2E004E6F204D6F76652E00456EEF
:100DC000642066696C65206C6973740A004265670B
:100DD000696E2066696C65206C6973740A004E6FD9
:100DE000206D656469610A00526573756D696E678F
:100DF00020534400286E6F2066696C652900437596
:100E00007272656E742066696C653A200050726972
:100E10006E742074696D653A20000A5374617473AE
:100E20003A2046696C616D656E7420757365643A2D
:100E300020002C204C6F6E67657374206A6F623AD5
:100E40002000546F74616C2074696D653A20005302
:100E5000746174733A20002C204661696C65643AB1
:100E600020002C2046696E69736865643A20005042
:100E700072696E74733A200053746174733A20007F
:100E80006F6B006F6666003A0435042E0427041960
:100E90000444454255473A004D3131332053004216
:100EA000656420436F6F6C696E672E2E2E0042655D
:100EB000642048656174696E672E2E2E00544D3390
:100EC000442043522D58204F46462E002F2F0020FD
:100ED0005200416363656C65726174696F6E3A209C
:100EE00050005741524E494E4721204C6F77205AAF
:100EF000204A65726B206D6179206C656164207495
:100F00006F20756E77616E746564207061757365AE
:100F1000732E0A004D3230362058004F4646004F9F
:100F20004E0020204D61783A2000200020204D699D
:100F30006E3A2000536F667420656E6473746F7030
:100F4000733A200046523A0020466C6F773A2000F0
:100F50004261627973746570205A004D424C2041A1
:100F6000646A757374205A0020643A0020693A005C
:100F700020703A00496E76616C69642065787472FD
:100F8000756465720A0020643A0020693A00207096
:100F90003A0064697300656E0043290A0061626C5F
:100FA000656420286D696E2074656D702000436F44
:100FB0006C64206578747275646573206172652055
:100FC00000504944204175746F74756E6500504936
:100FD00044204175746F74756E65206661696C6537
:100FE00064212042616420686561746572206964CF
:100FF0000A004F666673657473204170706C696592
:1010000064004572723A20546F6F2066617221004D
:10101000546F6F206661722066726F6D2072656614
:101020006572656E636520706F696E740A00454570
:1010300050524F4D204F4B0A002E0A002028302DD1
:10104000313029002076616C7565206F7574206FD2
:10105000662072616E676500416476616E6365202B
:101060004B00506F7765722D6C6F737320726563E0
:101070006F7665727920004D383400446F6E6520BC
:101080007072696E74696E672066696C650A004DDE
:101090003737004D3331004361703A004D454154BC
:1010A0005041434B00434F4F4C45525F54454D50C8
:1010B00045524154555245004348414D4245525FC7
:1010C00054454D50455241545552450042414259B4
:1010D0005354455050494E470041524353004D4FE1
:1010E00054494F4E5F4D4F44455300544845524D6F
:1010F000414C5F50524F54454354494F4E004C4F62
:101100004E475F46494C454E414D45004155544F71
:101110005245504F52545F53445F535441545553BA
:101120000053445F5752495445005245504541547D
:10113000005344434152440050524F4D50545F536A
:101140005550504F525400454D455247454E435916
:101150005F50415253455200434153455F4C49470C
:1011600048545F4252494748544E45535300544FE8
:1011700047474C455F4C494748545300534F4654EA
:10118000574152455F504F574552004255494C44D4
:101190005F50455243454E54004C4556454C494ED0
:1011A000475F44415441005A5F50524F42450052FC
:1011B000554E4F5554004155544F4C4556454C00E3
:1011C0005052494E545F4A4F420050524F47524589
:1011D0005353004155544F5245504F52545F54455C
:1011E0004D5000564F4C554D4554524943004545CE
:1011F00050524F4D0042494E4152595F46494C456D
:101200005F5452414E534645520053455249414C5A
:101210005F584F4E5F584F4646004649524D574122
:1012200052455F4E414D453A4D61726C696E2032B8
:101230002E302E375F4457372E332E3120544D3306
:10124000442053534D444E4E202841707220323971
:1012500020323032312031333A35363A323129209A
:10126000534F555243455F434F44455F55524C3AA7
:1012700068747470733A2F2F6769746875622E638F
:101280006F6D2F496E73616E6974794175746F6DFE
:101290006174696F6E2F4D61726C696E2F74726527
:1012A000652F437265616C6974794477696E5F324A
:1012B0002E302050524F544F434F4C5F564552539F
:1012C000494F4E3A312E30204D414348494E455FFB
:1012D000545950453A544D33442043522D582045DB
:1012E000585452554445525F434F554E543A32205C
:1012F000555549443A63656465326132662D34312F
:1013000061322D343734382D396231322D63353521
:101310006336326633363766660A0043616E6E6F37
:1013200074206F70656E2073756264697220002589
:1013300069730025696D202569730025696820257A
:10134000696D202569730025696420256968202559
:10135000696D202569730025697920256964202538
:1013600069682025696D20256973003D3D447769D2
:101370006E20496E697420436F6D706C6574653DB5
:101380003D002A2A2A4E6F7A7A6C6554656D705337
:1013900074617475735B325D203D003D3D4865614D
:1013A00074696E6720446F6E65204368616E67657F
:1013B0002046696C616D656E743D3D00202073743C
:1013C00061727470726F677265737320003D3D7750
:1013D00061697477617920353D3D003D3D776169F4
:1013E0007477617920343D3D003D3D7761697477C4
:1013F000617920333D3D003D3D77616974776179C6
:1014000020313D3D003D3D6F6E5072696E745469F0
:101410006D657253746F707065643D3D003D3D6F46
:101420006E466163746F727952657365743D3D00F9
:10143000270A0A0000272027002027002D006E6FB2
:1014400074696669636174696F6E200063616E63BD
:10145000656C005072696E742041626F72746564CD
:10146000004469736D6973730055492041626F725E
:1014700074656400726573756D65002A2A2A43508D
:101480006C617920546F6E652A2A2A005761726E4A
:10149000696E673A20436C65616E20436972636CC4
:1014A000652072657175697265732058590A005715
:1014B00061726E696E673A20526164697573204F7C
:1014C0007574206F662052616E67650A004E6F7AF0
:1014D0007A6C6520746F6F20636F6C64202D2053CD
:1014E0006B697070696E6720776970650A003D3DB1
:1014F0006F6E5072696E7454696D65725061757368
:1015000065643D3D00486F6D696E67204661696C9A
:101510006564006F70656E005452494747455245F7
:1015200044003A20007A5F6D696E00795F6D696EE4
:1015300000785F6D696E005265706F7274696E67D6
:1015400020656E6473746F70207374617475730AB0
:101550000000809D4300009A430000C84300000043
:1015600000000000000000000020746F6F206C6F0E
:101570006E6720657874727573696F6E207072651E
:1015800076656E7465640A0020636F6C642065780C
:1015900074727573696F6E2070726576656E7465AE
:1015A000640A000000000000000000000000005776
:1015B00061726E696E673A20486F6D696E6720428E
:1015C000756D702044697669736F72203C20310A12
:1015D0000002020400809D4300009A430000C843BB
:1015E0000000004100000041000000400000000138
:1015F000000000010000800055555500000040002B
:1016000033333300AAAA2A004992240000002000A4
:10161000C7711C0099991900D1451700555515003F
:101620003BB11300244912001111110000001000F9
:101630000F0F0F00E3380E0043790D00CCCC0C00E7
:10164000C3300C00E8A20B0064210B00AAAA0A0018
:10165000703D0A009DD80900427B090092240900D0
:10166000DCD3080088880800104208000000080049
:10167000F0C107008787070075500700711C07003D
:101680003EEB0600A1BC06006990060066660600F7
:10169000703E06006118060017F4050074D10500BD
:1016A0005BB00500B290050062720500555505005B
:1016B00078390500B81E0500050505004EEC04004C
:1016C00087D40400A1BD040090A70400499204003F
:1016D000C17D0400EE690400C756040044440400C0
:1016E0005C320400082104004110040000000400E2
:1016F0003FF00300F8E0030026D20300C3C3030059
:10170000CCB503003AA803000A9B0300388E0300FF
:10171000C08103009F750300D0690300505E030081
:101720001D53030034480300913D0300333303008D
:1017300016290300381F030097150300300C03001F
:10174000030303000BFA020049F10200BAE80200A9
:101750005CE002002DD802002DD0020059C8020022
:10176000B0C0020031B90200DAB10200AAAA020038
:10177000A0A30200BC9C0200FA9502005C8F02004C
:10178000DF88020082820200457C02002776020088
:1017900027700200436A02007C640200D05E0200EF
:1017A0003F590200C8530200FFFDFCFAF8F6F4F2BC
:1017B000F0EEECEAE9E7E5E3E1E0DEDCDAD9D7D503
:1017C000D4D2D0CFCDCBCAC8C7C5C3C2C0BFBDBCA1
:1017D000BAB9B7B6B4B3B2B0AFADACAAA9A8A6A512
:1017E000A4A2A1A09E9D9C9A99989795949392905B
:1017F0008F8E8D8B8A8988878684838281807F7E85
:101800007D7B7A797877767574737271706F6E6D8F
:101810006C6B6A696867666564636261605F5E5D80
:101820005C5B5A5958585756555453525150504F63
:101830004E4D4C4B4A4A494847464645444342422E
:1018400041403F3E3E3D3C3B3B3A393838373635E8
:1018500035343332323130302F2E2E2D2C2B2B2A93
:101860002929282727262525242323222121202032
:101870001F1E1E1D1C1C1B1B1A19191818171616C3
:10188000151514131312121111100F0F0E0E0D0D4A
:101890000C0C0B0A0A0909080807070606050504C7
:1018A000040303020201000020746F6F206C6F6E4E
:1018B0006720657874727573696F6E2070726576D3
:1018C000656E7465640A0020636F6C6420657874CB
:1018D000727573696F6E2070726576656E7465647B
:1018E0000A003D3D6F6E5072696E7454696D657289
:1018F000537461727465643D3D003D3D6F6E537479
:101900006F726553657474696E67733D3D003D3D4C
:101910006F6E436F6E66696775726174696F6E533F
:10192000746F72655772697474656E3D3D005365DE
:101930007474696E67732053746F726564000A2053
:10194000696E6974207A70726F62655F7A6F66661D
:10195000736574203D20003D3D6F6E436F6E666978
:101960006775726174696F6E53746F7265526561E9
:10197000643D3D00454550524F4D20496E697469A4
:10198000616C697A65640A003B200020204D363086
:10199000332000546F6F6C2D6368616E67696E67EA
:1019A0003A002055005431204C002055005430207E
:1019B0004C0046696C616D656E74206C6F61642FBC
:1019C000756E6C6F6164206C656E677468733A0045
:1019D000204B0020204D3930302054004C696E657A
:1019E000617220416476616E63653A0020204D3457
:1019F0003133205300506F7765722D4C6F73732015
:101A00005265636F766572793A0020440020490080
:101A100020204D3330342050002044002049002045
:101A2000204D333031205000504944207365747488
:101A3000696E67733A002020473239205334205AA8
:101A400000204A002020473239205333204900200B
:101A5000204D3432302053004D6573682042656458
:101A6000204C6576656C696E673A0020204D3230F7
:101A700036205800486F6D65206F66667365743A4E
:101A80000020580020530020204D323035204200E5
:101A9000416476616E6365643A20423C6D696E5FB5
:101AA0007365676D656E745F74696D655F75733EB0
:101AB00020533C6D696E5F66656564726174653E56
:101AC00020543C6D696E5F74726176656C5F66650B
:101AD0006564726174653E20583C6D61785F785F23
:101AE0006A65726B3E20593C6D61785F795F6A650B
:101AF000726B3E205A3C6D61785F7A5F6A65726BEB
:101B00003E20453C6D61785F655F6A65726B3E00A3
:101B100020540020520020204D323034205000410B
:101B20006363656C65726174696F6E2028756E6998
:101B300074732F7332293A20503C7072696E745F4F
:101B4000616363656C3E20523C72657472616374BC
:101B50005F616363656C3E20543C74726176656CB2
:101B60005F616363656C3E0020204D323031205848
:101B7000004D6178696D756D20416363656C6572B8
:101B80006174696F6E2028756E6974732F733229C2
:101B90003A0020204D3230332058004D6178696D75
:101BA000756D206665656472617465732028756E55
:101BB0006974732F73293A005374657073207065CC
:101BC0007220756E69743A0020204D3230302053F7
:101BD0000020440020204D32303020540020446941
:101BE0007361626C65640A0046696C616D656E7450
:101BF0002073657474696E67733A0020286D6D29CF
:101C0000002020473231202020203B20556E69746F
:101C10007320696E206D6D003D3D6F6E4C6F616489
:101C200053657474696E67733D3D000000FA4300AC
:101C300000FA4300002041000096420000A042004C
:101C400000A0420000C8430000BE42DC050000DCEA
:101C5000050000640000004B00000024F4D4305064
:101C6000C38E20C2A24017828B7011127A910D810F
:101C70006CD90AA861E108C7586607615143061E7E
:101C80004B5D05C145A7041A411104093D98037134
:101C90003931034036DB0265339102D4305402807F
:101CA0002E1D02632CEE01752AC501B028A001107B
:101CB0002781018F2564012B244B01E0223401ACE4
:101CC000211F018D200D01801FFC00841EED009757
:101CD0001DDF00B81CD200E61BC600201BBC006440
:101CE0001AB200B219A8000A19A0006A189900D106
:101CF00017910040178B00B516840031167E00B393
:101D00001579003A157300C7146F0058146A00EE75
:101D10001366008813630025135E00C7125B006C16
:101D200012570015125400C111510070114F0021BB
:101D3000114B00D61049008D104700461044000298
:101D4000104200C00F4000800F3E00420F3C0006D2
:101D50000F3B00CB0E3800930E37005C0E3500278A
:101D60000E3400F30D3200C10D3100900D300060D3
:101D70000D2E00320D2D00050D2C00D90C2B00AEC0
:101D80000C2900850C29005C0C2700350C27000E5F
:101D90000C2600E80B2400C40B2400A00B23007DBC
:101DA0000B23005A0B2100390B2100180B2000F8DF
:101DB0000A1F00D90A1E00BB0A1E009D0A1D0080D2
:101DC0000A1D00630A1C00470A1B002C0A1B001195
:101DD0000A1A00F7091A00DD091900C4091900AB35
:101DE000091900920917007B091800630917004CB4
:101DF00009160036091600200916000A091500F513
:101E0000081500E0081400CC081400B8081400A459
:101E1000081400900813007D0812006B0813005886
:101E2000081200460812003408110023081100129D
:101E300008110001081100F0071000E0071000D0A1
:101E4000071000C0071000B0070F00A10710009195
:101E5000070E0083070F0074070F0065070E005779
:101E6000070E0049070E003B070D002E070E00204D
:101E7000070D0013070D0006070D00F9060C00ED15
:101E8000060D00E0060C00D4060C00C8060C00BCD1
:101E9000060C00B0060C00A4060B0099060C008D81
:101EA000060B0082060B0077060B006C060B006128
:101EB000060A0057060B004C060A0042060A0038C4
:101EC000060A002E060A0024060A001A060A001056
:101ED00006090007060A00FD050900F4050900EBE4
:101EE000050900E2050900D9050900D0050900C768
:101EF000050900BE050900B5050800AD050800A5E7
:101F00000509009C050800940508008C050800845C
:101F10000508007C050800740508006C05070065CD
:101F20000508005D050700560508004E0507004737
:101F30000507004005080038050700310507002A9D
:101F4000050700230507001C050600160507000FFE
:101F50000507000805060002050700FB040600F55A
:101F6000040700EE040600E8040600E2040700DBB4
:101F7000040600D5040600CF040600C9040600C309
:101F8000040600BD040600B7040600B1040500AC59
:101F9000040600A6040600A00405009B04060095A4
:101FA000040500900406008A0405008504050080ED
:101FB0000406007A04050075040500700405006B32
:101FC00004050066040500610405005C0405005773
:101FD000040500520405004D0405004804050043B3
:101FE0000405003E0404003A0405003504050030F1
:101FF0000404002C04050027040400230405001E2B
:102000000404001A04040016040500110404000D61
:10201000040400090405000404040000040400FC96
:10202000030400F8030400F4030400F0030400ECCC
:10203000030400E8030400E4030400E0030400DCFC
:10204000030400D8030400D4030400D0030400CC2C
:10205000030400C8030300C503030024F404D920CB
:102060001BC40C5C0E9804C4095F0265077101F47F
:1020700005F900FB04B30048048700C10369005858
:1020800003550003034500BE023A008402310053A9
:10209000022A002902250004022000E4011C00C8D5
:1020A000011900AF01170098011400840113007199
:1020B0000110006101100051010E0043010D0036B6
:1020C000010B002B010B0020010B00150109000C76
:1020D00001090003010800FB000800F3000800EB01
:1020E000000700E4000600DE000600D8000600D26B
:1020F000000600CC000500C7000500C2000500BDB9
:10210000000400B9000400B5000400B1000400ADF3
:10211000000400A9000400A5000300A20003009F22
:102120000004009B00030098000300950002009348
:10213000000300900003008D0002008B0003008864
:102140000002008600020084000300810002007F7C
:102150000002007D0002007B00020079000200778F
:10216000000100760002007400020072000100719C
:102170000002006F0002006D0001006C0002006AA6
:1021800000010069000200670001006600010065AF
:1021900000010064000200620001006100010060B3
:1021A0000001005F0002005D0001005C0001005BB7
:1021B0000001005A000100590001005800010057B9
:1021C00000010056000100550001005400010053B9
:1021D00000000053000100520001005100010050B6
:1021E0000001004F0001004E0000004E0001004DB4
:1021F0000001004C0001004B0000004B0001004AB0
:1022000000010049000100480000004800010047AB
:1022100000010046000000460001004500000045A6
:10222000000100440001004300000043000100429F
:102230000000004200010041000000410001004098
:102240000001003F0000003F0001003E0000003E92
:102250000001003D0000003D0001003C0000003C8A
:102260000000003C0001003B0000003B0001003A80
:102270000000003A00010039000000390001003878
:10228000000000380000003800010037000000376F
:102290000001003600000036000000360001003565
:1022A000000000350000003500010034000000345B
:1022B0000000003400010033000000330000003350
:1022C0000001003200000032000000320001003145
:1022D000000000310000003100010030000000303B
:1022E000000000300001002F0000002F0000002F30
:1022F0000000002F0001002E0000002E0000002E24
:102300000001002D0000002D0000002D0000002D18
:102310000001002C0000002C0000002C0000002C0C
:102320000001002B0000002B0000002B0000002B00
:102330000001002A0000002A0000002A0000002AF4
:1023400000010029000000290000002900000029E8
:1023500000000029000100280000002800000028DB
:1023600000000028000000280001002700000027CE
:1023700000000027000000270000002700010026C1
:1023800000000026000000260000002600000026B5
:1023900000010025000000250000002500000025A8
:1023A000000000250000002500010024000000249A
:1023B000000000240000002400000024000100238D
:1023C0000000002300000023000000230000002381
:1023D0000000002300000023000100220000002272
:1023E0000000002200000022000000220000002265
:1023F0000001002100000021000000210000002158
:102400000000002100000021000000210001002048
:10241000000000200000002000000020000000203C
:102420000000002000000020000000200001001F2C
:102430000000001F0000001F0000001F0000001F20
:102440000000001F0000001F0001001E0000001E11
:102450000000001E0000001E000000232C0000B839
:10246000220000561800003A0F0000B8080000B122
:10247000040000710200003E01000020436F756EF1
:102480007420583A0023646566696E6520444546A9
:1024900041554C545F0000626564004B6420004B62
:1024A0006920004B702000504944204175746F74BE
:1024B000756E652066696E69736865642120507564
:1024C0007420746865206C617374204B702C204BF1
:1024D0006920616E64204B6420636F6E7374616E5B
:1024E00074732066726F6D2062656C6F7720696E01
:1024F000746F20436F6E66696775726174696F6E81
:102500002E680A00504944204175746F74756E65D9
:10251000206661696C6564212074696D656F7574EE
:102520000A00504944204175746F74756E652066C9
:1025300061696C6564212054656D706572617475A4
:10254000726520746F6F20686967680A00204B64A9
:102550003A2000204B693A2000204B703A2000209E
:10256000436C617373696320504944200A00204E14
:102570006F206F76657273686F6F740A00205475F0
:102580003A2000204B753A2000206D61783A2000F7
:10259000206D696E3A200020643A20002062696153
:1025A000733A2000504944204175746F74756E650C
:1025B0002073746172740A00504944204175746F2D
:1025C00074756E65206661696C6564212054656D63
:1025D000706572617475726520746F6F20686967C9
:1025E000680A0042656400453100626564002C2081
:1025F00073797374656D2073746F707065642120D6
:102600004865617465725F49443A200048656174A9
:10261000696E67204661696C65640048656174692C
:102620006E67206661696C6564004D3131322053FC
:10263000687574646F776E001000C90210012C0178
:102640004001220170011801B0010E01F0010401E6
:102650005002FA00B002F0003003E600D003DC00C4
:102660009004D2007005C800A006BE000008B400A7
:10267000B009AA00D00BA000600E960060118C007B
:102680000015820020197800C01D6E00A022640091
:10269000B0275A00902C500000314600E0343C0036
:1026A00010383200903A2800603C1E00A03D140013
:1026B000803E0A00203F0000544845524D414C20C6
:1026C00052554E4157415900546865726D616C20F6
:1026D00052756E61776179004572723A204D4158AA
:1026E00054454D50004D415854454D502074726929
:1026F000676765726564004572723A204D494E54B1
:10270000454D50004D494E54454D502074726967F7
:10271000676572656400202F002042403A00204027
:102720003A0020573A0020573A00496E76616C69AA
:10273000642065787472756465720A004163746917
:1027400076652045787472756465723A2000486F2A
:1027500074656E6420746F6F20636F6C640A007C14
:102760003C3E5E2B3D3F2F5B5D3B2C2A225C0043B1
:10277000616E6E6F74206F70656E20737562646930
:10278000722000534420496E6974204661696C00D0
:1027900053442063617264206F6B0A006F70656E32
:1027A000526F6F74206661696C65640A00766F6CA5
:1027B000756D652E696E6974206661696C65640A61
:1027C000004E6F20534420636172640A000A4D3248
:1027D00034004D3233202573002E0A006F70656E71
:1027E000206661696C65642C2046696C653A20003E
:1027F00046696C652073656C65637465640A0020C6
:1028000053697A653A200046696C65206F70656E81
:1028100065643A2000454E4420535542524F55546A
:10282000494E450A002220706F73002220706172A9
:10283000656E743A2200535542524F5554494E45E5
:102840002043414C4C207461726765743A220053F6
:10285000756263616C6C204F766572666C6F770091
:102860004578636565646564206D617820535542E1
:10287000524F5554494E452064657074683A002E95
:102880000A0044656C6574696F6E206661696C65E9
:10289000642C2046696C653A200046696C652064AA
:1028A000656C657465643A005344207072696E7497
:1028B000696E67206279746520004E6F74205344FE
:1028C000207072696E74696E670A00577269746964
:1028D0006E6720746F2066696C653A2000667265C9
:1028E000736800646F696E67002066696C653A20E2
:1028F000004E6F7720002F6175746F25632E67007F
:102900002020506C616E6E6572427566666572421B
:10291000797465733A20002046726565204D656DB7
:102920006F72793A2000436F6D70696C65643A206C
:1029300041707220323920323032310A00204C612D
:10294000737420557064617465643A20323032319A
:102950002D30342D3138207C20417574686F723AE7
:102960002054696E794D616368696E657333440AFA
:1029700000322E302E375F4457372E332E310A0067
:102980004D61726C696E0020536F66747761726579
:102990002052657365740A00205761746368646F20
:1029A000672052657365740A002042726F776E204B
:1029B0006F75742052657365740A002045787465DC
:1029C000726E616C2052657365740A00506F776592
:1029D0007255700A0073746172740A004739310AC3
:1029E00047315A350A4739300A4D38340A4D3130AB
:1029F0003453300A4D3134305330004D31303031A2
:102A0000006572726F722077726974696E672074E4
:102A10006F2066696C650A00446F6E65207361768D
:102A2000696E672066696C652E0A004D3239004573
:102A30006E6473746F7073002553202563202563C3
:102A400020256320256300205A3A0020593A0020AF
:102A5000583A00656E6473746F7073206869743AD5
:102A6000200070012C0190012701B0012201C0015A
:102A70001D01F00118011002130130020E01600265
:102A8000090190020401C002FF000003FA004003A4
:102A9000F5008003F000D003EB002004E600700492
:102AA000E100E004DC004005D700C005D20040068C
:102AB000CD00D006C8008007C3003008BE00F00873
:102AC000B900C009B400B00AAF00B00BAA00D00C26
:102AD000A500000EA000500F9B00C01096005012E1
:102AE000910000148C00C0158700B0178200B01947
:102AF0007D00D01B7800001E730040206E009022E5
:102B00006900F024640040275F0090295A00E02B00
:102B10005500102E500020304B0010324600E0339C
:102B2000410090353C001037370070383200A03932
:102B30002D00B03A2800A03B2300603C1E00103D51
:102B40001900903D1400103E0F00703E0A00C03E78
:102B50000500003F0000403FFBFF803FF6FFC03F05
:102B6000F1FF00000A0B02090C0D0E080703040117
:102B70000000000000000000000000000000000055
:102B80000000000000000000000000000000121122
:102B90001000000000000000000000000000000025
:102BA0000000000000000000FFFFFF486F6D65207F
:102BB000257325732573204669727374003D3D6F3C
:102BC0006E55736572436F6E6669726D526571758D
:102BD000697265643D3D00220A00556E6B6E6F7729
:102BE0006E20636F6D6D616E643A2022002042009A
:102BF0002050006F6B00204500205A002059002013
:102C00004D393220580020453A00205A3A002059C8
:102C10003A00583A0043616E6E6F7420656E7465B9
:102C200072207375626469723A20004D323520500B
:102C30000A4D323400526573756D65005549205058
:102C400061757365004E6F204D61746368203A00B2
:102C50004D32320A4D32310052656672657368003A
:102C600050675570005067446F776E004973204677
:102C7000696C6520004973204469722000476F55D4
:102C80007044697200486173204D65646961004653
:102C9000696C656E616D652053656C656374656410
:102CA000004D3130303043004D3130303000466916
:102CB0006C616D656E7420537461742030202D201A
:102CC000330046696C616D656E74205374617420C5
:102CD00030202D20320046696C616D656E74205382
:102CE0007461742030202D2031002046696C616DA4
:102CF000656E7420526573706F6E7365204E6F0041
:102D0000526573756D652059657320647572696EBF
:102D100067207072696E74000A204E6F2046696CDD
:102D2000616D656E7400496E76616C6964204F70E8
:102D300074696F6E004D3530300053746F726520CA
:102D400053657474696E677300426564205049442A
:102D50002053746172746564004D3939390A4D32FB
:102D6000383050305331363000424C546F75636800
:102D7000205265736574004D3530320A4D35303060
:102D800000496E697420454550524F4D00486F749C
:102D9000656E642050494420537461727465640008
:102DA000456E676C69736820416C72656164792057
:102DB000536574004368696E657365204E6F7420B7
:102DC000537570706F7274656400496E4C616E6704
:102DD00043686F696365000A202A2A2A7265636462
:102DE00061742E646174615B305D203D0047323850
:102DF0000A4731204631303030205A313000556E8C
:102E0000737570706F72746564204F7074696F6E43
:102E10002053656C65637465640047323652323501
:102E20003500473238004731204631303030205AA3
:102E3000302E30004732380A4731204631303030AA
:102E4000205A302E30004D353030005A204F666603
:102E5000736574203A202573004D353030005A20B8
:102E60004F6666736574203A202573004732380A2E
:102E7000473146313530305A302E30004732385ADB
:102E80000A473146313530305A302E30004D383413
:102E900000473146313030305A302E30004732381A
:102EA0000A473146313030305A302E30004D616E95
:102EB00075616C53657454656D700052657175650C
:102EC00073746564204F6666736574204265796F1C
:102ED0006E64204C696D697473005A204F66667386
:102EE0006574203A20257300526F756E64696E67B1
:102EF00020746F207374657000526571756573740A
:102F00006564204F6666736574200053746F70208B
:102F10005472696767657265640053746F70204E00
:102F20006F0053746F705072696E740048616E6404
:102F30006C6520446174612041646A757374203249
:102F40002053657474696E672053637265656E20E3
:102F50000048616E646C6520446174612050726940
:102F60006E7446696C6520332053657474696E67AE
:102F70002053637265656E200048616E646C652045
:102F800044617461205072696E7446696C652032C8
:102F90002053657474696E672053637265656E2093
:102FA000004D38340048616E646C65204461746182
:102FB000205072696E7446696C6520506F7374009E
:102FC00048616E646C652044617461205072696E62
:102FD0007446696C652050726500426567696E537E
:102FE0007769746368003D3D20436865636B6B657A
:102FF000793D3D007265636461742E616464722082
:103000003D3D007265636461742E646174615B3080
:103010005D203D3D0077616974776179203D3D0019
:1030200020202A2A2A2A2A2A2A5254535F48616ECB
:10303000646C65446174612A2A2A2A2A2A2A2A2071
:1030400000526573656E643A20000000220025007E
:1030500028002B002E003100340002010000050181
:1030600008010B0100002100240027002A002D0088
:103070003000330001010000040107010A010505C9
:103080000505070508080808020202020A0A0808DE
:10309000040404040101010101010101030303030C
:1030A00003030303040707070C0C0C0C0C0C0C0C9B
:1030B0000202020206060606060606060B0B0B0BAC
:1030C0000B0B0B0B010210202008081020401020D1
:1030D00040800201020108040201010204081020DC
:1030E00040808040201008040201800402018040DA
:1030F0002010080402010804020101020408102043
:1031000040800102040810204080436F6F6C696E9C
:10311000672E2E2E0048656174696E672E2E2E0074
:103120004520255300544D33442043522D582052FE
:10313000656164792E005072696E74696E672E2E17
:103140002E005072696E7420506175736564006E54
:103150006F74696669636174696F6E2000504944D9
:103160002054756E652046696E6973686564004D0C
:1031700032340000D800CE0011241FBECFEFD1E2C0
:10318000DEBFCDBF00E00CBF13E0A0E0B2E0ECE496
:10319000F1E502E00BBF02C007900D92AC3FB10712
:1031A000D9F726E1ACEFB3E001C01D92AB37B2070F
:1031B000E1F718E1CBEBD8E100E006C02197010967
:1031C000802FFE010F94C724CA3BD10780E0080777
:1031D000A9F70F9436120D9494280C9400009F9236
:1031E000AF92BF92CF92DF92EF92FF920F931F9315
:1031F000CF93DF9300D01F921F92CDB7DEB7E8EADE
:10320000F7E10027BB27462F572FA82FAA2341F409
:10321000A52F542FB85FAA2319F4A52F5527B85FFF
:10322000A03138F45295A295452F4F70507FA42BB2
:10323000BC5FA03428F4550FAA1F550FAA1FBE5F0C
:10324000A03818F4550FAA1FB395550FAA1FEA0FFF
:10325000F01F449151E0AA27B85081F1C8F0B0FFA7
:1032600002C0440F551FB1FF04C0440F551F440F47
:10327000551FB2FF06C052954295142F1F70407F14
:10328000512BB3FF1BC0A52F542F44270C945E195C
:10329000B195B0FF02C055954795B1FF04C0559553
:1032A000479555954795B2FF05C05295407F429589
:1032B000452B5F70B3FF02C0452F5527DD24CC247A
:1032C000BB24B2E0649FD018C108B00AB00B749F51
:1032D000C018B108B00B849FB018B109659FC01821
:1032E000B108B00B759FB018B109859FB0196A9FDE
:1032F000B018B1097A9FB0194D9DA12C992433279C
:10330000992722275D9DA00C911C301F901F201F24
:10331000AD9D900C311D901F201F4C9DA00C911C49
:10332000301F901F201F5C9D900C311D901F201F8F
:10333000AC9D300D911D201F4B9D900C311D901F99
:10334000201F5B9D300D911D201FAB9D900D211DF9
:103350004B9F300D911D201F5B9F900D211DAB9F3A
:10336000200DB1E0BB24CC24DD24639FD018C1081C
:10337000B00AB00B739FC018B108B00B839FB01890
:10338000B109699FC018B108B00B799FB018B10995
:10339000899FB019629FB018B109729FB019D61AEF
:1033A000C70AB80A20F0B1E03B0F901F201F11247C
:1033B000792F632F90E0822F0F900F900F900F9036
:1033C0000F90DF91CF911F910F91FF90EF90DF90C1
:1033D000CF90BF90AF909F900895AF92BF92CF9241
:1033E000DF92EF92FF920F931F93CF93DF93C8E882
:1033F000DCE002E715E088E9A82E8CE0B82EC12CAD
:10340000D12C7601C39469917991899199910F9406
:10341000031E288939894A895B890F94641E0F9499
:103420004F26F80161937193819391938F01C61692
:10343000D706E806F90610F46B017C01AC16BD0650
:1034400011F76FEF7FEFCB01A70196010F94422494
:10345000209382053093830540938405509385051E
:10346000DF91CF911F910F91FF90EF90DF90CF9060
:10347000BF90AF9008957F928F929F92AF92BF922C
:10348000CF92DF92EF92FF920F931F93CF93DF9330
:1034900070905F0BC5E6D5E096E3C92E92E0D92E79
:1034A00026E1E22E22E0F22E07E51BE0772009F468
:1034B0005EC0F80180809180A280B38020E030E07F
:1034C000A901C501B4010F94FE1D882309F44FC062
:1034D00020E030E040E05FE3C501B4010F94641EDA
:1034E0009B01AC010F94641E2BED3FE049E450E4D6
:1034F0000F94641E9B01AC0160E070E080E89FE3E4
:103500000F94D6254B015C0189929992A992B992A8
:10351000F601619171916F01072E000C880B990BD8
:103520000F94051E2AE037ED43E25CE30F94641E1E
:10353000A50194010F94641EF70161937193819327
:1035400091937F010C5F1F4FF5E0CD36DF0709F047
:10355000ADCFDF91CF911F910F91FF90EF90DF9052
:10356000CF90BF90AF909F908F907F900895812CC7
:10357000912C80E8A82E8FE3B82EC6CF0F931F930F
:10358000CF93DF9350E0FC01E40FF51F8081440FDF
:10359000551F440F551F435A5A4FEA01882329F1FA
:1035A00088819981AA81BB81EB01088119812A81D7
:1035B0003B810097A105B10569F40C591F4F2F4FAE
:1035C0003F4FDA010D931D932D933C9313978FEF8B
:1035D000808306C0081B190B2A0B3B0B37FDF7CF66
:1035E000DF91CF911F910F910895188219821A824D
:1035F0001B82F6CF2F923F924F925F926F927F92F3
:103600008F929F92AF92BF92CF92DF92EF92FF92F2
:103610000F931F93CF93DF93CDB7DEB764970FB6A9
:10362000F894DEBF0FBECDBF7A8B698BDC018D9025
:103630009D90AD90BC90139714962D913D914D9116
:103640005C9117972D833E834F83588720E030E0AD
:1036500040EA51E4C501B4010F94DB2421EC3FE0C2
:103660004CE75CE30F94641E0F94482664300CF41E
:1036700027C163E0E62E660FFF08F701EE0FFF1F7C
:10368000EE0FFF1FE059FB4E408051806280738037
:103690001701BFEF2B1A3B0A20E030E040EA51E46B
:1036A0006D817E818F8198850F94DB2421EC3FE032
:1036B0004CE75CE30F94641E0F94482664300CF4CE
:1036C00003C163E0062F660F110BF801EE0FFF1F19
:1036D000EE0FFF1FE059FB4E208131814281538163
:1036E00029833A834B835C83A8014F5F5F4F5C8BD8
:1036F0004B8BA5E0AE9DC001AF9D900D11249A8724
:103700008987FC01E00FF11FEE0FFF1FEE0FFF1F77
:10371000E251F54FC080D180E280F380F101EE0FDD
:10372000FF1FEE0FFF1FE059FB4EA30192016081C6
:103730007181828193810F94DB246B877C878D87D5
:103740009E87A3019201C501B4010F94DB242B01D4
:103750003C0125E0229DF001239DF00D1124F88B02
:10376000EF87E00FF11FEE0FFF1FEE0FFF1FE2517B
:10377000F54FA701960160817181828193810F9439
:10378000DB242B853C854D855E850F94D625A301D2
:1037900092010F94641EA70196010F94DC246B0123
:1037A0007C01E985FA854B895C89E40FF51FEE0FF2
:1037B000FF1FEE0FFF1FE251F54F80809180A28026
:1037C000B380EF85F889E40FF51FEE0FFF1FEE0FB2
:1037D000FF1FE251F54FA501940160817181828143
:1037E00093810F94DB242B853C854D855E850F945A
:1037F000D625A30192010F94641EA50194010F9494
:10380000DC24A70196010F94DB244B015C01EB89BA
:10381000FC89EE0FFF1FEE0FFF1FE059FB4E2981C1
:103820003A814B815C8160817181828193810F94A7
:10383000DB249B01AC01C501B4010F94D6254B01DB
:103840005C0129813A814B815C816D817E818F8110
:1038500098850F94DB249B01AC01C501B4010F9442
:10386000641EA70196010F94DC24A989BA892D91C1
:103870003D914D915C910F94641E2091F708309119
:10388000F8084091F9085091FA080F94DC246496E6
:103890000FB6F894DEBF0FBECDBFDF91CF911F9161
:1038A0000F91FF90EF90DF90CF90BF90AF909F90DF
:1038B0008F907F906F905F904F903F902F900895E2
:1038C00067FFD8CE60E0D6CE67FFFCCE60E0FACED0
:1038D0008F929F92AF92BF92CF92DF92EF92FF9220
:1038E000CF93DF93EC018090370C9090380CA09030
:1038F000390CB0903A0C20E030E0A901C501B401C8
:103900000F94FE1D882309F454C0C880D980EA8032
:10391000FB80A7019601C501B4010F94FE1D181686
:103920000CF04CC020912F0C3091300C4091310C98
:103930005091320CC701B6010F94FE1D882331F15E
:10394000C0922F0CD092300CE092310CF092320CDD
:103950002091330C3091340C4091350C5091360C41
:10396000688179818A819B810F94641E9B01AC01DF
:1039700060E070E080E89FE30F94DB2460930E0228
:1039800070930F02809310029093110260910E02C7
:1039900070910F028091100290911102DF91CF91EE
:1039A000FF90EF90DF90CF90BF90AF909F908F905F
:1039B000089560E070E080E89FE3F0CF60E070E0A1
:1039C000CB01ECCFCF93DF9324E0829FC001112481
:1039D000EC01C55CD34FFC01E459F44F805A944F7D
:1039E000DC012D913D914D915C91608171818281CD
:1039F00093810F94DC24688379838A839B83DF918E
:103A0000CF91089580919B1290919C12891B877091
:103A100089F48091080E81110DC0809164129091FB
:103A20006512892B39F481E09091070A911103C046
:103A300080E0089581E00895CF93DF93DB01F901E1
:103A40009C919130C1F0943080F094509C938830D8
:103A5000D1F480819181009771F0019791838083E7
:103A6000480F591FEA01188206C08C3539F49C5F53
:103A70009C93943041F4DF91CF9108958B3339F7C3
:103A800081E08C93F8CF20813181B9016F5F7F4F46
:103A900071836083420F531FEA0188838081918183
:103AA0008F3591056CF7E7CF0F931F9381E000915D
:103AB0008B1410918C1420918D1430918E144091A0
:103AC0008714509188146091891470918A14041796
:103AD00015072607370708F480E01F910F91089516
:103AE00090E080E00895282F9091540B833021F4CA
:103AF00095FD0FC094FD0FC0892F90E0B0E0A0E0CD
:103B000004C0B695A795979587952A95D2F78170A9
:103B1000089581E0089580E008952FEB280F2A3161
:103B200008F047C0E22FF0E0809104059091050570
:103B3000A0910605B091070504C0B695A795979585
:103B400087952A95D2F780FD02C081700895E651CD
:103B5000FB4FE081EE2341F18091E80A9091E90A60
:103B6000E80FF92FF11D808190ED980F9A3030F019
:103B70008E3251F4818180538A3098F4F093D404CA
:103B8000E093D30481E008958D3211F08B3249F433
:103B9000818190ED980F9A3088F38E3211F48281F2
:103BA000EACFF0E0E0E0EACF1092D4041092D30420
:103BB000E9CF80E008950E948D1D882341F081E0C7
:103BC0002091D3043091D404232B09F480E008958C
:103BD000129A479A08955F9A8091870C8E7F8093FE
:103BE000870C8A9A8091870C8D7F8093870C8091B7
:103BF000080180958170809306018091870C8B7FEE
:103C00008093870C0C94E81D269A2E9A08958C3286
:103C100021E0920714F08CE291E090935612809389
:103C200055120C9411F5EBE3F9E010821182128227
:103C3000138214820C9411F52F923F924F925F924F
:103C40006F927F928F929F92AF92BF92CF92DF92AC
:103C5000EF92FF920F931F93CF93DF93CDB7DEB711
:103C60006C970FB6F894DEBF0FBECDBF8C015B0121
:103C70005A834983FC01EE5AFF4F208131814281F2
:103C8000538129873A874B875C87CA01B9010F9412
:103C9000031E6B017C01D5012D913D914D915C91ED
:103CA0000F94641E0F94BA252B013C01E981FA811F
:103CB0002081318142815381C701B6010F94641E76
:103CC0000F94BA254B015C01C301B2010F944F263A
:103CD000698B7A8B8B8B9C8B68377105810591057D
:103CE00040F428E730E040E050E0298B3A8B4B8BE2
:103CF0005C8BC501B4010F944F266D877E878F873B
:103D0000988B683771058105910540F448E750E0CC
:103D100060E070E04D875E876F87788BF801E25A2C
:103D2000FF4F4080518062807380C301B2010F94C5
:103D3000051E69837A838B839C8369897A898B8941
:103D40009C890F94031E6D8B7E8B8F8B988F20E048
:103D500030E0A90169817A818B819C810F94FE1DDD
:103D6000882309F4E1C1A7019601C701B6010F94A8
:103D7000641E4B015C012D893E894F89588DCA0113
:103D8000B9010F94641E9B01AC01C501B4010F94ED
:103D9000DB244B015C0129813A814B815C81CA01A2
:103DA000B9010F94DC249B01AC01C501B4010F944F
:103DB000D6250F94BA250F944F266D837E838F836B
:103DC000988766277727CB016419750986099709B3
:103DD0000F94051E4B015C016D857E858F8598894A
:103DE0000F94031E2B013C0120E030E0A901C50126
:103DF000B4010F94FE1D882309F49AC1A301920116
:103E0000C301B2010F94641E698F7A8F8B8F9C8FD0
:103E1000A7019601C701B6010F94641E9B01AC0176
:103E2000698D7A8D8B8D9C8D0F94DB246B017C01C9
:103E3000A5019401C501B4010F94DC249B01AC01E0
:103E4000C701B6010F94D6250F947E26D80195960A
:103E50008D909D90AD90BC909897750164012D81D7
:103E60003E814F815885C21AD30AE40AF50A0F949D
:103E70004F26C61AD70AE80AF90AF7FE8EC02D891E
:103E80003E894F89588DCA01B9010F94641E6B0198
:103E90007C0129813A814B815C81CA01B9010F946F
:103EA000DC2469877A878B879C8720E030E0A90132
:103EB00069817A818B819C810F94FE1D882309F48E
:103EC0003BC1C501B4010F94031E29853A854B857A
:103ED0005C850F94641EA70196010F94DB246D830B
:103EE0007E838F839887A3019201C301B2010F944F
:103EF000641E9B01AC016D817E818F8198850F943A
:103F0000DC242B013C0120E030E040E850E46981F2
:103F10007A818B819C810F94641E9B01AC01C3014B
:103F2000B2010F94D6250F94BA252B013C0120E055
:103F300030E0A9010F943C2718161CF0412C512C9D
:103F40003201C301B2010F944F266D837E838F83AC
:103F5000988786169706A806B90620F48D829E8259
:103F6000AF82B8866D817E818F8198850F94031E04
:103F700029853A854B855C850F94641EA7019601BF
:103F80000F94DC240F948A270F944F2669877A8731
:103F90008B879C87C12CD12C760169857A858B858E
:103FA0009C8529893A894B895C89621B730B840B38
:103FB000950B0F94031E29813A814B815C810F94EC
:103FC000D62520E034E244EF59E40F94641E0F94A8
:103FD0004F264B015C0169857A858B859C852D85F3
:103FE0003E854F855889621B730B840B950B0F948C
:103FF000031E29813A814B815C810F94D62520E0F4
:1040000034E244EF59E40F94641E0F944F262B01C1
:104010003C013FE683169104A104B10408F090C06E
:10402000F401EE0FFF1FEE0FFF1FE451FA4E8591D2
:104030009591A591B4918983292E3A2EBD8B4FE697
:10404000441651046104710408F083C0F201EE0FBC
:10405000FF1FEE0FFF1FE451FA4E459155916591F8
:1040600074919A01CB014D815E816F817885D80171
:104070009A964D935D936D937C939D974C0D5D1D2A
:104080006E1D7F1DF80146A757A760AB71ABEA5ABA
:10409000FF4F49895A896B897C89408351836283A8
:1040A0007383D6968D929D92AD92BC92D997F8016A
:1040B00042AE53AE64AE75AEFE9649814083218216
:1040C00032825D8953833496208331838283938344
:1040D00069857A858B859C85D2966D937D938D932A
:1040E0009C93D59778962D853E854F85588920835A
:1040F0003183428353836C960FB6F894DEBF0FBEB4
:10410000CDBFDF91CF911F910F91FF90EF90DF9086
:10411000CF90BF90AF909F908F907F906F905F9067
:104120004F903F902F90089560E070E0CB0141CE1A
:1041300060E070E0CB0188CE60E070E0CB01F3CEB0
:10414000C501B4010E94EF186983272E382E9D8B7C
:1041500076CFC301B2010E94EF189B0184CFEF928A
:10416000FF920F931F93CF93DF93CDB7DEB78C01F0
:10417000EDB6FEB60F944B1D01962DB73EB7281B2A
:10418000390B0FB6F8943EBF0FBE2DBF8DB79EB74B
:104190000196B8010F94441D0E94E2F10FB6F89405
:1041A000FEBE0FBEEDBEDF91CF911F910F91FF902C
:1041B000EF9008958C38910514F08CE890E090937E
:1041C000EC118093EB110C9471C42F923F924F929B
:1041D0005F926F927F928F929F92AF92BF92CF9297
:1041E000DF92EF92FF920F931F93CF93DF93D62F1F
:1041F000C72FFC0180809180A280B380C501B401EB
:1042000020E831E541E050E00F944224C9016DE619
:1042100071E00F94B3246B017C01C501B40120E16E
:104220003EE040E050E00F944224CA01B90128E189
:1042300030E040E050E00F944224362E272E062F27
:10424000172F8CE3482E512C612C712CC501B40121
:10425000A30192010F944224B62EA72ECA01B901E0
:10426000A30192010F944224CB01C114D10479F12E
:10427000AF92BF927F936F932F923F92FF92EF92F4
:10428000DF92CF9287E593E19F938F93CF93DF9354
:104290000F94951D8DB79EB70E960FB6F8949EBFDE
:1042A0000FBE8DBF8D2F9C2FDF91CF911F910F914E
:1042B000FF90EF90DF90CF90BF90AF909F908F9046
:1042C0007F906F905F904F903F902F900895E114F2
:1042D000F104C9F0AF92BF927F936F932F923F92F8
:1042E000FF92EF9287E493E19F938F93CF93DF93B5
:1042F0000F94951DEDB7FEB73C960FB6F894FEBF30
:104300000FBEEDBFCFCF012BB9F0AF92BF927F931D
:104310006F932F923F928BE393E19F938F93CF9371
:10432000DF930F94951D8DB79EB70A960FB6F8943C
:104330009EBF0FBE8DBFB6CF892BA9F0AF92BF92A3
:104340007F936F9383E393E19F938F93CF93DF9357
:104350000F94951DEDB7FEB738960FB6F894FEBFD3
:104360000FBEEDBF9FCFAF92BF928FE293E19F93BD
:104370008F93CF93DF930F94951D0F900F900F9015
:104380000F900F900F908ECFAB01BC0140938B1418
:1043900050938C1460938D1470938E1483EF95E179
:1043A0000C941BB28091D3049091D404009731F007
:1043B0004AE050E070E060E00D94191C60E070E0AD
:1043C000CB0108958091D3049091D404009731F0EB
:1043D0004AE050E070E060E00D94EB1A60E070E0BD
:1043E000CB010895CF93DF93EB010E94DB1D88235F
:1043F00019F00E94E221EB01CE01DF91CF910895E7
:104400000E94E22197FD0CC00E94E2216F3F7105DE
:104410008105910509F034F40E94E221862F089568
:1044200080E008958FEF0895CF93C62F0E94DB1D83
:10443000882319F0CF910C9400228C2FCF910895EE
:104440008091D3049091D404892B41F00E940022E2
:1044500091E0811101C090E0892F089591E0FCCF97
:10446000CF93DF93C82FD62F0E94DB1D882321F026
:10447000DF91CF910C9420228C2F0E948D1D8111F1
:1044800001C08D2FDF91CF9108950E94E221CB01D1
:104490000895CF93DF93EB010E94DB1D882321F069
:1044A000DF91CF910C944522CE01DF91CF910895F9
:1044B0000F931F93CF938091D3049091D4040097CE
:1044C000E9F0FC018F01C1912C2F2F7D81F0C534C3
:1044D00011F0C536B9F7F801108270E060E00F9472
:1044E0008D19F801C083CF911F910F91089570E04D
:1044F00060E0CF911F910F910D948D1960E070E0F5
:10450000CB01F1CFCF92DF92EF92FF926A017B0154
:104510000E94DB1D882331F0FF90EF90DF90CF9059
:104520000C945822C701B601FF90EF90DF90CF9016
:1045300008954F925F926F927F928F929F92AF9267
:10454000BF92CF92DF92EF92FF921F93CF93DF93B0
:1045500000D01F92CDB7DEB719821A821B821C824F
:10456000CE0101964C0185EDC82E8AE0D82E9BEF36
:10457000E92E9CE0F92E2BE3A22E2CE0B22E10E0C7
:1045800088E5810F0E94DB1DF40181934F01882390
:1045900009F4E0C00E9458222B013C01812F0E94A7
:1045A000731D882309F4CCC0F70120813181428139
:1045B0005381C301B2010F94DC24F601608371833F
:1045C000828393831F5FF4E0CF0ED11C84E0E80E5A
:1045D000F11C94E0A90EB11C133091F685E40E9401
:1045E000DB1D8C83882309F4C0C00E9458226B0114
:1045F0007C0183E00E94731D882371F02091070DD8
:104600003091080D4091090D50910A0DC701B60176
:104610000F94DC246B017C01C092E10AD092E20A83
:10462000E092E30AF092E40A8091F608882359F1B7
:1046300080918F1482FF27C08C81882321F189818A
:10464000811103C08A818823F1F02DEC3CEC4CE40D
:104650005DE36091810B7091820B8091830B90914F
:10466000840B0F94DC249B01AC016091030D7091CD
:10467000040D8091050D9091060D0F943C2718169E
:1046800014F40E9449EF40E050E0BA0186E40E9431
:10469000822220E030E0A9010F943C27181684F410
:1046A0000E94582220E030E040E752E40F94D625E3
:1046B00060934702709348028093490290934A02A4
:1046C0008091530B83FD28C08091F209882321F14A
:1046D0002091070D3091080D4091090D50910A0D60
:1046E0006091E10A7091E20A8091E30A9091E40AF4
:1046F0000F94DB242091FF093091000A4091010AB8
:104700005091020A0F94DC246093FF097093000A11
:104710008093010A9093020A0F900F900F900F90D0
:10472000DF91CF911F91FF90EF90DF90CF90BF90DE
:10473000AF909F908F907F906F905F904F90089573
:10474000F5012081318142815381C301B2010F946F
:10475000DB2433CFF70180819181A281B381F601FF
:1047600080839183A283B3832DCF8091070D909195
:10477000080DA091090DB0910A0D8093E10A909364
:10478000E20AA093E30AB093E40A4ECF0F931F937B
:10479000CF93DF9300D01F92CDB7DEB78C01089680
:1047A0000E94681C69837A838B839C83BE016F5F40
:1047B0007F4FC8010E94FA1A9B01AC01F801608585
:1047C0007185828593850F94DB24F801608771875A
:1047D000828793870F900F900F900F90DF91CF916A
:1047E0001F910F9108950F931F93CF93DF930CE9BF
:1047F0001CE0C0EDDCE0F801219131914191519133
:104800008F0160E070E080E89FE30F94D625699304
:10481000799389939993FCE0C03EDF0761F70E948A
:1048200088EDDF91CF911F910F910C94ED190F93AB
:104830001F93CF93DF9300D01F92CDB7DEB72091A7
:10484000FA0C2223E1F08C0108960E94681C69830F
:104850007A838B839C83BE016F5F7F4FC8010E9468
:10486000FA1A9B01AC01F8016085718582859385F8
:104870000F94DC24F80160877187828793870F90FB
:104880000F900F900F90DF91CF911F910F9108958E
:1048900080919B1290919C12891B877019F490E073
:1048A00080E0089590919812992351F0833030F46C
:1048B0008FEF890F19F080939812F1CF1092981210
:1048C00080919C1228E6829FC001112488579A4F3C
:1048D000FC01208120FDE3CF20919C122F5F2770E7
:1048E0002093991230919C1220919A12321304C095
:1048F0002091991220939A12089590916F0081E06F
:1049000091FD02C080E0089590916F009D7F90938B
:104910006F00089580FF04C090916F0990FD8E7F15
:1049200081FF05C090916F09969590FD8D7F82FF64
:1049300006C090916F099695969590FD8B7F08958E
:104940008F929F92AF92BF92CF92DF92EF92FF929F
:10495000CF93DF9320914B02222309F49EC0EC01F8
:1049600080916F09C82ED12CF12CE12C80FF2CC036
:1049700080904D0290904E02A0904F02B090500255
:10498000288139814A815B81C501B4010F943C279C
:10499000181624F488829982AA82BB8280905902D8
:1049A00090905A02A0905B02B0905C0228813981FD
:1049B0004A815B81C501B4010F94FE1D87FF04C0CD
:1049C00088829982AA82BB82D701C601B695A79533
:1049D0009795879580FF2CC080905102909052024D
:1049E000A0905302B09054022C813D814E815F8192
:1049F000C501B4010F943C27181624F48C829D82C3
:104A0000AE82BF8280905D0290905E02A0905F02B5
:104A1000B09060022C813D814E815F81C501B4015F
:104A20000F94FE1D87FF04C08C829D82AE82BF82E0
:104A300082E0F694E794D794C7948A95D1F7C0FEA4
:104A40002CC0C0905502D0905602E0905702F090D2
:104A50005802288539854A855B85C701B6010F94C0
:104A60003C27181624F4C886D986EA86FB86C090AF
:104A70006102D0906202E0906302F09064022885A7
:104A800039854A855B85C701B6010F94FE1D87FFF6
:104A900004C0C886D986EA86FB86DF91CF91FF9055
:104AA000EF90DF90CF90BF90AF909F908F90089540
:104AB00024E0829FC0011124FC01E35AFA4E459183
:104AC000559165917491DC01A55BBD4F12964D9394
:104AD0005D936D937C9315978F5A9A4EFC01459187
:104AE0005591659174911E964D935D936D937C9352
:104AF000519708950C9488ED80915C05659B55C095
:104B0000816080935C059091030180915C0591FF29
:104B10004EC0826080935C0580915C054B9B49C0D0
:104B2000846080935C0580911B0980FF10C0809198
:104B3000050A80FF0CC080915C0580FF08C0809151
:104B4000470A81608093470A80E00E9464CC80918C
:104B50001B09869580FF11C08091050A869580FF0C
:104B60000CC080915C0581FF08C08091470A82607B
:104B70008093470A81E00E9464CC80911B0986954E
:104B8000869580FF18C08091050A8695869580FFDE
:104B900012C080915C0582FF0EC08091470A84603C
:104BA0008093470A82E00C9464CC8E7FAACF8D7FDD
:104BB000B1CF8B7FB6CF08950F931F938091A31130
:104BC000813019F50E9405F50091C8081091C908B7
:104BD0002091CA083091CB08601B710B820B930B9C
:104BE00028EE33E040E050E00F9442246091CC087E
:104BF0007091CD088091CE089091CF08620F731FFD
:104C0000841F951F1F910F9108956091D008709196
:104C1000D1088091D2089091D308D6CF1092A311D9
:104C20001092C8081092C9081092CA081092CB08B6
:104C30001092D0081092D1081092D2081092D30886
:104C40001092CC081092CD081092CE081092CF0886
:104C50000895CF92DF92EF92FF92CF93C62FFC017F
:104C6000C080D180E280F38020E030E0A901C7015C
:104C7000B6010F94FE1D20E030E0A90187FD14C0AD
:104C800020E030E048EC52E4C701B6010F943C2725
:104C900024E630E040E050E0181634F0C701B601D9
:104CA0000F9448269B01AC01AFEFB0E00F94832432
:104CB00024E630E040E050E00F946424B9018C2FEA
:104CC000CF91FF90EF90DF90CF900C942FCC8091FC
:104CD000090180FD06C080918F1483FB882780F92D
:104CE000089580E00895CF92DF92EF92FF92FC0149
:104CF000C080D180E280F380663019F510924009BF
:104D000010924109109242091092430910924409ED
:104D10000E9471C420E030E0A901C701B6010F94E0
:104D2000FE1D87FF1DC0C12CD12C7601C701B60125
:104D30000F944927CB01FF90EF90DF90CF900C9418
:104D4000DA200E94131E20E030E0A901C701B6015D
:104D50000F94FE1D87FF15C0C12CD12C760121C0F8
:104D600020E030E04CE053E4C701B6010F943C274B
:104D70001816E4F6C12CD12C9CE0E92E93E4F92E10
:104D8000D5CF20E030E046E953E4C701B6010F94E7
:104D90003C27181634F4C12CD12C86E9E82E83E484
:104DA000F82EC701B6010F944927CB01FF90EF9071
:104DB000DF90CF900C94071E9091870C977081E044
:104DC000973009F080E0089560919E1170919F11D5
:104DD000072E000C880B990B0F94051E2091D80C00
:104DE0003091D90C4091DA0C5091DB0C0F94641E79
:104DF00020E030E0A9010F94DC240895E091F90C43
:104E0000E150E73028F4F0E0E651FD4F808108954D
:104E100080E00895CF93DF931092470C1092E00C3E
:104E20001092E20C1092E10C109259051092580564
:104E3000CFEFDFEF80918F1485FD07C00E947CAD1E
:104E4000D093E612C093E512F5CF8FEF9FEF9093CA
:104E5000E6128093E512DF91CF9108958F929F9291
:104E6000AF92BF92CF92DF92EF92FF920F931F9378
:104E7000CF93DF9310920D0510920C052FE3209332
:104E80000B0510920A051092090510920805109260
:104E900004051092050510920605109207059C0165
:104EA000F90190812F5F3F4F9032D1F39E34C9F4C6
:104EB000818190ED980F9A3020F08D3211F08B3275
:104EC00081F432969F012F5F3F4F808180538A305B
:104ED00008F47BC09F012F5F3F4F8081803209F42F
:104EE00076C0F093E90AE093E80A8F010F5F1F4F45
:104EF000C0816AE270E0C8010F942A28009731F05F
:104F0000FC01319780818032E1F31182CD3429F0A8
:104F1000C43519F0C73409F04BC0F80180810F5F28
:104F20001F4F8032D1F380538A3008F041C0C093C4
:104F30000B0530E020E04AE0DF011196429FC001FE
:104F4000439F900D11249C01205331098081280F2B
:104F5000311D87FD3A95818190ED980F9A30C8F107
:104F600030930A05209309058E3261F4329690E061
:104F70004AE0DF0131968C9150ED580F5A3058F1CC
:104F800090930805CD01DC0101964C914032D9F394
:104F9000CD3489F52E31310539F018F52731310539
:104FA00019F02C31310539F5B0930D05A0930C059E
:104FB000DF91CF911F910F91FF90EF90DF90CF90F5
:104FC000BF90AF909F908F900895F9017BCFF9012A
:104FD00081CFFD01B1CF949F800D112490ED980FEA
:104FE000C8CF2537310538F027373105E8F2203AA8
:104FF00083E03807C9F2D091E80A40E050E0BA01F6
:1050000010E000E0C12CD12C7601C394FD01319653
:105010008C91882309F47FC08132E1F4CD34D1F43E
:1050200020323105B9F4409304055093050560938F
:10503000060570930705F0930D05E0930C0563E2F8
:1050400070E0CF010F942A28009709F4B1CFFC013A
:105050001082AECF81548A3108F058C0DF019D9193
:10506000903291F0A0EDA90FAA30E8F09E3271F4D1
:10507000918190539A30B8F00115110519F48F0100
:105080000150110990E013C0FD01E8CF9D3211F0ED
:105090009B3291F79181A0EDA90FAA3020F09E32AA
:1050A00059F79281E6CF9E2F9D1B309759F3A82F79
:1050B000B0E04601570104C0880C991CAA1CBB1C17
:1050C0008A95D2F7482959296A297B29A651BB4FCD
:1050D0009C9380818154DF018A3108F497CFDF01EE
:1050E0008191882309F492CF90ED980F9A30B8F30C
:1050F00093ED980F923098F38B3289F3CD0101969E
:10510000EC91E03209F082CFDC01F8CF01151105F6
:1051100001F78D01DECF10930D0500930C05409330
:10512000040550930505609306057093070540CF6D
:105130000F931F93CF93DF93C82FD0E0FE01EE0FA4
:10514000FF1FEA5CFD4F71836083CC0FDD1FCC0F26
:10515000DD1F8E010A5E1D4F072E000C880B990B78
:105160000F94051E2AE037ED43E25CE30F94641EC2
:10517000CB59DA4F288139814A815B810F94641EB3
:10518000F8016083718382839383DF91CF911F91B4
:105190000F910895E8E7FBE087EBDF011D928A9508
:1051A000E9F708958091F608811104C00E94CA2889
:1051B0000C94DDBA80918F1482FD0C9449EF089510
:1051C0008091780B882361F090912E0C891308C090
:1051D00080918F1483FF04C08BEB9BE00C94A7B9E4
:1051E00080E00895FC01238121110C94DCB5089521
:1051F000CF93DF931092F7081092F8081092F908F5
:105200001092FA08EEEEFAE084E6DF011D928A952C
:10521000E9F7C0E0D0E06D2F8C2F0E9415F0DF5F22
:10522000D530C9F7CF5FC530A9F7DF91CF91089589
:10523000EF92FF920F931F93CF93DF930EEE1AE03E
:10524000C5E07801D5E0F70161917191819191916B
:105250007F0120E030E0A9010F94FE1D81110EC0F6
:10526000D15089F7C1500C5E1F4FC111EACFDF91B9
:10527000CF911F910F91FF90EF90089581E0F7CFAC
:10528000EFE6F0E08081826080830895CF92DF9224
:10529000EF92FF92CF93DF93C82F0E947D2494E07A
:1052A000C99FE0011124FE01E75DF64FC080D18067
:1052B000E280F38081110E944029C053D34FC7017F
:1052C000B6010F94051E288139814A815B810F94B4
:1052D000641EDF91CF91FF90EF90DF90CF90089503
:1052E000CF92DF92EF92FF92CF93DF93C82F0E946D
:1052F0007D2494E0C99FE0011124FE01E35EF64F96
:10530000C080D180E280F38081110E944029C05387
:10531000D34FC701B6010F94051E288139814A81F8
:105320005B810F94641EDF91CF91FF90EF90DF902F
:10533000CF9008950E947D2490919C1290939B128F
:1053400090939A129093991294E69093981220ED6C
:1053500033E03093E60A2093E50A81110E94402948
:1053600081E080931C090895CF93DF93CDB7DEB71A
:105370002C970FB6F894DEBF0FBECDBF0E9466EE2D
:105380000E947D249CE0E9E2F9E0DE0111960190A3
:105390000D929A95E1F781110E944029CE01019664
:1053A0000E9444CC2C960FB6F894DEBF0FBECDBF42
:1053B000DF91CF9108954F925F926F927F928F927B
:1053C0009F92AF92BF92CF92DF92EF92FF92409066
:1053D000FB0C5090FC0C6090FD0C7090FE0C8090CB
:1053E000FF0C9090000DA090010DB090020DC090A8
:1053F000030DD090040DE090050DF090060D0E9475
:10540000ED190E943B1A80E00E94E21C80E00E949D
:10541000582581E00E94E21C81E00E94582582E02C
:105420000E94E21C82E00E9458258BEF98E00E94C7
:10543000CBEE0E94F323A30192016091FB0C7091CB
:10544000FC0C8091FD0C9091FE0C0F94FE1D8111BF
:105450001CC0A50194016091FF0C7091000D80911A
:10546000010D9091020D0F94FE1D81110EC020912F
:10547000030D3091040D4091050D5091060DC701AB
:10548000B6010F94FE1D882371F0FF90EF90DF901E
:10549000CF90BF90AF909F908F907F906F905F90D4
:1054A0004F900C94B429FF90EF90DF90CF90BF9075
:1054B000AF909F908F907F906F905F904F900895E6
:1054C0008091A0119091A111892B79F48091A01164
:1054D0009091A111892B49F42091A0113091A11133
:1054E00081E0232B19F480E0089581E00895CF92A4
:1054F000DF92EF92FF926B017C0183E3C816D10427
:10550000E104F10470F082E3C81AD108E108F1085F
:1055100062E370E080E090E00E94D2F40E94F0C765
:10552000ECCFC701B6010E94D2F4FF90EF90DF905C
:10553000CF900C94F0C78091040A882331F062E088
:1055400070E080E090E00C94772A089520915A054D
:1055500020FF14C020E83EE3629FA001639F500D2E
:10556000729F500D1124CA0196958795969587953F
:10557000009731F08A950000E9F708950C94772A96
:1055800008958091F90C882341F0813041F064E660
:1055900070E080E090E00C94772A129AF8CF479A56
:1055A000F6CF90918F1493FB882780F993FF06C064
:1055B00081E09091F615911101C080E00895CF939C
:1055C000C0915B05CF7739F50E94D12A882319F164
:1055D0008091871490918814A0918914B0918A14B5
:1055E0000097A105B105B9F0BC01CD016D597F4F00
:1055F0008F4F9F4F24E630E040E050E00F9442246C
:1056000060918B1470918C1480918D1490918E14F4
:105610000F944224C22F8C2FCF91089570E060E048
:1056200080E00E942FCC70E060E081E00C942FCCF1
:1056300081E008958F929F92AF92BF92CF92DF92B6
:10564000EF92FF920F93CF93DF931F92CDB7DEB708
:105650005C017B0149016B01C40ED51EF5018081FF
:1056600091810F941C248983002311F0F70180831A
:10567000BE016F5F7F4FC4010E94CFE5F5018081BD
:105680009181019691838083FFEFEF1AFF0AEC145A
:10569000FD0421F780E00F90DF91CF910F91FF90F3
:1056A000EF90DF90CF90BF90AF909F908F90089534
:1056B0000F93AB0100910F0921E0022720E139E0AF
:1056C000BC0184EE98E00E941A2B0F9108959091EE
:1056D000D10095FD0CC09091D00095FF08C080933B
:1056E000D6008091D00080648093D00008952091EE
:1056F00012042F5F2F770FB607FC27C09091130479
:10570000921328C09091D00095FF1EC09091130471
:1057100040911204941306C09091D1009F7D909304
:10572000D10012C0E92FF0E0EE5EFB4F32819F5FA7
:105730009F773093D600909313043091D00030645B
:105740003093D000491741F3D9CF909113049213AD
:1057500001C0FBCFE0911204F0E0EE5EFB4F8283CC
:10576000209312048091D10080628093D10008952B
:105770008F929F92AF92BF92CF92DF92EF92FF9261
:105780000F931F93CF93DF937C0121E5E20EF11C71
:10579000D7014C914A3509F0A4C06C01B2E5CB0E9B
:1057A000D11CF6013081353A09F09BC0EC01C05B99
:1057B000DF4F2881233008F494C08C0100561F4F1E
:1057C000D8014C93E15BFF4F308331962083EF5437
:1057D000F1093081E05BFF4F30833038B1F431960E
:1057E000AC54B1093C913083E854F109AF5ABF4F32
:1057F00050E040E02250330B42175307CCF4808135
:1058000032968D934F5F5F4FF7CF233031F53138AC
:1058100009F074C0FC01EC55FF4FDC01AC5ABF4FDE
:105820002C9120833196885A9F4FDC018C91808384
:105830004801B12CA12C888190E002968A159B0525
:105840000CF43FC0F40181914F010E94672B0E942C
:10585000E5E5FFEFAF1ABF0AEECF323821F5FC01C4
:10586000EC5AFF4F30814181E05BFF4F408331961E
:105870003083DC01AA55BF4F50E040E02350330B8A
:1058800042175307ACF6FA01EE7FE45AFF4FE80FD8
:10589000F91F608171817C9311966C9311974E5F13
:1058A0005F4F1296EDCF243019F6333809F6FC011C
:1058B000EC5AFF4F20813181E05BFF4F30833196FE
:1058C000B0CF80E5DE011D928A95E9F78AE1F80103
:1058D00011928A95E9F78AE5D7018C9385EAF6015A
:1058E0008083DF91CF911F910F91FF90EF90DF9018
:1058F000CF90BF90AF909F908F900895323809F06D
:1059000097CFADCFAF92BF92CF92DF92EF92FF923F
:105910000F931F93CF93DF93EC0184E6C82E80E2B0
:10592000D82EE12CF12C02E8A12C90E2B92E15E042
:105930000093F413C092F513D092F613E092F7138C
:10594000F092F813B092FE13A092FD131093F1138E
:1059500081EA93E10E94B82B8FEFC81AD80AE80AAF
:10596000F80A88E7C81680E2D806E104F10401F7D6
:1059700024E630E240E050E0BE0181EA93E1DF91AD
:10598000CF911F910F91FF90EF90DF90CF90BF903C
:10599000AF900C94EAE5CF92DF92EF92FF920F93D3
:1059A0001F93CF93DF93CDB7DEB77C01CDB6DEB6C4
:1059B0000F944B1D01962DB73EB7281B390B0FB620
:1059C000F8943EBF0FBE2DBF0DB71EB70F5F1F4F20
:1059D000B701C8010F94441DC8010E94822C0FB664
:1059E000F894DEBE0FBECDBEDF91CF911F910F9117
:1059F000FF90EF90DF90CF9008958F929F92AF929B
:105A0000BF92CF92DF92EF92FF920F931F93CF93AB
:105A1000DF930E940A273AE0C32E30E2D32EE12C16
:105A2000F12C15E002E846015701CAE0D0E01092DF
:105A3000FE131092FD131093F1130093F413809250
:105A4000F5139092F613A092F713B092F81381EA2F
:105A500093E10E94B82B21978FEF881A980AA80A21
:105A6000B80A209721F78AE0C80ED11CE11CF11C6E
:105A700082EDC81680E2D806E104F104A1F6C12C3B
:105A800020E2D22EE12CF12CD5E0C2E81092FE13D8
:105A90001092FD13D093F113C093F413C092F51339
:105AA000D092F613E092F713F092F81381EA93E1A3
:105AB0000E94B82B1092FE131092FD13D093F11395
:105AC000C093F413D701C6018C529F4FAF4FBF4F05
:105AD0008093F5139093F613A093F713B093F813F4
:105AE00081EA93E10E94B82B8FEFC81AD80AE80A1E
:105AF000F80A8AE0C81680E2D806E104F10431F61B
:105B00009EEDC92E90E2D92EE12CF12CD5E0C2E811
:105B10001092FE131092FD13D093F113C093F4135F
:105B2000C092F513D092F613E092F713F092F813A7
:105B300081EA93E10E94B82B8FEFC81AD80AE80ACD
:105B4000F80A86EEC81680E2D806E104F10401F7EF
:105B5000CC24C39482E1D82EE12CF12C0AE010E091
:105B6000D5E0C2E81093FE130093FD13D093F11318
:105B7000C093F413C092F513D092F613E092F7138A
:105B8000F092F81381EA93E10E94B82B1093FE1370
:105B90000093FD13D093F113C093F413D701C60102
:105BA0008096A11DB11D8093F5139093F613A093D9
:105BB000F713B093F81381EA93E10E94B82B8FEFAB
:105BC000C81AD80AE80AF80A85E1C81682E1D80698
:105BD000E104F10439F682E190E09093FE138093A2
:105BE000FD13D093F113C093F41384E190E1A0E08E
:105BF000B0E08093F5139093F613A093F713B0934E
:105C0000F81381EA93E1DF91CF911F910F91FF90FB
:105C1000EF90DF90CF90BF90AF909F908F900C94BB
:105C2000B82B1F920F920FB60F9211240BB60F9242
:105C30002F938F939F93EF93FF9380911304209161
:105C40001204821306C08091D1008F7D8093D10011
:105C500012C0E82FF0E0EE5EFB4F92818F5F8F77EE
:105C60009093D600809313049091D0009064909309
:105C7000D000281741F3FF91EF919F918F912F91C1
:105C80000F900BBE0F900FBE0F901F9018951F9294
:105C90000F920FB60F9211240BB60F920F931F9312
:105CA0002F933F934F935F936F937F938F939F9324
:105CB000AF93BF93CF93DF93EF93FF93C091D60041
:105CC00000910F05D0910E0511E01D0F1F739091EB
:105CD0001104913108F09FC0E92FF0E08827EC58BB
:105CE000F14D8F4F0D94C724852EB42EC32ED22E86
:105CF000D92E0B2FDD2E0B2FE12EE52E0B2FE92EAB
:105D0000ED2EF12EF82E0B2F032FC03229F028F59F
:105D1000CA3011F0CD3031F5011731F0ED2FF0E040
:105D2000E25FFA4FC283D12FD0930E05FF91EF911E
:105D3000DF91CF91BF91AF919F918F917F916F91A3
:105D40005F914F913F912F911F910F910F900BBE3B
:105D50000F900FBE0F901F901895CD3481F081E009
:105D6000CE3471F080E10CC0CA3338F4C033A0F6F1
:105D7000C03291F2CD32B1F7CFCFCD3499F782E076
:105D800080931104C9CFC13359F018F4C03221F205
:105D9000E9CF88E0C433A1F38BE0C83389F3E2CFC5
:105DA00083E0EECF84E0C03359F386E0C13341F3A2
:105DB000D9CF85E0C833B1F6E3CF87E0C23391F69F
:105DC000DFCF89E0C13371F6DBCF8AE0C03351F613
:105DD000D7CF8CE0C73331F6D3CF8DE0C63311F681
:105DE000CFCFC03209F498CF8EE0C33549F2BACF95
:105DF00080ED8C0F8A3008F08FCF9FE090931104D4
:105E00008093100489CFCA3019F0CD3009F084CFC7
:105E10001092110481CFCA3019F0CD3009F07CCF37
:105E200080915B148823A1F3973079F038F4953092
:105E300079F71092460210926612EACF9A3049F032
:105E40009F3031F70E94BCE5E3CF81E080933A09AF
:105E5000DFCF81E080933909DBCF9091C00095FFBF
:105E6000FCCF8093C6000895CF93DF93EC01899116
:105E7000882319F00E942D2FFACF8DE00E942D2F3C
:105E80008AE0DF91CF910C942D2FCF92DF92EF9289
:105E9000FF92CF936B017C01C42F4A3069F4F7FE67
:105EA0000BC0F094E094D094C094C11CD11CE11CB0
:105EB000F11C8DE20E942D2F4C2FC701B601CF910E
:105EC000FF90EF90DF90CF900C9415ADCF93DF93C0
:105ED000EC01FE0184912196882319F00E942D2F58
:105EE000F8CFDF91CF910895CF93DF93D091A31195
:105EF00082EE98E10E94662F8AE00E942D2F809109
:105F0000F80C873009F449C083E08093F30C81E0FA
:105F100080936C0280E190E09093FE138093FD13D8
:105F200085E08093F113C2E8C093F41384E190E11B
:105F3000A0E0B0E08093F5139093F613A093F713CD
:105F4000B093F81381EA93E10E94B82B61E070E00E
:105F500080E090E00E94A62A81E09AE59093FE13EB
:105F60008093FD1385E390E0909300148093FF13DA
:105F700087E08093F113C093F41384E890E0A0E0ED
:105F8000B0E08093F5139093F613A093F713B093BA
:105F9000F81381EA93E10E94B82B8091A31181301C
:105FA00089F1823061F50E94DC256093CC08709302
:105FB000CD088093CE089093CF0881E08093A31101
:105FC0000E9405F56093C8087093C9088093CA08B9
:105FD0009093CB08D23089F08091F3099091F40925
:105FE00001969093F4098093F3091092D4081092CB
:105FF000D5081092D6081092D70881E004C00E94FC
:106000000E26DBCF80E0DF91CF910895CF93C82F8C
:10601000CB010E94662F82E295E10E94662F83E108
:1060200095E1CC2311F088E195E10E94662F8AE08A
:10603000CF910C942D2F87E395E10E94662F8CB1B0
:1060400061E375E185FB882780F90E940630809125
:1060500003016BE275E1869581700E94063089B17B
:1060600065E275E183FB882780F90C940630809106
:10607000A3118130C1F58EEE94E10E94662F8AE073
:106080000E942D2F81E09AE59093FE138093FD13DB
:1060900087E590E0909300148093FF1387E080934E
:1060A000F11382E88093F41384E890E0A0E0B0E07C
:1060B0008093F5139093F613A093F713B093F8130E
:1060C00081EA93E10E94B82B82E08093A3110E94A1
:1060D00005F56093D0087093D1088093D20890930F
:1060E000D30881E0089580E008950F931F930E94E4
:1060F00005F50091EE091091EF092091F00930911A
:10610000F109011511052105310509F067C020913C
:10611000D312222309F45FC0E091D11221502093C1
:10612000D31221E02E0F2093D1123091D4122313D9
:1061300002C01092D11224E0E29FF0011124EB5230
:10614000FD4E00811181228133810093EA09109371
:10615000EB092093EC093093ED09600F711F811D4D
:10616000911D6093EE097093EF098093F00990936D
:10617000F1098091EC099091ED09892B61F11FB72C
:10618000F8948BE794E10E94662F8AE00E942D2FFD
:1061900084E096E09093FE138093FD1380EA90E8EC
:1061A000909300148093FF1387E08093F11382E8AB
:1061B0008093F41380EA90E0A0E0B0E08093F513C0
:1061C0009093F613A093F713B093F81381EA93E139
:1061D0000E94B82B1FBF1F910F910895601B710B78
:1061E000820B930B97FDF7CF40981092EE09109217
:1061F000EF091092F0091092F109EDCF0F931F9360
:10620000CF93DF938C01EB019091D3122091D412A4
:10621000921305C00E9475300E94F0C7F5CF80919F
:10622000D21234E0839FF0011124EB52FD4E118312
:106230000083D383C2839F5F9093D3128F5F28170D
:1062400039F08093D212DF91CF911F910F91089571
:106250001092D212F8CFCF92DF92EF92FF921F935B
:10626000CF93DF93182F662351F01092B60410924B
:10627000B2041092B3041092B4041092B5040E94B8
:1062800005F56B017C018091B2049091B304A0915B
:10629000B404B091B504A7019601281B390B4A0B31
:1062A0005B0BDA01C901B7FD3DC02091B60417FDB3
:1062B00013C0412F012E000C550B4C5F5F4F822FF6
:1062C000022E000C990B4817590764F184EF91E0F6
:1062D000A0E0B0E0211724F488EE93E0A0E0B0E065
:1062E0008C0D9D1DAE1DBF1D8093B2049093B30411
:1062F000A093B404B093B5042170C22F30E0D32F23
:1063000084E28C9FB0018D9F700D7C1B112460591D
:106310007C4F82E390E00E94FE308091B6048F5F54
:106320008093B604DF91CF911F91FF90EF90DF90A3
:10633000CF900895CF93DF9300D01F92CDB7DEB7F3
:1063400085E094E10E94662F8AE00E942D2F8091C3
:10635000F80C8330D9F119821A821B821C8260E00A
:10636000CE0101960E94292619821A821B821C8264
:1063700061E0CE0101960E94292681E080936B02A4
:106380001092F20C80936C0281E09AE59093FE13D8
:106390008093FD1383E390E0909300148093FF13A8
:1063A00087E08093F11382E88093F41384E890E00F
:1063B000A0E0B0E08093F5139093F613A093F71349
:1063C000B093F81381EA93E10E94B82B0F900F90DD
:1063D0000F900F90DF91CF9108956F927F928F92DF
:1063E0009F92AF92BF92CF92DF92EF92FF920F9364
:1063F0001F93CF93DF93CDB7DEB764970FB6F894B2
:10640000DEBF0FBECDBF1092D0008091D000826061
:106410008093D0001092D50080E18093D4008091C9
:10642000D10080618093D1008091D10088608093F9
:10643000D1008091D10080688093D1008091D100FB
:106440008F7D8093D1008AE58093F2138093A2130D
:1064500085EA8093F3138093A313E1E4F4E18AE1E6
:10646000DF011D928A95E9F78091F10C882309F4E8
:1064700073C283E090E09093FE138093FD1385E058
:106480008093F11382E88093F4138FE190E1A0E010
:10649000B0E08093F5139093F613A093F713B093A5
:1064A000F81381EA93E10E94B82B84E690E0909380
:1064B000FE138093FD1305E00093F11312E810938F
:1064C000F41386E090E1A0E0B0E08093F5139093A0
:1064D000F613A093F713B093F81381EA93E10E94A7
:1064E000B82B8BE090E09093FE138093FD13009304
:1064F000F1131093F41380E092E1A0E0B0E08093F8
:10650000F5139093F613A093F713B093F81381EA61
:1065100093E10E94B82B1092FE131092FD1300938A
:10652000F1131093F41384E390E1A0E0B0E08093C2
:10653000F5139093F613A093F713B093F81381EA31
:1065400093E10E94B82B1092FE131092FD1300935A
:10655000F1131093F4138AE390E1A0E0B0E080938C
:10656000F5139093F613A093F713B093F81381EA01
:1065700093E10E94B82B8091531290915412909302
:10658000FE138093FD130093F1131093F41386E32D
:1065900090E1A0E0B0E08093F5139093F613A09300
:1065A000F713B093F81381EA93E10E94B82B80911E
:1065B000E9119091EA119093FE138093FD130093DB
:1065C000F1131093F4138CE390E1A0E0B0E080931A
:1065D000F5139093F613A093F713B093F81381EA91
:1065E00093E10E94B82B82E090E09093FE13809399
:1065F000FD130093F1131093F4138EE190E1A0E0EA
:10660000B0E08093F5139093F613A093F713B09333
:10661000F81381EA93E10E94B82B81E080936B022A
:1066200070E6C72E70E1D72EE12CF12C1092FE13EC
:106630001092FD130093F1131093F413C092F5130D
:10664000D092F613E092F713F092F81381EA93E1F7
:106650000E94B82BBFEFCB1ADB0AEB0AFB0AE4E778
:10666000CE16E0E1DE06E104F10401F7CE01019669
:106670007C0184E1D7011D928A95E9F781E08F932F
:1066800090E99F938F939CE29F938F939F9380E9D0
:1066900093E09F938F93FF92EF920F94642820E6EC
:1066A00030E140E050E06DE973E081EA93E10E945F
:1066B000EAE52AE630E140E050E067EA73E081EA8B
:1066C00093E10E94EAE524E730E140E050E0B701C1
:1066D00081EA93E10E94EAE52EE730E140E050E0F4
:1066E00065EB73E081EA93E10E94EAE51092FE1304
:1066F0001092FD130093F1131093F4138EE090E1C8
:10670000A0E0B0E08093F5139093F613A093F713F5
:10671000B093F81381EA93E10E94B82B1092FE1314
:106720001092FD130093F1131093F4138FE090E196
:10673000A0E0B0E08093F5139093F613A093F713C5
:10674000B093F81381EA93E10E94B82B0FB6F89446
:10675000DEBF0FBECDBF4AE0C42E40E2D42EE12CF6
:10676000F12C55E0752E62E8662E460157010AE0CD
:1067700010E01092FE131092FD137092F1136092CC
:10678000F4138092F5139092F613A092F713B0923F
:10679000F81381EA93E10E94B82B01501109FFEF31
:1067A0008F1A9F0AAF0ABF0A0115110511F78AE077
:1067B000C80ED11CE11CF11C92EDC91690E2D9065D
:1067C000E104F10491F6C12C30E2D32EE12CF12C3E
:1067D00005E012E81092FE131092FD130093F113DE
:1067E0001093F413C092F513D092F613E092F713BE
:1067F000F092F81381EA93E10E94B82B1092FE13F5
:106800001092FD130093F1131093F413D701C601F6
:106810008C529F4FAF4FBF4F8093F5139093F61359
:10682000A093F713B093F81381EA93E10E94B82B79
:10683000AFEFCA1ADA0AEA0AFA0ABAE0CB16B0E2ED
:10684000DB06E104F10431F62EEDC22E20E2D22E59
:10685000E12CF12C05E012E81092FE131092FD13CA
:106860000093F1131093F413C092F513D092F61322
:10687000E092F713F092F81381EA93E10E94B82BAB
:10688000EFEFCE1ADE0AEE0AFE0AF6EECF16F0E2BF
:10689000DF06E104F10401F7CC24C39482E1D82E91
:1068A000E12CF12C9AE0A92EB12C05E012E8B0926F
:1068B000FE13A092FD130093F1131093F413C092F2
:1068C000F513D092F613E092F713F092F81381EAE1
:1068D00093E10E94B82BB092FE13A092FD13009397
:1068E000F1131093F413D701C6018096A11DB11DB9
:1068F0008093F5139093F613A093F713B093F813C6
:1069000081EA93E10E94B82B8FEFC81AD80AE80AEF
:10691000F80A95E1C91692E1D906E104F10439F6C5
:106920008BE693E10E94662F8AE00E942D2F6496E9
:106930000FB6F894DEBF0FBECDBFDF91CF911F9190
:106940000F91FF90EF90DF90CF90BF90AF909F900E
:106950008F907F906F90089582E090E08CCD0E94A0
:10696000ED311092570581E080936C028DE194E146
:106970000E94662F8AE00C942D2F0F931F93CF93C4
:106980008C01C62F87E990E10E94662FC8010E9402
:10699000662F8AE30E942D2F80E38C0F0E942D2FFB
:1069A0008AE0CF911F910F910C942D2F8AE192E1F3
:1069B0000E94662F60E08AE092E10E94BD3460E0B0
:1069C00085EF91E10E94BD3461E08EEE91E10E947D
:1069D000BD3461E083EE91E10E94BD3461E083ED5E
:1069E00091E10E94BD3460E08AEC91E10E94BD34E7
:1069F00061E080EC91E10E94BD3460E086EB91E1C2
:106A00000E94BD3460E08FEA91E10E94BD3460E0F5
:106A100087EA91E10E94BD3461E089E991E10E9439
:106A2000BD3461E08BE891E10E94BD3460E08CE709
:106A300091E10E94BD3460E08EE691E10E94BD3498
:106A400060E088E591E10E94BD3461E087E491E176
:106A50000E94BD3461E088E391E10E94BD3461E0B1
:106A600081E391E10E94BD3460E08AE291E10E94FD
:106A7000BD3461E081E291E10E94BD3461E08CE0CF
:106A800091E10E94BD3461E08EEF90E10E94BD343F
:106A900061E08BEE90E10E94BD3460E08EED90E10C
:106AA0000E94BD3461E089ED90E10E94BD3461E057
:106AB0008CEC90E10E94BD3460E088EB90E10E9494
:106AC000BD3460E085EA90E10E94BD3460E082E977
:106AD00094E10E94701D682F61708CE990E10C9424
:106AE000BD340E942D2F86E09BE00C94662F0F93FF
:106AF0001F93CF938C01C62F88E097E00E94662FEA
:106B0000C8010E94662FCC2331F08AE0CF911F91FB
:106B10000F910C942D2FCF911F910F9108950F94E9
:106B2000D51010926612109246020E94D12A882334
:106B300051F080918F1482FD06C08FE691E390930F
:106B400065128093641261E084E794E10E947735D6
:106B50000C94742F0F931F93CF93DF938C016F3F8F
:106B600019F41092E41160E02091E411862F062EB2
:106B7000000C990B2817190609F08CF56093E411A5
:106B800060E08EE394E10E947735C8010E94662F91
:106B90008AE00E942D2FC8010F944B1D800F911F7A
:106BA000EC01C01BD10BC034D1053CF00197FC01B6
:106BB0002491207C2038D1F3F3CFDD27AE01B8013A
:106BC00084EA91E10F946C1DCC55DE4E188284EA64
:106BD00091E1DF91CF911F910F910C94822CDF9165
:106BE000CF911F910F910895109266121092460254
:106BF00080918F14806480938F1461E08CE494E121
:106C00000E94773541E654E169E674E185E00E942F
:106C100008E860E083E594E10C94AA3560E081EE39
:106C200097E00E94773582E197E00E94662F8AE024
:106C30000C942D2FEF92FF920F931F93CF937C0113
:106C40008B01C42F60E081EE97E00E947735C70189
:106C50000E94662F80E20E942D2FC8010E94662F9D
:106C6000CC2319F08C2F0E942D2F8AE0CF911F91F9
:106C70000F91FF90EF900C942D2FDF92EF92FF92E7
:106C80000F931F93CF93DF93D82E7B018A01E901E5
:106C90000E940E36D092671240E0B70185EF97E070
:106CA0000E941A360115110531F040E0B8018EEE50
:106CB00097E00E941A36209731F040E0BE018EEE38
:106CC00097E00E941A3660E081EE97E00E947735E7
:106CD00089EE97E00E94662F8AE0DF91CF911F91A5
:106CE0000F91FF90EF90DF900C942D2FAF92BF92F9
:106CF000CF92DF92EF92FF920F931F93CF93DF9388
:106D000083EF96E00E94662F6091F7087091F80873
:106D10008091F9089091FA0845E00E940BBD80EE41
:106D200096E00E94662FC0E0D9E0D15021F080E2C9
:106D30000E942D2FFACF8C2F0E9441E6CF5FC530E5
:106D400099F78AE00E942D2F0EEE1AE0C0E080E253
:106D50000E942D2F8C2F0E9441E65801D5E080E241
:106D60000E942D2FF501C080D180E280F380A70121
:106D70009601C701B6010F94CE2781112CC020E0E7
:106D800030E0A901C701B6010F943C2787FD03C07D
:106D90008BE20E942D2F45E0C701B6010E940BBD7A
:106DA000D15084E1A80EB11CD111D9CF8AE00E9444
:106DB0002D2FCF5F0C5F1F4FC53049F68AE0DF9162
:106DC000CF911F910F91FF90EF90DF90CF90BF90E8
:106DD000AF900C942D2FF12C80E20E942D2FF39474
:106DE0008DE3F8E0FF12F9CFDBCF811107C08BE113
:106DF0009FE00E94662F8AE00C942D2F8FE19FE088
:106E0000F8CFCF93DF93EB010E94662FCE01DF9185
:106E1000CF910C94FFE6CF93C62F0E94662F8C2F44
:106E2000CF910C9441E6CF92DF92EF92FF926A01EC
:106E30007B010E94662F42E0C701B601FF90EF90F0
:106E4000DF90CF900C940BBDCF92DF92EF92FF9228
:106E50006A017B010E94662F4AE0C701B601FF90DC
:106E6000EF90DF90CF900C94452FCF93DF93EB0101
:106E70000E94662FCE01DF91CF910C9448E64F928D
:106E80005F926F927F928F929F92AF92BF92CF92BA
:106E9000DF92EF92FF920F931F93CF93DF9300D077
:106EA00000D01F921F92CDB7DEB780915605811199
:106EB0000AC480915405909155059C012F5F3F4F66
:106EC00030935505209354058E3E924008F4FBC341
:106ED00080915312909154129093FE138093FD135E
:106EE00005E00093F11312E81093F41386E390E1A8
:106EF000A0E0B0E08093F5139093F613A093F713FE
:106F0000B093F81381EA93E10E94B82B8091E911C4
:106F10009091EA119093FE138093FD130093F11367
:106F20001093F4138CE390E1A0E0B0E08093F513AC
:106F30009093F613A093F713B093F81381EA93E1BB
:106F40000E94B82B80915512909156129093FE1387
:106F50008093FD130093F1131093F41384E390E1F5
:106F6000A0E0B0E08093F5139093F613A093F7138D
:106F7000B093F81381EA93E10E94B82B8091EB1152
:106F80009091EC119093FE138093FD130093F113F5
:106F90001093F4138AE390E1A0E0B0E08093F5133E
:106FA0009093F613A093F713B093F81381EA93E14B
:106FB0000E94B82B81E080935605109255051092DF
:106FC00054058091F80C882339F10E94021D81112B
:106FD00023C0809153058F5F8093530580915305A3
:106FE000853620F0109253051092F80CE091F80CC1
:106FF000E150E73008F06AC00E2E000CFF0B882726
:10700000EB5FF74C8F4F0D94C7240F385E382A3A48
:10701000563A973ACF3A623810925305DFCF0E9422
:10702000DC26882309F452C081E080936C0287EF4C
:1070300093E10E94662F8AE00E942D2F80E190E06C
:107040009093FE138093FD1385E08093F11312E873
:107050001093F41384E190E1A0E0B0E08093F51385
:107060009093F613A093F713B093F81381EA93E18A
:107070000E94B82B81E09AE59093FE138093FD1354
:1070800086E390E0909300148093FF1387E0809351
:10709000F1131093F41384E890E0A0E0B0E0809343
:1070A000F5139093F613A093F713B093F81381EAB6
:1070B00093E10E94B82B1092F80C08C00E94DC26C5
:1070C000882321F00E94021D8823A9F380916C027D
:1070D000882309F4D8C6809157058111C0C284E085
:1070E00096E09093FE138093FD1380EA90E89093CE
:1070F00000148093FF1317E01093F11302E800933C
:10710000F41380EA90E0A0E0B0E08093F513909350
:10711000F613A093F713B093F81381EA93E10E945A
:10712000B82B8091670290916802A0916902B0919A
:107130006A020097A105B10509F03FC21092FE1343
:107140001092FD1315E01093F1130093F4138AE8E5
:1071500090E1A0E0B0E08093F5139093F613A09334
:10716000F713B093F81381EA93E10E94B82B89E0FA
:1071700090E09093FE138093FD131093F11300930E
:10718000F4138CE890E1A0E0B0E08093F5139093C5
:10719000F613A093F713B093F81381EA93E10E94DA
:1071A000B82B8091670290916802A0916902B0911A
:1071B0006A020097F1E0AF07B10508F441C2B0934D
:1071C000FE13A093FD13909300148093FF1387E0A8
:1071D0008093F11382E88093F41388E890E1A0E0B3
:1071E000B0E08093F5139093F613A093F713B09348
:1071F000F81381EA93E10E94B82B80916702909185
:107200006802A0916902B0916A02BA2FA92F982F43
:107210008827009721E0A207B10508F417C2B093B0
:10722000FE13A093FD13909300148093FF1387E047
:107230008093F11312E81093F41381EA90E0A0E038
:10724000B0E08093F5139093F613A093F713B093E7
:10725000F81381EA93E10E94B82B8091FA0C8823FD
:1072600009F4FAC183E090E09093FE138093FD133C
:1072700085E08093F1131093F41385E490E1A0E08E
:10728000B0E08093F5139093F613A093F713B093A7
:10729000F81381EA93E10E94B82B80915705875E2D
:1072A0008093570520915705822F90E0253608F0EE
:1072B00021C29093FE138093FD1385E08093F11318
:1072C00082E88093F41380E090E1A0E0B0E0809346
:1072D000F5139093F613A093F713B093F81381EA84
:1072E00093E10E94B82B0E94021D811114C20E94DA
:1072F000D12A811105C090915A0591FD0E94021D6D
:1073000090915A0580FB91F990935A0591FD03C223
:1073100080918F1482FDFFC18091A3118150823032
:1073200008F4F9C16091EB117091EC11072E000C7B
:10733000880B990B0F94051E6B017C0120E030E057
:10734000A9010F94FE1D882309F460C66091E9111C
:107350007091EA11072E000C880B990B0F94051EF3
:107360002B013C0120E030E040E050E4C701B601D1
:107370000F94DB24A30192010F943C2718160CF400
:1073800067C66091531270915412072E000C880B3F
:10739000990B0F94051E6D837E838F839887609170
:1073A000551270915612072E000C880B990B0F94F2
:1073B000051E4B015C0120E030E040E251E40F94F7
:1073C000DB242D813E814F8158850F943C27181670
:1073D0000CF43EC620E030E040E050E4C701B601C6
:1073E0000F94DC24A30192010F94FE1D87FD10C0B1
:1073F00020E030E040E251E4C501B4010F94DC2408
:107400002D813E814F8158850F94FE1D87FF0FC649
:1074100084E190E09093FE138093FD1385E08093C8
:10742000F11382E88093F41384E190E1A0E0B0E0EE
:107430008093F5139093F613A093F713B093F8137A
:1074400081EA93E10E94B82B8091F30C811121C64F
:1074500082E01FC689EE93E10E94662F8AE00E94B7
:107460002D2F81E09AE59093FE138093FD1380E425
:1074700090E0909300148093FF1317E01093F113A2
:1074800082E88093F41384E890E0A0E0B0E0809379
:10749000F5139093F613A093F713B093F81381EAC2
:1074A00093E10E94B82B1093F80C10CE8091E40C5D
:1074B000882309F40BCE0E94DC26882309F406CE2B
:1074C0000E94021D811102CE8BED93E10E94662F76
:1074D0008AE00E942D2F8091E50C90E0B0E0A0E0C2
:1074E000895B9F4FAE4FB54A21E03AE53093FE13DA
:1074F0002093FD13909300148093FF1387E08093F3
:10750000F11382E88093F41384E890E0A0E0B0E007
:107510008093F5139093F613A093F713B093F81399
:1075200081EA93E10E94B82B1092E40CC4CD0E9432
:10753000DC26882309F4CACD0E94021D8111C6CD24
:1075400081E080936C021092F80C8DEC93E10E9424
:10755000662F8AE00E942D2F81E09AE59093FE131A
:107560008093FD138EE490E0909300148093FF13BA
:1075700087E08093F11382E88093F41384E890E02D
:10758000A0E0B0E08093F5139093F613A093F71367
:10759000B093F81381EA93E10E94B82B97CD0E9433
:1075A000021D811193CD19821A821B821C8262E016
:1075B000CE0101960E94E6EC7ECD0196A11DB11D83
:1075C00035E0B695A795979587953A95D1F70197A8
:1075D000A109B1090097E1E0AE07B10548F1B09308
:1075E000FE13A093FD13909300148093FF13109348
:1075F000F11312E81093F4138AE890E1A0E0B0E0F0
:107600008093F5139093F613A093F713B093F813A8
:1076100081EA93E10E94B82B88E090E09093FE13FA
:107620008093FD1385E08093F1131093F413A9CD9B
:107630009093FE138093FD1385E08093F113D9CFCF
:107640009093FE138093FD1385E0C2CD9093FE13BB
:107650008093FD1385E0ECCD82E090E005CE8A3F7B
:1076600008F020CE8EEF809357058CEB93E10E94BB
:10767000662F8AE00E942D2F81E080936C0281E0CA
:107680009AE59093FE138093FD138DE290E0909322
:1076900000148093FF1387E08093F11382E88093B6
:1076A000F41384E890E0A0E0B0E08093F5139093A9
:1076B000F613A093F713B093F81381EA93E10E94B5
:1076C000B82B1092560528960FB6F894DEBF0FBE61
:1076D000CDBFDF91CF911F910F91FF90EF90DF9081
:1076E000CF90BF90AF909F908F907F906F905F9062
:1076F0004F900895845691099093FE138093FD1343
:1077000085E08093F11382E88093F41381E090E1A7
:10771000A0E0B0E0DCCD8CE090E09093FE1380938D
:10772000FD1315E01093F11382E88093F41384E1C4
:1077300090E1A0E0B0E08093F5139093F613A0934E
:10774000F713B093F81381EA93E10E94B82B0E94DB
:10775000DC2520E13EE040E050E00F94422421157A
:10776000310581E04807510508F470C05093FE13BD
:107770004093FD13309300142093FF1387E0809310
:10778000F11312E81093F41380E190E1A0E0B0E06F
:107790008093F5139093F613A093F713B093F81317
:1077A00081EA93E10E94B82B0E94DC2520E13EE0B3
:1077B00040E050E00F9442242CE330E040E050E001
:1077C0000F9442243093FE132093FD1305E00093A1
:1077D000F1131093F41382E190E1A0E0B0E0809304
:1077E000F5139093F613A093F713B093F81381EA6F
:1077F00093E10E94B82B0E94DF2A882309F401C478
:107800008F5F80935205E82EF12C833330F5EE0C18
:10781000FF1CF092FE13E092FD130093F1131093FE
:10782000F4138EE090E1A0E0B0E08093F513909324
:10783000F613A093F713B093F81381EA93E10E9433
:10784000B82B1092FE131092FD132BC03093FE1331
:107850002093FD131093F11394CF84E690E090935E
:10786000FE138093FD130093F1131093F4138EE035
:1078700090E1A0E0B0E08093F5139093F613A0930D
:10788000F713B093F81381EA93E10E94B82BA2E3B7
:10789000EA1AA0E8FA0AEE0CFF1CF092FE13E0923E
:1078A000FD130093F1131093F4138FE090E1A0E027
:1078B000B0E08093F5139093F613A093F713B09371
:1078C000F81381EA93E10E94B82B0E94DF2A90E02E
:1078D0009093FE138093FD1385E08093F11382E86B
:1078E0008093F41386E190E1A0E0B0E08093F5137B
:1078F0009093F613A093F713B093F81381EA93E1F2
:107900000E94B82B0E94E42620E030E048EC52E4CC
:107910000F94641E0F9448267093FE136093FD131A
:1079200005E00093F11312E81093F41386E290E15E
:10793000A0E0B0E08093F5139093F613A093F713B3
:10794000B093F81381EA93E10E94B82B809136023C
:10795000909137029093FE138093FD130093F113DF
:107960001093F41380E093E1A0E0B0E08093F5136E
:107970009093F613A093F713B093F81381EA93E171
:107980000E94B82B20E030E040E251E460919C0C72
:1079900070919D0C80919E0C90919F0C0F94641E91
:1079A0000F944F267093FE136093FD130093F11311
:1079B0001093F41382E492E1A0E0B0E08093F51319
:1079C0009093F613A093F713B093F81381EA93E121
:1079D0000E94B82B20E030E040E251E46091A00C1E
:1079E0007091A10C8091A20C9091A30C0F94641E35
:1079F0000F944F267093FE136093FD130093F113C1
:107A00001093F41386E492E1A0E0B0E08093F513C4
:107A10009093F613A093F713B093F81381EA93E1D0
:107A20000E94B82B20E030E040E251E46091A40CC9
:107A30007091A50C8091A60C9091A70C0F94641ED8
:107A40000F944F267093FE136093FD130093F11370
:107A50001093F4138AE492E1A0E0B0E08093F51370
:107A60009093F613A093F713B093F81381EA93E180
:107A70000E94B82B20E030E040E251E46091A80C75
:107A80007091A90C8091AA0C9091AB0C0F94641E7C
:107A90000F944F267093FE136093FD130093F11320
:107AA0001093F4138EE492E1A0E0B0E08093F5131C
:107AB0009093F613A093F713B093F81381EA93E130
:107AC0000E94B82B80917302909174029093FE13E0
:107AD0008093FD130093F1131093F41382E592E168
:107AE000A0E0B0E08093F5139093F613A093F71302
:107AF000B093F81381EA93E10E94B82B8091710250
:107B0000909172029093FE138093FD130093F113F2
:107B10001093F41384E592E1A0E0B0E08093F513B4
:107B20009093F613A093F713B093F81381EA93E1BF
:107B30000E94B82B20E030E040E251E460915812FE
:107B40007091591280915A1290915B120F94641E99
:107B50000F944F267093FE136093FD130093F1135F
:107B60001093F41386E592E1A0E0B0E08093F51362
:107B70009093F613A093F713B093F81381EA93E16F
:107B80000E94B82B2CEA35EC47E25EE360915C1270
:107B900070915D1280915E1290915F120F94D625C4
:107BA00020E030E040E251E40F94641E0F944F2631
:107BB0007093FE136093FD130093F1131093F4136D
:107BC0008AE592E1A0E0B0E08093F5139093F6137C
:107BD000A093F713B093F81381EA93E10E94B82BB6
:107BE0002CEA35EC47E25EE360916012709161121D
:107BF00080916212909163120F94641E20E030E035
:107C000040E251E40F94641E0F944F267093FE13CC
:107C10006093FD130093F1131093F4138EE592E13A
:107C2000A0E0B0E08093F5139093F613A093F713C0
:107C3000B093F81381EA93E10E94B82B20E030E082
:107C400040E251E46091EE117091EF118091F011DA
:107C50009091F1110F94641E0F944F267093FE13B0
:107C60006093FD130093F1131093F41382E692E1F5
:107C7000A0E0B0E08093F5139093F613A093F71370
:107C8000B093F81381EA93E10E94B82B2CEA35EC0B
:107C900047E25EE36091F2117091F3118091F4116B
:107CA0009091F5110F94D62520E030E040E251E4A8
:107CB0000F94641E0F944F267093FE136093FD1370
:107CC0000093F1131093F41386E692E1A0E0B0E084
:107CD0008093F5139093F613A093F713B093F813D2
:107CE00081EA93E10E94B82B2CEA35EC47E25EE38F
:107CF0006091F6117091F7118091F8119091F9113E
:107D00000F94641E20E030E040E251E40F94641EC2
:107D10000F944F267093FE136093FD130093F1139D
:107D20001093F4138AE692E1A0E0B0E08093F5139B
:107D30009093F613A093F713B093F81381EA93E1AD
:107D40000E94B82B8091EE0C811105C08091F00C3F
:107D5000882309F46DC06091531270915412072E5C
:107D6000000C880B990B0F94051E20E030E048ECC6
:107D700052E40F94641E6B017C0160915512709166
:107D80005612072E000C880B990B0F94051E9B01B1
:107D9000AC01C701B6010F94D6250F944F26653666
:107DA000710510F064E670E07093FE136093FD13AC
:107DB00005E00093F11312E81093F41384E290E1CC
:107DC000A0E0B0E08093F5139093F613A093F7131F
:107DD000B093F81381EA93E10E94B82B609153129B
:107DE00070915412072E000C880B990B0F94051EEE
:107DF0006B017C0120E030E04AE253E40F943C2721
:107E0000181624F48091EE0C811146C16091551230
:107E100070915612072E000C880B990B0F94051EBB
:107E20009B01AC01C701B6010F943C2787FFAFC18E
:107E30008091E40C882339F18091E30C91E0980F54
:107E40009093E30C90E09093FE138093FD1385E0F4
:107E50008093F11382E88093F41382E490E1A0E030
:107E6000B0E08093F5139093F613A093F713B093BB
:107E7000F81381EA93E10E94B82B8091E30C8A30D9
:107E800010F01092E30C0E946726882309F4B5C114
:107E90006091F60C7091F70CEE24E394F12C6115CF
:107EA0007105A9F090E080E00F94031E20E030E01F
:107EB00040E85EE30F94641E0F94BA2520E030E0A2
:107EC00040E85FE30F94DC240F944F267B0101E030
:107ED00010E08091E00C811102C010E000E0809180
:107EE000E5129091E6128F3F980711F40E9472B646
:107EF0009093E6128093E512080F191FB80190E0E5
:107F000080E00F94031E20E030E040E85EE30F9431
:107F1000641E0F94BA254B015C01F092FE13E092AF
:107F2000FD1305E00093F11312E81093F41380E1C0
:107F300093E1A0E0B0E08093F5139093F613A09343
:107F4000F713B093F81381EA93E10E94B82BC501AF
:107F5000B4010F944F267093FE136093FD130093AA
:107F6000F1131093F41382E193E1A0E0B0E0809369
:107F7000F5139093F613A093F713B093F81381EAD7
:107F800093E10E94B82B01E414E1AAE1FA2E80915A
:107F90000E0590910F052091500530915105891BD8
:107FA0008F7309F449C12A3131050CF0DBC190917E
:107FB0000E0580910F054FEF5FEF981749F0E82FFE
:107FC000F0E0E25FFA4F42818F5F8F7380930F057D
:107FD000F901EF5BFB4E4083809141148A3509F033
:107FE000B3C162E070E080E090E00E94A62A809138
:107FF000500590915105019690935105809350053D
:10800000C6CF1092FE131092FD1307CC609155124B
:1080100070915612072E000C880B990B0F94051EB9
:1080200020E030E0A9010F94FE1D81118FC98CE082
:1080300090E09093FE138093FD1385E08093F113FD
:1080400082E88093F41384E190E1A0E0B0E04ECCAC
:108050008DE090E09093FE138093FD1385E0809374
:10806000F11382E88093F41384E190E1A0E0B0E0A2
:108070008093F5139093F613A093F713B093F8132E
:1080800081EA93E10E94B82B8091F30C811101C029
:1080900081E08093F30C36CC1092EE0C20E030E0BF
:1080A00040E251E46091E60C7091E70C8091E80C9D
:1080B0009091E90C0F94641E0F9448267093FE1360
:1080C0006093FD130093F1131093F41384E590E192
:1080D000A0E0B0E08093F5139093F613A093F7130C
:1080E000B093F81381EA93E10E94B82B20E030E0CE
:1080F00040E251E46091EA0C7091EB0C8091EC0C41
:108100009091ED0C0F94641E0F9448267093FE130B
:108110006093FD130093F1131093F41388E590E13D
:10812000A0E0B0E08093F5139093F613A093F713BB
:10813000B093F81381EA93E10E94B82B8BE993E1A5
:108140000E94662F8AE00E942D2F81E09AE590938D
:10815000FE138093FD1381E490E0909300148093CC
:10816000FF1387E08093F1131093F41384E890E0F9
:10817000A0E0B0E08093F5139093F613A093F7136B
:10818000B093F81381EA93E10E94B82B51CE60912D
:10819000F00C662309F44CCE062E000C770B82E817
:1081A00093E10E9435378AE00E942D2F1092F00C47
:1081B00084E090E09093FE138093FD1385E080931C
:1081C000F11312E81093F4138EE890E1A0E0B0E010
:1081D0008093F5139093F613A093F713B093F813CD
:1081E00081EA93E10E94B82B81E09AE59093FE1317
:1081F0008093FD1383E590E0B0CF1092FE131092B0
:10820000FD1305E00093F11312E81093F41380E1DD
:1082100093E1A0E0B0E08093F5139093F613A09360
:10822000F713B093F81381EA93E10E94B82B1092F0
:10823000FE131092FD1393CE121613060CF492C087
:108240008091A5139091A613A091A713B091A813A4
:108250008C34E0E19E07A105B10509F432CA8A34E5
:108260009041A105B10509F42CCA20E030E040E2BC
:1082700051E46091FB0C7091FC0C8091FD0C90918D
:10828000FE0C0F94641E0F9448267093FE136093A7
:10829000FD1305E00093F11312E81093F41388E442
:1082A00090E1A0E0B0E08093F5139093F613A093D3
:1082B000F713B093F81381EA93E10E94B82B20E002
:1082C00030E040E251E46091FF0C7091000D80912C
:1082D000010D9091020D0F94641E0F944826709327
:1082E000FE136093FD130093F1131093F4138AE4CB
:1082F00090E1A0E0B0E08093F5139093F613A09383
:10830000F713B093F81381EA93E10E94B82B20E0B1
:1083100030E040E251E46091030D7091040D8091D2
:10832000050D9091060D0F94641E0F9448267093CE
:10833000FE136093FD130093F1131093F4138CE478
:1083400090E1A0E0B0E0B1C9121613060CF01FCE08
:10835000F8012F2D11922A95E9F7109251051092EC
:10836000500515CE9091A21380914114981321C00D
:108370009091A3138091421498131BC023303105B0
:10838000C4F0909143149093A1138091441480936E
:10839000A4139330D1F4982F9D7F9038B1F490912D
:1083A00045149F3409F059C0909146149B3409F04C
:1083B00054C0E1E4F4E18AE1DF011D928A95E9F716
:1083C00010925105109250053BCF833809F045C0FB
:1083D0008091451490914614982789279827B0E0FA
:1083E000A0E08093A5139093A613A093A713B09336
:1083F000A813C0904714D12CF12CE12CC092A913E2
:10840000D092AA13E092AB13F092AC1328E434E1BB
:1084100040E050E0BA014C155D056E057F0508F09F
:108420004AC0DB01CA01B695A79597958795069630
:10843000880F991FFC01EF55FC4ED9018C911196C4
:108440009C91892798278927918380834E5F5F4F6E
:108450006F4F7F4F2E5F3F4FDECF813861F58091A8
:10846000451490E0B0E0A0E08093A5139093A6138C
:10847000A093A713B093A81380914614482F50E0FF
:1084800070E060E04093A9135093AA136093AB137C
:108490007093AC13A7E4B4E1EDEAF3E190E030E0CF
:1084A00020E08217930739F04D9150E041935193AA
:1084B0002F5F3F4FF6CFE1E4F4E18AE1DF011D9247
:1084C0008A95E9F710925105109250050E948EF599
:1084D000B7CE8111B0C084E49CE00E94662F409129
:1084E0004A0950914B0960914C0970914D098CE6F5
:1084F0009CE00E94133740915209509153096091BA
:108500005409709155098DEE9BE20E9413374091FA
:108510004E0950914F09609150097091510986EFB1
:108520009BE20E9413376091560970915709072EFC
:10853000000C880B990B0F94051EAB01BC0180EF5A
:108540009BE20E9413376091580970915909072ED8
:10855000000C880B990B0F94051EAB01BC0189E63A
:108560009CE00E94133760915A0970915B09072EB5
:10857000000C880B990B0F94051EAB01BC0186E61D
:108580009CE00E94133760915E0970915F0983E659
:108590009CE00E943537609160097091610980E626
:1085A0009CE00E94353760917A0970E08DE59CE08F
:1085B0000E9435376091790970E090E080E00F9477
:1085C000031EAB01BC018AE59CE00E941337609159
:1085D000620970E090E080E00F94031EAB01BC01E3
:1085E00087E59CE00E94133740916309509164092C
:1085F000609165097091660981E89AE10E941337DC
:1086000040916709509168096091690970916A0900
:108610008CEF9BE20E94133740916B0950916C09DB
:1086200060916D0970916E0989EF9BE20E9413378A
:108630008AE00C942D2F80E59CE04FCF89ED96E0E9
:108640000C94662FCF92DF92EF92FF920F931F93BD
:10865000CF93DF9388E50E948D1DD82E89E40E9478
:108660008D1DC82E8823D1F10E944522D82F89E57F
:108670000E948D1D182F8AE40E948D1D082F8823CB
:1086800009F455C00E944522C82F8AE50E948D1D1D
:10869000E82EF12C811104C081E50E948D1DF82E79
:1086A000C11001C000E0802F90E0D11001C010E0A7
:1086B000810F911D019721F4E11062C0F11060C09B
:1086C0000E941E4384E29CE0DF91CF911F910F91A5
:1086D000FF90EF90DF90CF900C94662FD11002C0E6
:1086E000DFEFC5CF0E94582220913B0C30913C0C0B
:1086F00040913D0C50913E0C0F94DB2420E030E083
:1087000040EA51E40F94DB2420E030E042E052E400
:108710000F94DC2421EC3FE04CE75CE30F94641EF3
:108720000F944826D62F653008F4A1CFD9CF111168
:1087300002C0CFEFAACF0E94582220913F0C309167
:10874000400C4091410C5091420C0F94DB2420E0EE
:1087500030E040EA51E40F94DB2420E030E042E0D6
:1087600052E40F94DC2421EC3FE04CE75CE30F94EF
:10877000641E0F944826C62F653008F486CFD9CFE3
:10878000D7FD02C0C7FF05C00E941E438BE09CE0DE
:108790009BCF0E9458229B01AC010D2FDD0F110BC6
:1087A000AC2FCC0FBB0B60E070E0CB01FF2091F051
:1087B00065E0609FF001619FF00D1124EA0FFB1F3F
:1087C000EE0FFF1FEE0FFF1FE251F54F6081718129
:1087D00082819381E5E0E09FE001E19FD00D1124CB
:1087E000CA0FDB1FCC0FDD1FCC0FDD1FC251D54FD1
:1087F0000F94DC24688379838A839B83DF91CF91F4
:108800001F910F91FF90EF90DF90CF90089583ED2F
:1088100096E00C94662F0F931F93CF93811113C092
:10882000C42F8B010E94074488E899E10E94662FBB
:10883000C8010E94662FCC2331F08AE0CF911F91AE
:108840000F910C942D2FCF911F910F91089584E6D5
:1088500090E09093E5088093E4081092110910923B
:1088600010090C94B1E1CF9384E50E94DB1DC09107
:10887000F90C8823D9F00E940022C82F8230B4F06E
:108880000E9407448DE40E942D2F8091090590914C
:108890000A050E94FFE66C2FCC0F770B8EE39DE05C
:1088A0000E9435378AE00E942D2FCFEF8C2FCF9179
:1088B00008955F926F927F928F929F92AF92BF9234
:1088C000CF92DF92EF92FF920F931F93CF93DF939C
:1088D0001F92CDB7DEB77C0139018B015B01A40E7D
:1088E000B51ED12CC12CA016B10609F450C0F70159
:1088F00080809180F80151908F015982C4010F94BA
:108900001C245816B9F1652DC4010F942424FFEFDF
:10891000CF1ADF0AC6018F779927892B21F162E0F0
:1089200070E080E090E00E94D2F4C4010F941C2417
:1089300099818917F9F00E9407448FE394E00E941F
:10894000662F81E00F90DF91CF911F910F91FF90E3
:10895000EF90DF90CF90BF90AF909F908F907F90DF
:108960006F905F90089562E070E080E090E00E9478
:10897000772ADBCFBE016F5F7F4FC3010E94CFE537
:10898000F70180819181019691838083ACCF80E053
:10899000D9CFCF92DF92EF92FF920F931F93CF9395
:1089A000DF93CDB7DEB7CA5AD1090FB6F894DEBF50
:1089B0000FBECDBFCF55DF4F188219821A821B829E
:1089C000C15AD0408091C8039091C903A091CA03B5
:1089D000B091CB03CB55DF4F88839983AA83BB83A8
:1089E000C55AD04084E690E09093E5088093E4086F
:1089F00010921109109210091092120920E139E029
:108A000044E050E0BE016B557F4F84EE98E00E9439
:108A100059448091E4089091E50802969093E50806
:108A20008093E408109211091092100981E0C65554
:108A3000DF4F8883CA5AD040CE0186559F4F0E948F
:108A400036D920E139E048E450E068E87CE084EE83
:108A500098E00E94594420E139E040E150E06FEF96
:108A600078E084EE98E00E9459448AE097EDA3EA0A
:108A7000BCE3CF55DF4F88839983AA83BB83C15A58
:108A8000D040CE018F559F4F0E9448D98CE69BE085
:108A90000E943FD97E018DE6E80EF11C8FEFD701D1
:108AA0008C93C7010E9436D919821A821B821C82BC
:108AB0008E010F5F1F4FC8010E9448D98091370C6B
:108AC0009091380CA091390CB0913A0C89839A831B
:108AD000AB83BC83C8010E9448D985E08983F70134
:108AE000808387EF98E00E9448D9C8010E9436D958
:108AF000C7010E9436D920E139E044E650E06EEE2D
:108B00007AE084EE98E00E9459448CE0D8011D92EE
:108B10008A95E9F7C8010E943FD9CF55DF4F1882E7
:108B200019821A821B82C15AD0403AE0D32EDA94BD
:108B3000DD2031F0CE018F559F4F0E9448D9F7CFED
:108B400088E0F701982F11929A95E9F7D8011D92C4
:108B50008A95E9F783E0C755DF4F8883C95AD0402B
:108B6000C356DF4F8883CD59D040CE0187559F4FE4
:108B70000E9436D9CE0183569F4F0E9436D920E1FC
:108B800039E048E050E0B80184EE98E00E94594492
:108B900020E139E048E050E0B70184EE98E00E941F
:108BA0005944CF55DF4F188219821A821B82C15A4D
:108BB000D0402AE0C22ED12CB1E0CB1AD10831F03E
:108BC000CE018F559F4F0E9448D9F6CF19828FEF63
:108BD000F7018083C8010E942DD9C7010E9436D9B0
:108BE00080E1D82ED801ED2D1D92EA95E9F720E11C
:108BF00039E040E150E0B80184EE98E00E94594429
:108C00001982C8010E942DD9198A1A8A1B8A1C8AC6
:108C100080E090E0A0E8BFE38D879E87AF87B88BA8
:108C20008091581290915912A0915A12B0915B12F2
:108C300089839A83AB83BC832CEA35EC47E25EE3FD
:108C400060915C1270915D1280915E1290915F1242
:108C50000F94D6256D837E838F8398872CEA35EC1D
:108C600047E25EE36091601270916112809162123E
:108C7000909163120F94641E69877A878B879C8713
:108C800020E139E044E150E0B80184EE98E00E9430
:108C9000594484E190E09A838983C8010E941BD9DA
:108CA0008091EE119091EF11A091F011B091F1111E
:108CB00089839A83AB83BC832CEA35EC47E25EE37D
:108CC0006091F2117091F3118091F4119091F5116E
:108CD0000F94D6256D837E838F8398872CEA35EC9D
:108CE00047E25EE36091F6117091F7118091F811FF
:108CF0009091F9110F94641E69877A878B879C87FE
:108D0000C8010E9424D98CE0E9E7F2E0D801019083
:108D10000D928A95E1F7C8010E9424D91982C801F1
:108D20000E9436D98FE790E09A838983C8010E9418
:108D30001BD985E0E5E8F2E0D80101900D928A9513
:108D4000E1F720E139E045E050E0B80184EE98E039
:108D50000E9459448091F6088983C8010E942DD948
:108D600080E2EAE8F2E0D80101900D928A95E1F7FD
:108D700020E139E040E250E0B80184EE98E00E9442
:108D80005944D7011C92C7010E942DD98FE59BE061
:108D90000E942DD920E139E048E050E067E57BE012
:108DA00084EE98E00E945944CF55DF4F1882198213
:108DB0001A821B82C15AD040CE018F559F4F0E940C
:108DC00048D9CE018F559F4F0E9448D980E2F801C3
:108DD00011928A95E9F720E139E040E250E0B801CC
:108DE00084EE98E00E945944FE01F99688E0DF0184
:108DF0001D928A95E9F744E650E060E070E049830F
:108E00005A836B837C834D835E836F83788783E093
:108E100090E0A0E0B0E089879A87AB87BC874D8758
:108E20005E876F87788B498B5A8B6B8B7C8B8D8B96
:108E30009E8BAF8BB88F898F9A8FAB8FBC8F8D8FA6
:108E40009E8FAF8FB8A38EE190E0A0E0B0E089A341
:108E50009AA3ABA3BCA38DA39EA3AFA3B8A789A7D6
:108E60009AA7ABA7BCA78DA79EA7AFA7B8AB89ABA6
:108E70009AABABABBCAB8DAB9EABAFABB8AF20E1AD
:108E800039E040E450E0B80184EE98E00E94594493
:108E9000F8018D2D11928A95E9F720E139E040E142
:108EA00050E0B80184EE98E00E945944D8011D9228
:108EB000DA94E9F720E139E040E150E0B80184EECE
:108EC00098E00E94594420E139E048E050E060E732
:108ED00079E084EE98E00E9459449CE0D92EF80194
:108EE0008D2D11928A95E9F720E139E04CE050E0B0
:108EF000B80184EE98E00E9459448CE6D8011D9296
:108F00008A95E9F720E139E04CE650E0B80184EEBB
:108F100098E00E94594488ED98E00E9424D920E10D
:108F200039E040E150E066EE78E084EE98E00E949F
:108F3000594420E139E045E250E06AE479E084EE0A
:108F400098E00E945944F7011192DA94E9F7C75565
:108F5000DF4F1882C95AD04080E090E0A0E4B0E42E
:108F6000C356DF4F88839983AA83BB83CD59D040F2
:108F7000C7010E943FD9CE0187559F4F0E9436D925
:108F8000CE0183569F4F0E9448D980E3D7011D929E
:108F90008A95E9F78AEF98E10E94662F8AE00E949D
:108FA0002D2F20E139E040E350E0B70184EE98E056
:108FB0000E94594480911209811128C00091E4084F
:108FC0001091E5088091100990911109F7019183A2
:108FD000808384E690E09093E5088093E40820E1A4
:108FE00039E044E050E061EF72E084EE98E00E94E6
:108FF0005944C7010E941BD991E00A3A134009F471
:1090000090E080911209892B8093120980911209B6
:10901000811105C060E08EE299E10E94AA358EE0E0
:1090200099E10E94662F8AE00E942D2F90911209EB
:1090300081E08927C655DF4F0FB6F894DEBF0FBE1B
:10904000CDBFDF91CF911F910F91FF90EF90DF90F7
:10905000CF900895CF93DF9300D01F92CDB7DEB7A6
:109060008091F2098823C1F083E390E09C838B8395
:109070001A8219829E012F5F3F4F40E150E063EF5B
:1090800079E0CE0103960E9459448EE099E10E9456
:10909000662F8AE00E942D2F0F900F900F900F9057
:1090A000DF91CF910895CF92DF92EF92FF92CF930D
:1090B000C82F8091A3118150823008F069C00E94AE
:1090C0009A311092A3110E9405F56093D008709315
:1090D000D1088093D2089093D308C090D408D09040
:1090E000D508E090D608F090D7080E94DC25AB01A7
:1090F000BC014093D4085093D5086093D608709370
:10910000D7088091F7099091F809A091F909B091D9
:10911000FA098C199D09AE09BF09840F951FA61F76
:10912000B71F8093F7099093F809A093F909B093BA
:10913000FA09C1110AC0C1E00E942A488C2FCF91C0
:10914000FF90EF90DF90CF9008958091F509909176
:10915000F60901969093F6098093F5090E94DC25A3
:10916000C090FB09D090FC09E090FD09F090FE0949
:10917000C616D706E806F906F0F60E94DC256093CD
:10918000FB097093FC098093FD099093FE09D3CFEE
:10919000C0E0D2CFCF93DF9300D01F921F92CDB704
:1091A000DEB781E08093F20980E1E3EFF9E0DF01CF
:1091B0001D928A95E9F70E942A4886E18D8382E311
:1091C00090E09C838B831A8219829E012F5F3F4F10
:1091D00041E050E0BE016B5F7F4FCE0103960E94DD
:1091E00059440F900F900F900F900F90DF91CF91F7
:1091F0000895CF93DF93CDB7DEB7A8970FB6F89455
:10920000DEBF0FBECDBF8C01F42E0E949EC40E9413
:109210001E4383EB96E00E94662F0115110511F4A1
:109220000AEA16E080915A0580FD79C0816080933A
:109230005A0586E996E00E94662F8AE00E942D2F4B
:10924000CC24C3948AE5D82ED092FE13C092FD138D
:109250008FE090E0909300148093FF1397E0792EB5
:109260007092F11322E8E22EE092F41334E8832E98
:10927000912CA12CB12C8092F5139092F613A09210
:10928000F713B092F81381EA93E10E94B82BD092C1
:10929000FE13C092FD1388E590E090930014809334
:1092A000FF137092F113E092F4138092F5139092F1
:1092B000F613A092F713B092F81381EA93E10E949B
:1092C000B82B8AE289838A838B838C83F801DE0141
:1092D0001596BE016F5F7F4FCD01861B970B2491C2
:1092E000319621110CC0FB01E80FF91F8AE29F01A2
:1092F000261B370B2832310524F48193F8CF2D93A8
:10930000EBCF20E630E140E050E081EA93E10E94BB
:10931000EAE56AE070E080E090E00E94A62A61E061
:1093200081EA96E00E94773589EE93E030E6019776
:1093300029F0232F2A950000E9F7F9CFF89489EE58
:1093400093E038EE019729F0232F2A950000E9F7E2
:10935000F9CF0E949EC4FF2031F00E94EB1D0E94B5
:10936000041EA895FECF0E94E81DF9CF8091470A00
:10937000882319F01092470A089540E070E060E0F9
:1093800085E095E10E94F94880910B0D90910C0DBC
:109390002FEF3FEF981751F0E92FF0E0E55FF24F24
:1093A000228130E09F5F9F7790930C0DC901089553
:1093B0001F920F920FB60F9211240F900FBE0F90B5
:1093C0001F9018951F920F920FB60F9211240BB693
:1093D0000F920F931F932F933F934F935F936F932E
:1093E0007F938F939F93AF93BF93CF93DF93EF932D
:1093F000FF93C091C60000910C0DD0910B0D11E0B0
:109400001D0F1F7790910F04913108F09FC0E92F35
:10941000F0E08827E15FF54B8F4F0D94C724204A79
:109420004F4A5E4A6D4A744AA64A784AA64A7C4A1E
:10943000804AA64A844A884A8C4A934AA64A9E4A47
:10944000C03229F028F5CA3011F0CD3031F50117BE
:1094500031F0ED2FF0E0E55FF24FC283D12FD093D2
:109460000B0DFF91EF91DF91CF91BF91AF919F9144
:109470008F917F916F915F914F913F912F911F91AC
:109480000F910F900BBE0F900FBE0F901F9018956D
:10949000CD3481F081E0CE3471F080E10CC0CA336C
:1094A00038F4C033A0F6C03291F2CD32B1F7CFCF4D
:1094B000CD3499F782E080930F04C9CFC13359F0BE
:1094C00018F4C03221F2E9CF88E0C433A1F38BE075
:1094D000C83389F3E2CF83E0EECF84E0C03359F3A1
:1094E00086E0C13341F3D9CF85E0C833B1F6E3CF8D
:1094F00087E0C23391F6DFCF89E0C13371F6DBCF6D
:109500008AE0C03351F6D7CF8CE0C73331F6D3CFE2
:109510008DE0C63311F6CFCFC03209F498CF8EE07C
:10952000C33549F2BACF80ED8C0F8A3008F08FCF67
:109530009FE090930F048093100489CFCA3019F0F4
:10954000CD3009F084CF10920F0481CFCA3019F0CA
:10955000CD3009F07CCF80915B148823A1F3973044
:1095600079F038F4953079F710924602109266122D
:10957000EACF9A3049F09F3031F70E94BCE5E3CF43
:1095800081E080933A09DFCF81E080933909DBCF16
:109590008EBD0DB407FEFDCF08958FEF8EBD0DB4C7
:1095A00007FEFDCF8EB50895909164009B7F909348
:1095B0006400982F906A96959CBD80FD03C091E051
:1095C000863009F490E09DBD0895CF93DF93EB01C1
:1095D0000E94662FCE01DF91CF910C94DAB12F92C9
:1095E0003F924F925F926F927F928F929F92AF9233
:1095F000BF92CF92DF92EF92FF920F931F93CF9380
:10960000DF93009709F0AAC11092E20C1092E10CCE
:109610009093590580935805BAE0CB2EB0E2DB2E2B
:10962000E12CF12C15E002E846015701C4E1D0E03D
:1096300010924413109243131093371300933A136C
:1096400080923B1390923C13A0923D13B0923E1334
:1096500087EE92E10E94B82B21972FEF821A920A8F
:10966000A20AB20A209721F744E1C40ED11CE11CE2
:10967000F11C8AE5C81680E2D806E104F104A1F6DF
:10968000C12CA0E2DA2EE12CF12CD5E0C2E8109238
:10969000441310924313D0933713C0933A13C092DC
:1096A0003B13D0923C13E0923D13F0923E1387EEB1
:1096B00092E10E94B82B1092441310924313D0935E
:1096C0003713C0933A13D701C6018C529F4FAF4F47
:1096D000BF4F80933B1390933C13A0933D13B093E3
:1096E0003E1387EE92E10E94B82BEFEFCE1ADE0A0E
:1096F000EE0AFE0AFAE0CF16F0E2DF06E104F1041A
:1097000031F6FEEDCF2EF0E2DF2EE12CF12CD5E08C
:10971000C2E81092441310924313D0933713C093AE
:109720003A13C0923B13D0923C13E0923D13F09257
:109730003E1387EE92E10E94B82B2FEFC21AD20A95
:10974000E20AF20A46EEC41640E2D406E104F1044D
:1097500001F7CC24C394E2E1DE2EE12CF12C0AE0E7
:1097600010E0D5E0C2E81093441300934313D09364
:109770003713C0933A13C0923B13D0923C13E0923C
:109780003D13F0923E1387EE92E10E94B82B1093A6
:10979000441300934313D0933713C0933A13D70164
:1097A000C6018096A11DB11D80933B1390933C137D
:1097B000A0933D13B0933E1387EE92E10E94B82B25
:1097C0008FEFC81AD80AE80AF80AE5E0CE16E2E1F7
:1097D000DE06E104F10439F60091E10C1091E20C8F
:1097E0000115110509F0D6C08091E00C882309F419
:1097F000E1C02AE030E240E050E06CEC73E087EE3C
:1098000092E10E94EAE5C1E0D0E003E010E0E090E0
:10981000E10CF090E20C35E0332E42E8242E442493
:109820004A94542C64E0662E712C7FE1C72E74E0BC
:10983000D72E8091E10C9091E20C800F911FE816D9
:10984000F90608F0D5C0C7010E9405E7882309F48E
:1098500081C0809107126AEF71E1882311F067E0FF
:1098600072E1FB0101900020E9F7CF010197861B0F
:10987000970BF4E1FC9F9001FD9F300D1124265FB2
:109880003F4D50E040E0459710F0FB01128A87EE13
:1098900092E10E94EAE5CE018F5F9D4EB0E0A0E02C
:1098A00021964E0124E0880C991C2A95E1F7FDEFE2
:1098B0008F1AFFE99F0AB12CA12C20918F1424FF4D
:1098C0007EC07092441360924313309237132092FB
:1098D0003A1380933B1390933C13A0933D13B093A2
:1098E0003E1387EE92E10E94B82BD0924413C092AF
:1098F00043133092371320923A1380923B13909285
:109900003C13A0923D13B0923E1387EE92E10E9469
:10991000B82BB7018CE394E10E94013780910712C4
:1099200067E072E1811102C06AEF71E189E394E1BD
:109930000E94E54A67E47CE085E394E10E94E54A01
:109940006AEF71E184E394E10E94E54A80E394E1E7
:109950000E94662F2FEFE21AF20A6BCF2091E10CE2
:109960003091E20CA9014150510960915805709164
:1099700059056817790738F42C5F3F4F3093E20C94
:109980002093E10C45CE4430510508F43DCE2450DF
:109990003109F4CF0430110569F48091E00C88237B
:1099A00031F083E090E09093E20C8093E10CD0E002
:1099B000C0E02DCFD0E0C0E004E010E028CF10924E
:1099C0004413109243133092371320923A1380932A
:1099D0003B1390933C13A0933D13B0933E1387EE3B
:1099E00092E10E94B82B509244134092431381CFCE
:1099F000DF91CF911F910F91FF90EF90DF90CF906B
:109A0000BF90AF909F908F907F906F905F904F909E
:109A10003F902F900895AF92BF92CF92DF92EF9236
:109A2000FF920F931F93CF93DF93CDB7DEB7E697E7
:109A30000FB6F894DEBF0FBECDBF00910C0510919C
:109A40000D05F80101900020E9F731976F01C01A68
:109A5000D10AF801CF01801B910B8C159D053CF4B8
:109A600081918F32B9F7DF0111971C92F3CF8BE10F
:109A7000EFEAF4E1DE015C9601900D928A95E1F740
:109A8000F12CE12CEC14FD040CF05DC0F801EE0D9E
:109A9000FF1D8081811103C08FEFE81AF80A580179
:109AA000AE0CBF1CF5018081882309F44CC0FFEF88
:109AB000EF1AFF0AF801EE0DFF1D7F01E01AF10A0F
:109AC00081918111FACFCE014C960E946DB68BE147
:109AD000FE017C96DE01119601900D928A95E1F7C8
:109AE000B501CE0101960E947BAECE0101960E9487
:109AF000F2288FE20E942D2F8091071281113BC026
:109B000089ED93E00E94DAB180918F1484FF1BC02D
:109B100019821C8221E0A501BE01645E7F4FCE0147
:109B200001960E94AFB8811129C08AE00E942D2FB2
:109B30000E940744B5018BE193E10E94E54ACE0102
:109B400001960E94F2288AE00E942D2FCE014C96A9
:109B50000E94F228E6960FB6F894DEBF0FBECDBF86
:109B6000DF91CF911F910F91FF90EF90DF90CF90F9
:109B7000BF90AF90089587E092E1C4CFCE014C969C
:109B80000E94DCB58BE1FE013196DE015C9601900E
:109B90000D928A95E1F7CE0101960E94F22872CFCC
:109BA0002F923F924F925F926F927F928F929F92ED
:109BB000AF92BF92CF92DF92EF92FF920F931F93DB
:109BC000CF93DF9300D000D000D01F921F92CDB76B
:109BD000DEB7B82E8091080E843008F0D1C10E9403
:109BE00005F56B017C018091080E811108C0809100
:109BF0000B0D90910C0D891B8F7709F4FDC581E643
:109C0000A82E13C08A3019F08D3009F0F6C01092DA
:109C1000F30D8091910D9091920DFC01E357F24F5D
:109C20001682892BF1F40E94F0C78091080E8430CF
:109C300008F0ECC080910B0D90910C0D891B8F7773
:109C400009F4E4C00E94C44997FFDCCF0E941E4380
:109C500085E895E00E94662F80910B0D80930C0D96
:109C6000E4CF1092920D1092910D03E91DE0F801DE
:109C70008191803209F446C08E3409F0A9C060E8B1
:109C800075E0C8010F947B1D4C01892B41F06EE4F7
:109C900070E0C80104960F942A28009709F4C801BF
:109CA0004AE050E070E060E001960F94EB1A2B015F
:109CB0003C0180918D0D90918E0DA0918F0DB091F2
:109CC000900D0196A11DB11D481659066A067B0626
:109CD00029F060E08DE495E0892851F16AE270E0B6
:109CE000C8010F9459289C01009729F1982F901BC7
:109CF000912C992349F09150F801E90FF11D8081D1
:109D00009826F7CF8F01B3CF4AE050E070E060E0D3
:109D1000C90101960F94EB1A292D30E050E040E084
:109D2000621773078407950751F060E08EE295E0B3
:109D30000E9452EC7ACF60E084E095E0F9CF409247
:109D40008D0D50928E0D60928F0D7092900D8091BE
:109D5000480A8130E1F067E470E0C8010F942A28D6
:109D60000097A9F04AE050E070E060E001960F949F
:109D7000EB1A643071058105910548F483E694E09F
:109D80000E94662F60E089E594E00E94AA35C092A7
:109D9000EA0AD092EB0AE092EC0AF092ED0A809186
:109DA000930D8B3309F441CF8091080E843008F075
:109DB0003CCF80910A0E8A9DC001112463E97DE0A9
:109DC000855F914F0F94352880E00E940CEC2DCFD9
:109DD00080918F1480FFBBCF6BE27AE2C8010F94B1
:109DE0007B1D009731F0FC01838180538A3008F09D
:109DF000AECF60E08AED94E09BCF21E93DE043E9FE
:109E00005DE063EF7DE00E941C1D0FCF80918F14F9
:109E100082FFB6C01A82198271E6F72EE0E1EE2EBB
:109E2000F9E6DF2E8091080E843008F0A9C00E9468
:109E3000541D8111A5C041E050E0BE016B5F7F4F12
:109E400083EF95E10E942FB40D8110E0019711F08E
:109E50000FEF1FEF8091FB159091FC15A091FD1560
:109E6000B091FE1580938B1490938C14A0938D1455
:109E7000B0938E140E94541D0F3F100749F48111B6
:109E800007C00E941E4383EA95E00E94662FCACF56
:109E900040910A0E242F30E00A3061F00D3051F06D
:109EA000882309F45FC089819A81009719F001968F
:109EB0009A8389831092940489819A81F29EF00199
:109EC000F39EF00D1124E85FF14FE80FF91F1382A4
:109ED000892B69F50E94F0C70E94541D882309F45C
:109EE000A1CF0E94366683EF95E10E94DCB5809198
:109EF0008614882391F18150809386148D9DC00132
:109F0000112462E08058964F0E9431BBE091861484
:109F100024E0E29FF0011124E458F64F6081718142
:109F2000828193810E94C4210E94E4AD7BCF1A827A
:109F3000198281E00E940CEC80918B1490918C141A
:109F4000A0918D14B0918E148093040E9093050E01
:109F5000A093060EB093070EBFCF0E94E5B5E09226
:109F6000480A60CF4F9DA0011124455F514F9E01CB
:109F70002F5F3F4F64E974E0802F0E941C1D52CF79
:109F80000E9405F56B017C01B11004C08091A21103
:109F9000882351F0C0929A11D0929B11E0929C11AB
:109FA000F0929D11BB24B3948091E5049091E60456
:109FB000A091E704B091E8040097A105B105B1F0C4
:109FC00040919A1150919B1160919C1170919D113B
:109FD000840F951FA61FB71FA7019601281B390BD9
:109FE0004A0B5B0BDA01C901B7FF92C180910802ED
:109FF00090910902A0910A02B0910B02892B8A2B41
:10A000008B2B09F099C10E9405F54B015C018091F1
:10A010006612811108C020919B1290919C1281E0E0
:10A02000291301C080E0209153123091541291E025
:10A0300089272A3A31050CF480E091E04091990497
:10A0400050919A0460919B0470919C04452B462B7F
:10A05000472B09F490E0981789F0882309F4BDC1D3
:10A06000D501C40180569444A24FBF4F80939904F8
:10A0700090939A04A0939B04B0939C044090070D86
:10A080005090080D6090090D70900A0D2091950474
:10A09000309196044091970450919804C301B20105
:10A0A0000F94FE1D882319F18091990490919A04D0
:10A0B000A0919B04B0919C04409295045092960408
:10A0C0006092970470929804892B8A2B8B2B09F449
:10A0D00049C0D501C40180569444A24FBF4F80931C
:10A0E000990490939A04A0939B04B0939C0480914C
:10A0F000990490919A04A0919B04B0919C040097BC
:10A10000A105B10579F1881A990AAA0ABB0AB7FC18
:10A1100029C01092990410929A0410929B041092F4
:10A120009C0483E096E00E94662F60E08FEE95E04D
:10A130000E94AA3580915512909156121816190650
:10A1400024F490E080E00E94071E8091EB11909132
:10A15000EC111816190634F41092EC111092EB1150
:10A160000E9471C48091A1049091A204A091A304C3
:10A17000B091A40446015701881A990AAA0ABB0A99
:10A18000D501C401B7FDB9C120919B1290919C12D9
:10A1900080912C0240912D02291323C19091550BDF
:10A1A000899FC0011124880F892F881F990B9195D1
:10A1B0008D838091560B489FC0011124880F892FF1
:10A1C000881F990B91958E830E9405F569837A8388
:10A1D0008B839C8340E0BE016F5F7F4FCE0105966D
:10A1E0000E94BE1A6D8170E089E00E94FCF341E09C
:10A1F000BE016F5F7F4FCE0105960E94BE1A6E8131
:10A2000070E087E00E94FCF380914509882309F4FF
:10A2100067C10091140210911502C80102972091A4
:10A22000551230915612281739070CF459C18090F5
:10A230009C128F82188619861A861B8680919B1223
:10A240009F80891509F4E7C0892D90E038E6A32E98
:10A25000A89EF001A99EF00D1124E857FA4F4589F8
:10A2600056896789708D452B462B472B81F4418D8C
:10A27000528D638D748D452B462B472B41F4458DB4
:10A28000568D678D70A1452B462B472BE1F128E6B3
:10A29000B22EB89E9001B99E300D1124A9014857E5
:10A2A0005A4F1A01FA0161817281838194810F945E
:10A2B0008A274B015C01F10161A172A183A194A1E4
:10A2C0000F94031E2B013C01F10165A176A187A12A
:10A2D00090A50F94031E9B01AC01C301B2010F9422
:10A2E000D625A50194010F94641E4B015C012885BD
:10A2F00039854A855B850F943C27181624F4888697
:10A300009986AA86BB868F818F5F87708F8396CF51
:10A310000E941E436091E80A7091E90A82EB95E081
:10A320000E94E54A8AE00E942D2F40E070E060E044
:10A3300090E080E00E94F94890919B1280919C12DD
:10A34000981749F0C0929A11D0929B11E0929C11FB
:10A35000F0929D1158CEBB2019F01092A50453CE57
:10A360000E9405F500919A1110919B1120919C116A
:10A3700030919D118090080290900902A0900A02ED
:10A38000B0900B02080D191D2A1D3B1D601B710B9F
:10A39000820B930B97FDE1CF8091A504811133CE01
:10A3A00081E08093A5045F9A8091870C8E7F8093D3
:10A3B000870C8A9A8091870C8D7F8093870C80917F
:10A3C000080180958170809306018091870C8B7FB6
:10A3D0008093870C0E94E81D16CE80E090E0DC019F
:10A3E00045CE20919C1258E6259F900111242857B4
:10A3F0003A4FF901EE59FF4F9081899FC001112416
:10A40000880F892F881F990B91958D832D593F4F68
:10A41000F9018081D0CE20913202309133024091F7
:10A42000340250913502688579858A859B850F9421
:10A43000641E4B015C01B801012E000C880B990BC6
:10A440000F94051E9B01AC01C501B4010F94DC24DF
:10A4500069837A838B839C8340911202509113020B
:10A46000B801CE0101960E94AEC789809A80AB8068
:10A47000BC8040909D0450909E0460909F0470901A
:10A48000A004A3019201C501B4010F94FE1D87FF32
:10A4900016C028E431EE4AE75FE3C301B2010F942E
:10A4A000641E20E037ED43EA5CE30F94DC24A50151
:10A4B00094010F94641E69837A838B839C836981E2
:10A4C0007A818B819C8160939D0470939E0480931C
:10A4D0009F049093A0040F944826CB010E94071E6E
:10A4E000F4E6CF0ED11CE11CF11CC092A104D09265
:10A4F000A204E092A304F092A4040E94F0C7809109
:10A50000480A882309F439C190910901892F80955F
:10A510008170109100021817C9F020918F142062E9
:10A5200020938F148093000290FD40C164EF71E08E
:10A5300080E090E00E94772A0E9407B680918F14F5
:10A5400083FD7DC1111134C10E94FD2C0E9405F5CF
:10A550006B017C01109107021123F1F08091E90455
:10A560008823D1F04091A6045091A7046091A804DB
:10A570007091A90446015701841A950AA60AB70AE0
:10A58000B501A40177FD1AC0833009F430C10CF085
:10A590001FC181300CF024C1212F30E0A8EEB3E0C0
:10A5A0000F949624C60ED71EE81EF91EC092A6046C
:10A5B000D092A704E092A804F092A9048091A3117C
:10A5C000813009F073C00E9405F56B017C01809118
:10A5D000AE049091AF04A091B004B091B104A70172
:10A5E0009601281B390B4A0B5B0BDA01C901B7FD39
:10A5F0003AC0D701C601805F984DAF4FBF4F8093DF
:10A60000AE049093AF04A093B004B093B1048090D3
:10A61000D4089090D508A090D608B090D7080E9492
:10A62000DC25AB01BC014093D4085093D50860935E
:10A63000D6087093D7088091F7099091F809A091F6
:10A64000F909B091FA0988199909AA09BB09840F77
:10A65000951FA61FB71F8093F7099093F809A09341
:10A66000F909B093FA098091AA049091AB04A091E2
:10A67000AC04B091AD0446015701881A990AAA0AA0
:10A68000BB0AD501C401B7FD11C020E8C20E2EEEF1
:10A69000D21E26E3E21EF11CC092AA04D092AB04A3
:10A6A000E092AC04F092AD040E942A480E947530FA
:10A6B0000E943F378091E404882381F10E9405F5D0
:10A6C0006B017C018091E0049091E104A091E2048F
:10A6D000B091E30446015701881A990AAA0ABB0AF5
:10A6E000D501C401B7FD1AC02091E40430E0A8EE02
:10A6F000B3E00F949624C60ED71EE81EF91EC09232
:10A70000E004D092E104E092E204F092E30480914C
:10A71000F90C0E94AFBD8AE00E942D2F8091DF04CA
:10A72000882359F10E9405F56B017C018091DB04BF
:10A730009091DC04A091DD04B091DE04A7019601A4
:10A74000281B390B4A0B5B0BDA01C901B7FD15C099
:10A750002091DF0430E0A8EEB3E00F949624C60EFB
:10A76000D71EE81EF91EC092DB04D092DC04E092F2
:10A77000DD04F092DE040E94A2AD2B960FB6F89491
:10A78000DEBF0FBECDBFDF91CF911F910F91FF9024
:10A79000EF90DF90CF90BF90AF909F908F907F9081
:10A7A0006F905F904F903F902F9008950E94F6B564
:10A7B000123008F0CBCE0E94FD2C60E080E496E0E1
:10A7C00056C08EE496E09093651280936412BECEDC
:10A7D000843009F0E1CE0E94074485E596E004C08C
:10A7E0000E94074484E896E00E94662FD5CE0E941E
:10A7F00007448DE696E0F8CF8091EA0A9091EB0A43
:10A80000A091EC0AB091ED0AA7019601281B390B23
:10A810004A0B5B0BDA01C901885E9340A109B109BB
:10A82000B7FDEDC98DE995E00E94662FC092EA0A56
:10A83000D092EB0AE092EC0AF092ED0AE0C91230F5
:10A84000C8F488E196E00E94662F8AE00E942D2FCE
:10A850000E940A2790E080E00E94EF4A1092F70CD5
:10A860001092F60C1092F50C60E081E396E00E94E5
:10A87000AA356CCE123009F069CE0E9461BA8823E5
:10A8800079F081E00E9437BA47EB50E068E77BE05F
:10A8900084E994E10E942FB484E994E10E94DCB53C
:10A8A0000E94E02881118DCF0E94CA280E94DDBA43
:10A8B0000E9432BA4BCE2F923F924F925F926F928C
:10A8C0007F928F929F92AF92BF92CF92DF92EF9240
:10A8D000FF920F931F93CF93DF93CDB7DEB7C5578A
:10A8E000D1090FB6F894DEBF0FBECDBF3B014A01C0
:10A8F00059013E2C6D96DFAECEAE6D97DC012D91E9
:10A900003D914D915C91A1962CAF3DAF4EAF5FAFA5
:10A91000A19720919C0C30919D0C40919E0C5091E0
:10A920009F0CA1966CAD7DAD8EAD9FADA1970F94A0
:10A93000641E0F944927AD966CAF7DAF8EAF9FAF6D
:10A94000AD97D3012D913D914D915C91A5962CAF82
:10A950003DAF4EAF5FAFA5972091A00C3091A10CF9
:10A960004091A20C5091A30CA5966CAD7DAD8EAD1F
:10A970009FADA5970F94641E0F944927E1966CAF85
:10A980007DAF8EAF9FAFE197D4012D913D914D9159
:10A990005C91A9962CAF3DAF4EAF5FAFA9972091C8
:10A9A000A40C3091A50C4091A60C5091A70CA9962F
:10A9B0006CAD7DAD8EAD9FADA9970F94641E0F94C5
:10A9C0004927E5966CAF7DAF8EAF9FAFE597D50178
:10A9D0002D913D914D915C9167962CAF3DAF4EAF5F
:10A9E0005FAF67972091A80C3091A90C4091AA0CF9
:10A9F0005091AB0C67966CAD7DAD8EAD9FAD6797FA
:10AA00000F94641E0F9449276B966CAF7DAF8EAF89
:10AA10009FAF6B978091530B83FF1CC06B962CAD3F
:10AA20003DAD4EAD5FAD6B972093CD123093CE12FE
:10AA30004093CF125093D01267968CAD9DADAEADC2
:10AA4000BFAD67978093BD129093BE12A093BF12C3
:10AA5000B093C012D8012C901196BC91BDAFF801F3
:10AA6000F2812296FFAF2297D8011396BC912896C7
:10AA7000BFAF289780919B1290919C12891B809563
:10AA8000877019F40E94D04DF5CFE0919B12E696A5
:10AA9000EFAFE697F0919B12FBAF8091E50A9091A2
:10AAA000E60A892B11F00C941C5E8091C1129091E2
:10AAB000C212A091C312B091C412AD964CAC5DAC61
:10AAC0006EAC7FACAD97481A590A6A0A7B0A80912E
:10AAD000C5129091C612A091C712B091C812E1960A
:10AAE0008CAC9DACAEACBFACE197881A990AAA0AAF
:10AAF000BB0A8091C9129091CA12A091CB12B09159
:10AB0000CC12E5962CAD3DAD4EAD5FADE597281B63
:10AB1000390B4A0B5B0B2FAB38AF49AF5AAF809163
:10AB2000CD129091CE12A091CF12B091D0126B960F
:10AB30002CAD3DAD4EAD5FAD6B97281B390B4A0B6D
:10AB40005B0B2FA338A749A75AA7232B242B252B10
:10AB500009F490C08091520B811132C080913A0269
:10AB600090913B0201972091531230915412281773
:10AB7000390734F56B968CAD9DADAEADBFAD6B971F
:10AB80008093CD129093CE12A093CF12B093D01297
:10AB900067962CAD3DAD4EAD5FAD67972093BD126E
:10ABA0003093BE124093BF125093C0120E940744CC
:10ABB00087EC98E10E94662F1FA218A619A61AA674
:10ABC00034E0339E800111240A5E1D4F6FA178A5E9
:10ABD00089A59AA50F94051ED8012D913D914D91FF
:10ABE0005C910F94641E6B017C0120E030E0A901B0
:10ABF0000F943C2787FF04C0F7FAF094F7F8F0941D
:10AC000020E030E84BE354E46091A80C7091A90C6B
:10AC10008091AA0C9091AB0C0F94641EA701960131
:10AC20000F94FE1D87FF26C06B962CAD3DAD4EAD3B
:10AC30005FAD6B972093CD123093CE124093CF121D
:10AC40005093D01267968CAD9DADAEADBFAD6797FA
:10AC50008093BD129093BE12A093BF12B093C01206
:10AC60000E94074488EA98E10E94662F1FA218A656
:10AC700019A61AA6D301C2018827B7FD8395992783
:10AC8000AA27BB278BA7B7FE03C0E82FE260EBA77C
:10AC90002FA938AD49AD5AAD57FF03C03BA534606D
:10ACA0003BA78FA198A5A9A5BAA5B7FF03C09BA5EF
:10ACB00098609BA7A4E03A9E800111240A5E1D4F74
:10ACC0006FA178A589A59AA50F94051EF80120818A
:10ACD0003181428153810F94641E6B017C0120E01D
:10ACE00030E0A9010F943C2787FFC7C1C701B60117
:10ACF00090583BAD232F30E03CA32BA35BAD48E63F
:10AD0000549F90011124D901A857BA4FBCAFABAFE3
:10AD100020E030E040E05FE30F94DC240F944F2606
:10AD20006FA778AB89AB9AABEBADFCAD1082EA5B59
:10AD3000FF4F2BA520838FA998ADA9ADBAAD2F9653
:10AD40008CAF9DAFAEAFBFAF2F97B7FF0DC0B09523
:10AD5000A095909581959F4FAF4FBF4F2F968CAF89
:10AD60009DAFAEAFBFAF2F978BA69CA6ADA6BEA6DC
:10AD7000B7FE0BC022273327A901281939094A0930
:10AD80005B092BA73CA74DA75EA74BAA5CAA6DAA9F
:10AD90007EAA77FE0BC088279927DC0184199509C4
:10ADA000A609B7098BAB9CABADABBEAB2BA93CA93D
:10ADB0004DA95EA9ABADBCAD55962D933D934D937A
:10ADC0005C9358972BA53CA54DA55EA559962D9350
:10ADD0003D934D935C935C972F962CAD3DAD4EAD5E
:10ADE0005FAD2F975D962D933D934D935C93909718
:10ADF000C301B2010F94051E2091D00C3091D10CEB
:10AE00004091D20C5091D30C0F94641E27966CAFD6
:10AE10007DAF8EAF9FAF2797698B7A8B8B8B9C8B87
:10AE2000C501B4010F94051E2091D40C3091D50CAE
:10AE30004091D60C5091D70C0F94641E63966CAF62
:10AE40007DAF8EAF9FAF63976D8B7E8B8F8B988F0F
:10AE50006FA978AD89AD9AAD0F94051E2091D80CDD
:10AE60003091D90C4091DA0C5091DB0C0F94641E98
:10AE70004B015C01898E9A8EAB8EBC8E2091DC0CCE
:10AE80003091DD0C4091DE0C5091DF0CC701B60112
:10AE90000F94641E6B017C01CD8EDE8EEF8EF8A2C6
:10AEA0002BA93CA94DA95EA92630310541055105C4
:10AEB0000CF0E6C08BA59CA5ADA5BEA50697A10587
:10AEC000B1050CF0DDC02F962CAD3DAD4EAD5FADA4
:10AED0002F9726303105410551050CF0D1C020E0F7
:10AEE00030E0A901C701B6010F943C2787FF04C0D9
:10AEF000F7FAF094F7F8F09488E64BA15CA1849FF0
:10AF00008001859F100D112408571A4F20E030E072
:10AF1000A901C701B6010F94DC24D8011D966D93D9
:10AF20007D938D939C93509788E6ABA1BCA18A9F9B
:10AF3000F0018B9FF00D1124E857FA4F2FA538A987
:10AF400049A95AA921A332A343A354A32F968CAD98
:10AF50009DADAEADBFAD2F972BA53CA54DA55EA574
:10AF600082179307A407B50710F4DA01C9012BA9CA
:10AF70003CA94DA95EA982179307A407B50710F451
:10AF8000DA01C9012FA538A949A95AA9821793073F
:10AF9000A407B50710F4DA01C90128E64BA15CA1AA
:10AFA000249FF001259FF00D1124E857FA4F85A347
:10AFB00096A3A7A3B0A70697A105B10508F41FC6DD
:10AFC000DF01AE59BF4F8091550B8C931196809144
:10AFD000560B8C9331A645284628472809F05F98E0
:10AFE00088E6ABA1BCA18A9FF0018B9FF00D1124D4
:10AFF000E857FA4F818D928DA38DB48D892B8A2BC2
:10B000008B2B09F08A9888E62BA13CA1829FF00146
:10B01000839FF00D1124E857FA4F858D968DA78DEB
:10B02000B0A1892B8A2B8B2B29F08091080181708C
:10B03000809306018FA598A9A9A9BAA9892B8A2B63
:10B040008B2B09F4FBC580918605882319F081506C
:10B050008093860580918705882319F0815080931D
:10B060008705311068C0129880E180938605809131
:10B07000870581116CC0479A6AC0C701B60139CEF5
:10B080006D96EEADFFAD6D97C080D180E280F3800C
:10B0900020E030E0A901C701B6010F94FE1D88230E
:10B0A00079F088E62BA13CA1829FF001839FF00DEF
:10B0B0001124E857FA4FC586D686E786F08A34CF42
:10B0C00027962CAD3DAD4EAD5FAD2797CA01B901B6
:10B0D0000F94641E6B017C0163962CAD3DAD4EADAB
:10B0E0005FAD6397CA01B9010F94641E9B01AC0167
:10B0F000C701B6010F94DC246B017C01A50194010A
:10B10000C501B4010F94641E9B01AC01C701B601D7
:10B110000F94DC240F948A2728E64BA15CA1249F7E
:10B12000F001259FF00D1124E857FA4F65877687C7
:10B130008787908BF9CE80918605811101C0129A84
:10B1400091E0391294CF479880E180938705E09091
:10B15000C80CF090C90C0091CA0C1091CB0C76C5AC
:10B160002FA538A949A95AA9232B242B252B09F44B
:10B1700006C12091BC0C3091BD0C4091BE0C509189
:10B18000BF0C21966CAD7DAD8EAD9FAD21970F9418
:10B19000641E0F94BA250F944F262B013C018FA5F6
:10B1A00098A9A9A9BAA9892B8A2B8B2B09F4F0C0DD
:10B1B000E091F90C94E0E99FF0011124E059F64F79
:10B1C00020813181428153812FA738AB49AB5AABE3
:10B1D00020E030E0A9016FA578A989A99AA90F9468
:10B1E000FE1D882309F4D4C08FA198A5A9A5BAA5EE
:10B1F000181619061A061B060CF0CAC088E6ABA181
:10B20000BCA18A9F80018B9F100D112408571A4FF3
:10B210001801B7E42B0E311C81E0F10180832091ED
:10B22000B1123091B2124091B3125091B412A19662
:10B230006CAD7DAD8EAD9FADA1970F94DB246FA358
:10B2400078A789A79AA72091B5123091B61240919C
:10B25000B7125091B812A5966CAD7DAD8EAD9FAD75
:10B26000A5970F94DB244B015C012091B91230911A
:10B27000BA124091BB125091BC12A9966CAD7DAD33
:10B280008EAD9FADA9970F94DB246B017C012FA19C
:10B2900038A549A55AA5CA01B9010F94641E6FA328
:10B2A00078A789A79AA7A5019401C501B4010F94B5
:10B2B000641E9B01AC016FA178A589A59AA50F9486
:10B2C000DC244B015C01A7019601C701B6010F9474
:10B2D000641E9B01AC01C501B4010F94DC240F94E2
:10B2E0008A276B017C012091BD123091BE124091E2
:10B2F000BF125091C01267966CAD7DAD8EAD9FAD03
:10B3000067970F94DB24A70196010F94D6256B0154
:10B310007C01F801E25BFF4FC082D182E282F382BE
:10B3200020E030E040E450E40F943C2718160CF481
:10B33000FDC0A70196016FA578A989A99AA90F94C4
:10B34000641E9B01AC0160910B0970910C09809106
:10B350000D0990910E090F94D62521962CAD3DAD87
:10B360004EAD5FAD21970F94641E0F944F26641568
:10B37000750586059705B8F42B013C0114C0209192
:10B38000C40C3091C50C4091C60C5091C70CF9CE3D
:10B3900088E62BA13CA1829FF001839FF00D112430
:10B3A000E153FA4F10828091820590918305A0911C
:10B3B0008405B0918505EBADFCADC18CD28CE38CDE
:10B3C000F48C258D368D478D50A12FA338A749A722
:10B3D0005AA721A132A143A154A12FA738AB49AB51
:10B3E0005AAB2BA53CA54DA55EA582179307A407D4
:10B3F000B50708F49EC08BA99CA9ADA9BEA9892B4D
:10B400008A2B8B2BE1F0609172057091730580910E
:10B41000740590917505641575058605970578F492
:10B420000F9432242BA93CA94DA95EA90F94422464
:10B43000241535054605570510F429013A01C114B4
:10B44000D104E104F104F1F0609176057091770583
:10B4500080917805909179056415750586059705A5
:10B4600088F42BA53CA54DA55EA50F943224A70119
:10B4700096010F944224241535054605570510F40E
:10B4800029013A012FA138A549A55AA5232B242B20
:10B49000252B01F160917A0570917B0580917C05E7
:10B4A00090917D05641575058605970598F42BA583
:10B4B0003CA54DA55EA50F9432242FA138A549A522
:10B4C0005AA50F944224241535054605570510F456
:10B4D00029013A018FA598A9A9A9BAA9892B8A2B74
:10B4E0008B2B09F400C660917E0570917F058091D9
:10B4F000800590918105641575058605970508F00E
:10B50000F2C52BA53CA54DA55EA50F9432242FA511
:10B5100038A949A95AA90F9442242415350546058E
:10B52000570508F0E0C529013A01DDC5D1011C929B
:10B530003ACF2BA93CA94DA95EA9232B242B252B5F
:10B54000B9F16091720570917305809174059091C5
:10B550007505641575058605970550F50F94031E4E
:10B560002FA938AD49AD5AAD0F94641E4B015C0153
:10B570006BA97CA98DA99EA90F94031E9B01AC0108
:10B58000C501B4010F94D6254B015C01C301B20182
:10B590000F94031E9B01AC01C501B4010F94FE1D65
:10B5A00087FF06C0C501B4010F944F262B013C0153
:10B5B000C114D104E104F104A9F160917605709100
:10B5C0007705809178059091790564157505860554
:10B5D000970540F50F94031E2FA938AD49AD5AAD1C
:10B5E0000F94641E4B015C01C701B6010F94031E4A
:10B5F0009B01AC01C501B4010F94D6256B017C0100
:10B60000C301B2010F94031E9B01AC01C701B60137
:10B610000F94FE1D87FF06C0C701B6010F944F2689
:10B620002B013C018FA198A5A9A5BAA5892B8A2B2E
:10B630008B2BB9F160917A0570917B0580917C0527
:10B6400090917D05641575058605970550F50F9455
:10B65000031E2FA938AD49AD5AAD0F94641E6B017E
:10B660007C016FA178A589A59AA50F94031E9B0163
:10B67000AC01C701B6010F94D6256B017C01C30153
:10B68000B2010F94031E9B01AC01C701B6010F94D8
:10B69000FE1D87FF06C0C701B6010F944F262B0180
:10B6A0003C012FA538A949A95AA9232B242B252BC6
:10B6B00009F419C560917E0570917F058091800520
:10B6C00090918105641575058605970508F00BC5F1
:10B6D0000F94031E2FA938AD49AD5AAD0F94641EC7
:10B6E0006B017C016FA578A989A99AA90F94031E03
:10B6F0009B01AC01C701B6010F94D6256B017C01FB
:10B70000C301B2010F94031E9B01AC01C701B60136
:10B710000F94FE1D87FFE7C4C701B6010F944F26A3
:10B720002B013C01E0C4A5019401C301B2010F94B7
:10B73000D6259B01AC016FA17BA58FA59FA90F9476
:10B74000641E6FA37BA78FA79FAB21E02BABB8C56F
:10B7500080E090E0A0E8BFE327968CAF9DAFAEAF4E
:10B76000BFAF2797E5C5F7FAF094F7F8F094A70173
:10B770009601C501B4010F943C2718160CF03AC687
:10B780007501640137C6C701B6010F94FE1D87FD20
:10B7900009C020E030E0A901C501B4010F943C27A5
:10B7A00018162CF4A5019401C701B6011FC6B7FAFB
:10B7B000B094B7F8B094A5019401C701B6010F94F5
:10B7C000FE1D87FF17C6DCCF2FA03BA40FA51FA926
:10B7D00070C681E0C6C6CBA0DCA091C78BE0C82EA6
:10B7E00087EDD82E83E2E82E8BE3F82EC8C78B2D89
:10B7F000902FAA2DB32DF60185839683A783B0875A
:10B800000C941664DCA2CBA20C94166410919A12CC
:10B81000D12CC12C08E680919B12811709F48BC0B2
:10B82000812E912C089DC001099D900D11249C0131
:10B8300028573A4F1901D9018C91560183FD6FC0E9
:10B840005901C114D10409F46AC0C6010E9484CC14
:10B85000811165C0F601808181FD4CC0D101159632
:10B860004D905D906D907C901897D60115962D9116
:10B870003D914D915C9118972BA33CA34DA35EA3E2
:10B88000A30192016BA17CA18DA19EA10F94FE1D2D
:10B8900087FF30C0F6016189728983899489905845
:10B8A0009B01AC010F94DC24D6011D962D913D9196
:10B8B0004D915C9150970F94641E9B01AC016BA15C
:10B8C0007CA18DA19EA10F94DB246B017C01A301BF
:10B8D00092010F94FE1D87FF0DC0F10180818160F0
:10B8E0008083C5010E9484CC8823E9F0D1018C912A
:10B8F0008E7F8C93089DF001099DF00D1124E8576F
:10B90000FA4F21853285438554856581768187810B
:10B9100090850F94FE1D811102C010939A121F5F33
:10B920001770650178CFF101C582D682E782F08673
:10B9300010939A12DFCFD0909C1280909B1228E631
:10B94000D81409F4C7C08FEF880D8770289FF001C5
:10B950001124E857FA4F908193FDBAC0312C212C65
:10B960001BA21BAE10E000E0F12CE12CD81409F46E
:10B97000C0C0F8E6DF9E8001112408571A4FD80195
:10B980008C9183FDA9C015966D917D918D919C91AF
:10B9900018970F948A27B62EC72EA82E992EE11439
:10B9A000F10409F493C0F701808180FD04C0D8013F
:10B9B0008C9180FF8BC0F701808181608083C701FB
:10B9C0000E9484CC81117EC0D70111966D917D912A
:10B9D0008D919C9114970F948A276FA378A789A7BC
:10B9E0009AA79B01AC0160E070E080E89FE30F94B0
:10B9F000D6252B013C01AC019B016B2D7C2D8A2DA2
:10BA0000992D0F94641E69837A838B839C83232DE5
:10BA1000322D4BA15BADC301B2010F94641E698B43
:10BA20007A8B8B8B9C8BAE014F5F5F4FBE016F5E3D
:10BA30007F4FC7010E941C1EF701E95BFF4F808109
:10BA4000882309F43FC0E091F90CB4E0EB9FF001CA
:10BA50001124E059F64FD701A25BBF4F2D913D91C4
:10BA60004D915C9160817181828193810F94641EFC
:10BA70002091A80C3091A90C4091AA0C5091AB0CCC
:10BA80000F94641E2B013C01AC019B016FA178A5B2
:10BA900089A59AA50F94641E0F944F26F701E65BC3
:10BAA000FF4F71836083A30192016B2D7C2D8A2D42
:10BAB000992D0F94641E0F944F26F701E45BFF4FFE
:10BAC00071836083F70180818E7F8083780108C055
:10BAD000882E36CF8D2C42CFB32CC22CABA09BAC82
:10BAE000D394FD2DF770DF2E3B2C2C2CABA29BAEFC
:10BAF0003DCF0115110509F482C0D8018C918160F8
:10BB00008C93C7010E9484CC811175C0F8016181BA
:10BB10007281838194810F948A276B017C01AC012F
:10BB20009B0160E070E080E89FE30F94D6254B0115
:10BB30005C012DEC3CEC4CE45DE30F94641E6983E6
:10BB40007A838B839C83A5019401632D722D8BA135
:10BB50009BAD0F94641E698B7A8B8B8B9C8BAE0193
:10BB60004F5F5F4FBE016F5E7F4FC8010E941C1E7A
:10BB7000F801E95BFF4F80818823E9F1E091F90C3E
:10BB800024E0E29FF0011124E059F64FD801A25BB6
:10BB9000BF4F2D913D914D915C916081718182816A
:10BBA00093810F94641E2091A80C3091A90C4091B0
:10BBB000AA0C5091AB0C0F94641E4B015C01AC01BC
:10BBC0009B01C701B6010F94641E0F944F26F80124
:10BBD000E65BFF4F718360832DEC3CEC4CE45DE34E
:10BBE000C501B4010F94641E0F944F26F801E45B65
:10BBF000FF4F71836083D8018C918E7F8C930E945C
:10BC0000402981E0CB58DF4F0FB6F894DEBF0FBE5E
:10BC1000CDBFDF91CF911F910F91FF90EF90DF90FB
:10BC2000CF90BF90AF909F908F907F906F905F90DC
:10BC30004F903F902F90089580E0E4CFE090CC0C9F
:10BC4000F090CD0C0091CE0C1091CF0C9701A80173
:10BC5000622D7DAD22968FAD229728969FAD2897B5
:10BC60000F94FE1D87FD08C0E22CFDAC22960FAD9F
:10BC7000229728961FAD289788E6ABA1BCA18A9F82
:10BC8000F0018B9FF00D1124E857FA4F85849684BC
:10BC9000A784B088A501940160E070E080E89FE38C
:10BCA0000F94D62521966CAF7DAF8EAF9FAF2197B5
:10BCB0009701A8010F94641E6B017C0180919B1277
:10BCC00090919912891B877022968FAF2297A701B6
:10BCD000960160E074E284E799E40F94D6250F940E
:10BCE00049272B013C0122968FAD2297825082304A
:10BCF000A0F56091980C7091990C80919A0C90919C
:10BD00009B0C6419750986099709161617061806FB
:10BD100019061CF5660F771F881F991F2296BFAD65
:10BD200022972B2F30E050E040E00F946424CA01AA
:10BD3000B9010F94051E0F944826640D751D861DCC
:10BD4000971D0F94051E9B01AC0160E074E284E72F
:10BD500099E40F94D6256B017C01A7019601C501DA
:10BD6000B4010F94641E9B01AC010F94641E2B96CA
:10BD70006CAF7DAF8EAF9FAF2B9788E6EBA1FCA198
:10BD80008E9F80018F9F100D112408571A4F2B96FC
:10BD90002CAD3DAD4EAD5FAD2B97D80111962D93D7
:10BDA0003D934D935C93149795962D913D914D91B4
:10BDB0005C9198972BA73CA74DA75EA7CA01B90134
:10BDC0000F94031E6FAB78AF89AF9AAF9B01AC01A4
:10BDD000C701B6010F94641E0F94BA250F944F2625
:10BDE00027966CAF7DAF8EAF9FAF2797F801EE5AC5
:10BDF000FF4F6083718382839383FE017196FCAB56
:10BE0000EBAB9E012F5F3F4F2D963FAF2EAF2D978F
:10BE10004CEA5CE061965FAF4EAF6197CE014D9604
:10BE20009AA389A36D963FAF2EAF6D9700E010E007
:10BE300020E8222E3FE3332EABA9BCA92D913D91E2
:10BE40004D915D91BCABABABC701B6010F94641EC5
:10BE50004B015C016D96EEADFFAD6D9781929192B5
:10BE6000A192B1926D96FFAFEEAF6D9720E030E0FA
:10BE7000A9010F943C2787FF04C0B7FAB094B7F824
:10BE8000B0946196AEADBFAD61974D905D906D90F1
:10BE90007D906196BFAFAEAF6197A5019401C301DC
:10BEA000B2010F94FE1D87FF10C0A5019401C301CC
:10BEB000B2010F94D6255B014C019801A1010F94AA
:10BEC000FE1D87FF02C085011401E9A1FAA12BA97B
:10BED0003CA9E217F30709F0AFCF2D8D3E8D4F8DB2
:10BEE00058A1C701B6010F94641E6B017C01CD8679
:10BEF000DE86EF86F88A20E030E0A9010F943C2727
:10BF00004601570187FF04C0B7FAB094B7F8B09460
:10BF10004090B80C5090B90C6090BA0C7090BB0C6B
:10BF2000A5019401C301B2010F94FE1D87FF10C04B
:10BF3000A5019401C301B2010F94D6255B014C0108
:10BF40009801A1010F94FE1D87FF02C08501140115
:10BF500020E030E040E85FE3B801C1010F94FE1D2E
:10BF600087FF66C09801A10169817A818B819C81DC
:10BF70000F94641E69837A838B839C839801A1014B
:10BF80006D817E818F8198850F94641E6D837E8381
:10BF90008F8398879801A10169857A858B859C8517
:10BFA0000F94641E69877A878B879C879801A1010B
:10BFB000C701B6010F94641E6D877E878F87988BAB
:10BFC00028E64BA15CA1249FC001259F900D112460
:10BFD000DC01A857BA4F7D016D01B2E5CB0ED11C33
:10BFE00027966CAD7DAD8EAD9FAD27970F94031E48
:10BFF0009801A1010F94641E0F944F26F6016083EF
:10C000007183828393839801A101B801C1010F94C8
:10C01000641E2B962CAD3DAD4EAD5FAD2B970F94AE
:10C02000641ED70111966D937D938D939C93149705
:10C030002FA938AD49AD5AAD21966CAD7DAD8EAD11
:10C040009FAD21970F94641E21966CAF7DAF8EAF8C
:10C050009FAF219788E6EBA1FCA18E9F80018F9F67
:10C06000100D112408571A4FD80155962D913D9166
:10C070004D915C9158972BAB3CAB4DAB5EAB232BFA
:10C08000242B252B09F06CC859968D919D910D900C
:10C09000BC91A02D892B8A2B8B2B09F061C8F8014C
:10C0A000858D968DA78DB0A1892B8A2B8B2B09F0BE
:10C0B00057C82091C00C3091C10C4091C20C5091D6
:10C0C000C30C21966CAD7DAD8EAD9FAD21970F94C5
:10C0D000641E0F94BA250F944F262B013C01F801E2
:10C0E000E95BFF4F108288E64BA15CA1849F800131
:10C0F000859F100D112408571A4FF801E25AFF4F7F
:10C100004082518262827382C301B2010F94031E86
:10C1100021962CAD3DAD4EAD5FAD21970F94D62548
:10C1200021966CAF7DAF8EAF9FAF2197D80151960E
:10C130006D937D938D939C935497F801E95BFF4F2A
:10C1400080818823C1F17801B8E4EB0EF11CA09145
:10C15000F90CE4E0AE9FD0011124A059B64FF801CC
:10C16000E25BFF4F20813181428153816D917D914E
:10C170008D919C910F94641E21962CAD3DAD4EADDA
:10C180005FAD21970F94641E2091A80C3091A90CEB
:10C190004091AA0C5091AB0C0F94641E9B01AC0112
:10C1A00060E074E284EF99E40F94D6250F944F2653
:10C1B000D7016D937C9388E62BA13CA1829FF0016F
:10C1C000839FF00D1124E857FA4F81819281A3815A
:10C1D000B4812B968CAF9DAFAEAFBFAF2B97BC0198
:10C1E000CD010F948A276B017C01AFEFB8E0619617
:10C1F000BFAFAEAF61972D960EAD1FAD2D97005F0F
:10C200001F4F2596BFAFAEAF25972D962EAC3FACF6
:10C210002D976FA3DBA68FA7FFAA1BAAD1018D9034
:10C220009D90AD90BD901D0120E030E0A901C501B9
:10C23000B4010F943C2787FF04C0B7FAB094B7F855
:10C24000B0942596EEADFFAD2597619171918191E6
:10C2500091912596FFAFEEAF259720E030E0A90140
:10C260000F94DC242B013C01A50194010F94FE1DC9
:10C2700087FF26C0FBA9FF2309F455CAA301920139
:10C28000B601C7010F94641E2B013C012FA13BA5F1
:10C290004FA55FA9C501B4010F94641E9B01AC01B9
:10C2A000C301B2010F94FE1D87FF0AC0A5019401CE
:10C2B000C301B2010F94D6256FA37BA78FA79FABB5
:10C2C0000215130509F0AACF22963FAD229733231A
:10C2D00009F47ACA80909D1290909E12A0909F12AD
:10C2E000B090A0122DEB37E346E855E3C501B40149
:10C2F0000F94FE1D87FD68CAC501B4010F948A27FB
:10C300001B018C019B01AC01B601C7010F94FE1DFE
:10C3100087FF1ECA9101A801B601C7010F94D62557
:10C3200027966CAF7DAF8EAF9FAF27971601870121
:10C33000A1EAB2E12396BFAFAEAF2397412C512CB7
:10C3400090E8692E9FE3792E1BAA2396EEADFFADF0
:10C35000239761917191819191912396FFAFEEAFF7
:10C36000239727962CAD3DAD4EAD5FAD27970F942B
:10C37000641E4B015C012D96AEADBFAD2D97CD90E7
:10C38000DD90ED90FD902D96BFAFAEAF2D97BBA980
:10C39000BB2371F0A30192010F94641E4B015C0159
:10C3A000A3019201C701B6010F94641E6B017C01C9
:10C3B000A5019401C701B6010F94FE1D20E030E0F5
:10C3C000A90187FFE0C9C701B6010F943C271816E1
:10C3D0004CF020E030E0A901C501B4010F94FE1D2E
:10C3E00087FFC1C9A7019601C501B4010F94DB24E1
:10C3F0006B017C016196EEADFFAD6197619171912A
:10C40000819191916196FFAFEEAF619720E030E0AE
:10C41000A9010F94DC244B015C01A70196010F9444
:10C42000FE1D87FF11C0A7019601C501B4010F943D
:10C43000D6259B01AC01C301B2010F94641E2B01F0
:10C440003C01FBA9FF5FFBAB21EB32E123964EAD34
:10C450005FAD23972417350709F077CF5BA95523E4
:10C4600041F0A3019201B101C8010F94641E1B01A8
:10C470008C0124EA30E74DE75FE3B101C8010F9476
:10C48000641E6B017C0120916E0530916F05409117
:10C490007005509171050F94FE1D87FF0AC02FA1F2
:10C4A0003BA54FA55FA9C701B6010F94FE1D87FDEF
:10C4B0008BC98FA19BA5AFA5BFA980936E05909353
:10C4C0006F05A0937005B093710528E6ABA1BCA1E0
:10C4D0002A9FC0012B9F900D1124FC01E857FA4FB1
:10C4E0007F019101A801B101C8010F94641ED70119
:10C4F00019966D937D938D939C931C9721966CADAB
:10C500007DAD8EAD9FAD219790589B01AC010F94EE
:10C51000DC24EBADFCAD25853685478550890F942D
:10C52000641E9B01AC016BE077ED83E29BE30F940B
:10C53000DB249B01AC018BE097EDA3E2BBE3F701A9
:10C5400085839683A783B08710812B966CAD7DADD4
:10C550008EAD9FAD2B970F94FE1D18160CF439C9A4
:10C5600083E0182B28E64BA15CA1249FC001259FE6
:10C57000900D112488579A4FDC011C9320E1FE0195
:10C580003196A1EAB2E101900D922A95E1F72B963E
:10C590002CAD3DAD4EAD5FAD2B9720939D123093EA
:10C5A0009E1240939F125093A012AD962CAD3DADBC
:10C5B0004EAD5FADAD972093C1123093C212409340
:10C5C000C3125093C412E1962CAD3DAD4EAD5FAD9C
:10C5D000E1972093C5123093C6124093C71250932F
:10C5E000C812E5962CAD3DAD4EAD5FADE5972093FD
:10C5F000C9123093CA124093CB125093CC126B964F
:10C600002CAD3DAD4EAD5FAD6B972093CD12309309
:10C61000CE124093CF125093D012A1962CAD3DADC7
:10C620004EAD5FADA1972093B1123093B2124093FB
:10C63000B3125093B412A5962CAD3DAD4EAD5FAD87
:10C64000A5972093B5123093B6124093B71250932A
:10C65000B812A9962CAD3DAD4EAD5FADA997209314
:10C66000B9123093BA124093BB125093BC12679622
:10C670002CAD3DAD4EAD5FAD67972093BD123093AD
:10C68000BE124093BF125093C0128C599F4FE0913D
:10C690006D0534E0E39FF0011124EC50F24F40812E
:10C6A000518162817381DC014D935D936D937C9325
:10C6B000139790919B1280919C12981303C084E66B
:10C6C00080939812E6968FADE6978F5F8770809380
:10C6D0009B1280919B1290919A12815087708917BA
:10C6E00009F429C910919B1220909A1280919B12F3
:10C6F000281609F48BC811501770D12CC12C1215B3
:10C7000009F484C8812E912CB8E6B89DF001B99D3A
:10C71000F00D1124E857FA4F808183FD73C8FCA304
:10C72000EBA3B1840285A38434844580568067805E
:10C730007084A30192016B2D702F8A2D932D0F947D
:10C74000FE1D811108C0C114D10409F46FC0D601C7
:10C750008C9180FF6BC0B8E6B89DF001B99DF00DDB
:10C760001124E857FA4F808181FD3DC0C114D104E6
:10C7700009F434C8F601C580D680E780F08428E645
:10C78000289DF001299DF00D1124E857FA4F618989
:10C7900072898389948990589B01AC010F94DC24A1
:10C7A000ABA1BCA11D962D913D914D915C915097EF
:10C7B0000F94641E9B01AC01C701B6010F94DB24EA
:10C7C000D62EC72E8BAF9FA3262F372FAC016B2DF4
:10C7D000702F8A2D932D0F94FE1D87FD04C0BD2C54
:10C7E0000C2DABAC3FA02B2D302F4A2D532DC30168
:10C7F000B2010F94FE1D8823C9F0B8E6B89DC001B0
:10C80000B99D900D1124FC01E857FA4F6F0180810A
:10C81000816080838BA19CA10E9484CC882311F429
:10C820000C94F75BD6018C918E7F8C93115017700E
:10C83000822D20909A12281611F40C94EB5B181795
:10C8400011F40C94065C8F5F8770F3CFAF92BF92A8
:10C85000CF92DF92EF920F931F93CF93DF93CDB7D9
:10C86000DEB764970FB6F894DEBF0FBECDBFA98ABE
:10C87000BA8ACB8ADC8AFC0180819181A281B38152
:10C8800089839A83AB83BC83FB0180819181A281E0
:10C89000B3818D839E83AF83B887FA0180819181B4
:10C8A000A281B38189879A87AB87BC87F901808190
:10C8B0009181A281B3818D879E87AF87B88BCE018E
:10C8C00001960E9417248091E50A9091E60A892B2F
:10C8D000F9F4CE0141966C019E01235F3F4FAE01FA
:10C8E000475F5F4FBE016B5F7F4F40970E945B5475
:10C8F00064960FB6F894DEBF0FBECDBFDF91CF9127
:10C900001F910F91EF90DF90CF90BF90AF9008955F
:10C9100080E0EECFAF92BF92CF92DF92EF920F9373
:10C920001F93A12CB12C6501E090F90C8C0127E03C
:10C930003DE043E05DE06FEF7CE08BEF9CE00E9428
:10C9400026641F910F91EF90DF90CF90BF90AF9032
:10C9500008952F923F924F925F926F927F928F92A3
:10C960009F92AF92BF92CF92DF92EF92FF920F937E
:10C970001F93CF93DF93CDB7DEB761970FB6F894CF
:10C98000DEBF0FBECDBF898BE82EF12CF701E85535
:10C99000F44D6491062E000C770B880B990B0F94C5
:10C9A000051E4B015C011701220C331C220C331CA9
:10C9B000F101E052FA4E2591359145915491C5010E
:10C9C000B4010F94641E2B013C01F101EC52FA4EAC
:10C9D000659175918591949120E030E040EC5FE3A2
:10C9E0000F94641EA50194010F94641EAB01BC0159
:10C9F00000E010E0980189890E9411F220E030E007
:10CA0000A901C301B2010F94FE1D882309F441C09E
:10CA1000B301A201705800E010E0980189890E94DA
:10CA200011F2A3019201C301B2010F94DC242B0186
:10CA30003C01F701EF52FA4E1491111107C00E9408
:10CA400007448FEA95E10E94662F1AE089898230B7
:10CA500008F0CFC060E070E88BE395E420E030E0C0
:10CA600040E752E40F94D6256B017C01612F70E002
:10CA700090E080E00F94031E9B01AC01C701B6015A
:10CA80000F94D6258B019C01B301A20189890E94D4
:10CA900011F281E090E0A0E0B0E0098804C0880FC6
:10CAA000991FAA1FBB1F0A94D2F72091870C282B2D
:10CAB0002093870C20916F09822B80936F09F101DD
:10CAC000ED55FA4E85919591A591B491810105504E
:10CAD000134FF80180839183A283B38310929F1137
:10CAE00010929E11F101E05AF44F108211821282CD
:10CAF000138289890E94E21C0E947A25F801C08075
:10CB0000D180E280F380F101EB52F54FC082D182F7
:10CB1000E282F3828CE0EAEAF2E0DE011196019013
:10CB20000D928A95E1F7E1E0F0E0EC0FFD1FE20DD8
:10CB3000F31D408051806280738020E030E0A901C5
:10CB4000C301B2010F94FE1D8823D1F120E030E033
:10CB5000A901C301B2010F943C2787FF04C077FAF3
:10CB6000709477F8709481010550134FA3019201DE
:10CB7000C501B4010F94641E9B01AC01C701B6014D
:10CB80000F94DB24F8016083718382839383F98996
:10CB900060E070E88BE395E4F23020F060E070E054
:10CBA00080E793E420E030E040E752E40F94D6259C
:10CBB0006D877E878F87988BCE010D960E948A6441
:10CBC00061960FB6F894DEBF0FBECDBFDF91CF9157
:10CBD0001F910F91FF90EF90DF90CF90BF90AF909B
:10CBE0009F908F907F906F905F904F903F902F908D
:10CBF000089560E070E080E793E430CFCF93DF9357
:10CC000080919B1290919C12891B8095877019F4DA
:10CC10000E94D04DF5CF80919B128F5F8770A091BD
:10CC20009B1298E6A99FD0011124FD01E857FA4F05
:10CC3000EF0119929A95E9F798E09083A356BA4FBD
:10CC400090E1E1ECF2E101900D929A95E1F72091EB
:10CC50009B1290919C12291303C094E69093981212
:10CC600080939B12DF91CF910C94402990919B125D
:10CC700080919C12981306C08091E50A9091E60A73
:10CC8000892B21F080E00E94D04DF0CF0895CF9203
:10CC9000DF92EF92FF92FC01C080D180E280F380AE
:10CCA0002091A80C3091A90C4091AA0C5091AB0C8A
:10CCB000C701B6010F94641E0F9449276093CD12EB
:10CCC0007093CE128093CF129093D012C092BD1267
:10CCD000D092BE12E092BF12F092C01290919B12BD
:10CCE00080919C12981731F0FF90EF90DF90CF90D9
:10CCF0000C94FE650E9436660E947D244091CD1200
:10CD00005091CE126091CF127091D012409335099C
:10CD1000509336096093370970933809882331F0AE
:10CD2000FF90EF90DF90CF900C944029FF90EF9010
:10CD3000DF90CF9008954F925F926F927F928F9283
:10CD40009F92AF92BF92CF92DF92EF92FF920F939A
:10CD50001F93CF93DF93EC018B017A016901F901F5
:10CD600080819181A281B381FA01408151816281E8
:10CD70007381F80180809180A280B38048805980BF
:10CD80006A807B804092B1125092B2126092B312CC
:10CD90007092B4128092B5129092B612A092B7120D
:10CDA000B092B8124093B9125093BA126093BB126A
:10CDB0007093BC128093BD129093BE12A093BF12C9
:10CDC000B093C0122091A80C3091A90C4091AA0CEC
:10CDD0005091AB0CF60160817181828193810F9437
:10CDE000641E0F9449274B015C012091A40C3091E3
:10CDF000A50C4091A60C5091A70CF70160817181A0
:10CE0000828193810F94641E0F9449276B017C01EA
:10CE10002091A00C3091A10C4091A20C5091A30C38
:10CE2000F80160817181828193810F94641E0F9457
:10CE300049272B013C0120919C0C30919D0C409185
:10CE40009E0C50919F0C688179818A819B810F94FF
:10CE5000641E0F9449276093C1127093C21280938D
:10CE6000C3129093C4124092C5125092C61260929F
:10CE7000C7127092C812C092C912D092CA12E09220
:10CE8000CB12F092CC128092CD129092CE12A09240
:10CE9000CF12B092D01290919B1280919C12981751
:10CEA00091F0DF91CF911F910F91FF90EF90DF9064
:10CEB000CF90BF90AF909F908F907F906F905F903A
:10CEC0004F900C94FE650E9436660E947D2440912E
:10CED000C9125091CA126091CB127091CC1200917C
:10CEE000C5121091C6122091C7123091C812C0907D
:10CEF000C112D090C212E090C312F090C412C0923E
:10CF00002909D0922A09E0922B09F0922C0900936A
:10CF10002D0910932E0920932F0930933009409347
:10CF20003109509332096093330970933409409169
:10CF3000CD125091CE126091CF127091D0124093C9
:10CF4000350950933609609337097093380988235F
:10CF500091F0DF91CF911F910F91FF90EF90DF90B3
:10CF6000CF90BF90AF909F908F907F906F905F9089
:10CF70004F900C944029DF91CF911F910F91FF901A
:10CF8000EF90DF90CF90BF90AF909F908F907F9069
:10CF90006F905F904F9008954F925F926F927F9243
:10CFA0008F929F92AF92BF92CF92DF92EF92FF92B9
:10CFB0000F931F93CF93DF93CDB7DEB72C970FB6A8
:10CFC000F894DEBF0FBECDBF2B013C0129873A8705
:10CFD0004B875C8747015801F601E080F1800281B0
:10CFE000138120E030E0A901B701C8010F94FE1DB4
:10CFF000882309F484C05E2D4F2D302F212F852FDB
:10D00000942FA32FB22F89839A83AB83BC8320E014
:10D0100030E0A901B701C8010F94FE1D811104C0C1
:10D02000E12CF12C08E413E4C701D8018D839E8321
:10D03000AF83B887A50194016091030D7091040D31
:10D040008091050D9091060D0F94FE1D87FF0CC079
:10D050008092030D9092040DA092050DB092060DE2
:10D06000CE0101960E948A644092FB0C5092FC0C07
:10D070006092FD0C7092FE0C89859A85AB85BC850B
:10D080008093FF0C9093000DA093010DB093020DBF
:10D09000CE0105960E948A64A50194016091030D5A
:10D0A0007091040D8091050D9091060D0F943C2711
:10D0B000181664F48092030D9092040DA092050D51
:10D0C000B092060DCE0101960E948A640E943666D7
:10D0D0002C960FB6F894DEBF0FBECDBFDF91CF9177
:10D0E0001F910F91FF90EF90DF90CF90BF90AF9086
:10D0F0009F908F907F906F905F904F90089550E039
:10D1000040E030E820E47BCFCF92DF92EF92FF92B5
:10D110000F931F936A01E090030DF090040D0091AE
:10D12000050D1091060DFB01208131814281538153
:10D13000FC0160817181828193810E94CC671F9183
:10D140000F91FF90EF90DF90CF9008952F923F9234
:10D150004F925F926F927F928F929F92AF92BF9207
:10D16000CF92DF92EF92FF920F931F93CF93DF93B3
:10D17000CDB7DEB7CD54D1090FB6F894DEBF0FBEE0
:10D18000CDBF2A969FAF8EAF2A9727967FAF6EAFFF
:10D1900027972C965FAF4EAF2C972E963FAF2EAFB2
:10D1A0002E9728960FAF28978CE0E6EBF2E0DE0191
:10D1B0001D9601900D928A95E1F78CE0E2ECF2E089
:10D1C000DE01599601900D928A95E1F780915512F2
:10D1D000909156128A3A9105F4F48DEC94E10E94F4
:10D1E000662FC35BDF4F0FB6F894DEBF0FBECDBF17
:10D1F000DF91CF911F910F91FF90EF90DF90CF9033
:10D20000BF90AF909F908F907F906F905F904F9066
:10D210003F902F90089580914B02882309F464C1B8
:10D2200080914C0281117BC1A0905902B0905A02AA
:10D23000C0905B02D0905C02E0904D02F0904E02F4
:10D2400000914F029090500220E030E84DE953E405
:10D25000B701802F992D0F943C2718160CF07CC035
:10D26000C701A02FB92D8D879E87AF87B88BEDAAF8
:10D27000F9AE0AAF9CAE20E030E848E953E4B701CC
:10D28000802F992D0F943C2718160CF082C0C701EF
:10D29000A02FB92D898F9A8FAB8FBC8F30905D02F4
:10D2A00020905E0290915F0221969FAF2197A091FE
:10D2B00060022296AFAF2297B09151022396BFAF82
:10D2C0002397E09152022496EFAF2497F0915302F6
:10D2D0002596FFAF25978090540220E030E040E291
:10D2E00052E46B2F7E2F8F2F982D0F943C2718160A
:10D2F0000CF05CC023968FAD239724969FAD2497A6
:10D300002596AFAD2597B82D898B9A8BAB8BBC8BAF
:10D310008D8F9E8FAF8FB8A38DAF9EAFAFAF182DFF
:10D3200040905502509056026090570270905802FB
:10D3300020E030E040E85FE3C301B2010F943C27F6
:10D3400018160CF05EC04D8A5E8A6F8A788E49A2EC
:10D350005AA26BA27CA267C020E030E84DE953E4FA
:10D36000B501C6010F94FE1D87FF0BC0C501D60194
:10D370008D879E87AF87B88BADAAB9AECAAEDCAE3B
:10D380007ACF1DAA20E829AF3DE93AAF83E48CAFFC
:10D3900072CF20E030E848E953E4B501C6010F94AC
:10D3A000FE1D87FF7BCFC501D60174CF20E030E0A2
:10D3B00040E252E4632D722D21968FAD2197229683
:10D3C0009FAD22970F94FE1D87FF15C0832D922DD0
:10D3D0002196AFAD21972296BFAD2297898B9A8B6C
:10D3E000AB8BBC8B8D8F9E8FAF8FB8A33DAE2EAE17
:10D3F000AFAF1B2F95CF1DAE1EAEA0E2AFAF12E4B4
:10D400008FCF4090610250906202609063027090F2
:10D41000640220E030E040E85FE3C301B2010F9412
:10D42000FE1D87FD90CF2C96EEADFFAD2C97408072
:10D430005180628073802DA939AD4AAD5CADC301C6
:10D44000B2010F94DC249B01AC01B501C6010F941D
:10D45000FE1D87FD3FC0A30192016DA979AD8AAD84
:10D460009CAD0F94DB249B01AC01B701802F992D5B
:10D470000F943C27181674F12DAD3EAD4FAD512FD2
:10D48000C301B2010F94DC249B01AC01632D722D0A
:10D4900021968FAD219722969FAD22970F94FE1D66
:10D4A00087FD18C0A30192016DAD7EAD8FAD912FA8
:10D4B0000F94DB249B01AC0123966FAD2397249638
:10D4C0007FAD249725968FAD2597982D0F943C27F7
:10D4D0001816B4F42A96AEADBFAD2A978C9182305F
:10D4E00079F48FEA94E17BCE1DAE1EAEB0E2BFAF01
:10D4F00012E41DAAE0E8E9AFFDE9FAAF23E42CAF9E
:10D500002A96EEADFFAD2A9780818230A9F4289645
:10D510009FAD28979370D1F58CE894E160CE1DAE55
:10D520001EAE30E23FAF12E41DAA80E889AF9DE94C
:10D530009AAFA3E4ACAFE4CF2896FFAD2897F0FDF7
:10D5400010C04091FB0C5091FC0C6091FD0C70914F
:10D55000FE0C498F5A8F6B8F7C8F4D875E876F874C
:10D56000788B28962FAD289721FD10C04091FF0C95
:10D570005091000D6091010D7091020D4D8F5E8FE5
:10D580006F8F78A3498B5A8B6B8B7C8B28963FAD22
:10D59000289732FD10C04091030D5091040D609109
:10D5A000050D7091060D49A35AA36BA37CA34D8B67
:10D5B0005E8B6F8B788F813009F461C0823009F403
:10D5C000A6C18CE0EBEFFCE0DE01119601900D921C
:10D5D0008A95E1F71DA61EA61FA618AA88E0FE01DF
:10D5E0003D96DE01959601900D928A95E1F78E01A8
:10D5F0000B5D1F4FAE01435D5F4FBE01675D7F4F07
:10D60000C8010E948468F12CD02EE12E2796AEAD81
:10D61000BFAD27978C9190E095958795F8161906E0
:10D620000CF026C21DA61EA61FA618AA88E0FE01A1
:10D630007996AD2DBE2D01900D928A95E1F7AE0140
:10D64000435D5F4FBE01675D7F4FC8010E948468E4
:10D650001DA61EA61FA618AA88E0FE013D96D801A9
:10D6600001900D928A95E1F7AE01435D5F4FBE01D7
:10D67000675D7F4FC8010E948468F394C7CF2D85F2
:10D680003E854F855889698D7A8D8B8D9C8D0F9441
:10D69000DB244B015C0120E030E0A9010F94FE1D6A
:10D6A000882309F49ECD29893A894B895C896D8D3F
:10D6B0007E8D8F8D98A10F94DB246B017C0120E07F
:10D6C00030E0A9010F94FE1D882309F48ACD8CE077
:10D6D000EBEFFCE0DE01119601900D928A95E1F7E7
:10D6E0001DA61EA61FA618AA88E0FE013D96DE0113
:10D6F000959601900D928A95E1F7AE01435D5F4FDB
:10D70000BE01675D7F4FCE0185960E9484682E968C
:10D71000AEADBFAD2E978C91880F89AF20E030E081
:10D72000A901C501B4010F943C272401350187FFED
:10D7300004C077FA709477F8709420E030E0A90183
:10D74000C701B6010F943C2787FF76C0D701C601F9
:10D75000B0588DAB9EABAFABB8AFA30192016DA932
:10D760007EA98FA998AD0F94FE1D181614F07501AF
:10D770006401B9ADAB2FB0E0BBAFAAAFBD01BB0F29
:10D78000880B990B0F94051E9B01AC01C701B601D4
:10D790000F94D6256B017C0100E02796EEADFFAD1E
:10D7A00027978081081708F057C110E0812F012EBC
:10D7B000000C990B2AAD3BAD821793070CF053C0B8
:10D7C000CE0149961C0110FD03C0DE011D961D010E
:10D7D000612F012E000C770B880B990B0F94051EFF
:10D7E000A70196010F94641E4B015C01A3019201F5
:10D7F0006DA97EA98FA998AD0F94FE1D1DA21EA232
:10D800001FA218A6A50194011816DCF06D857E856F
:10D810008F8598890F94DC246DA77EA78FA798AB7E
:10D82000B1016C5F7F4FAE014B5D5F4FCE018D96B6
:10D830000E9484681F5FBACFCDAADEAAEFAAF8AE15
:10D840008CCF69897A898B899C890F94DC246DA798
:10D850007EA78FA798ABAE014B5D5F4FBE01635DA6
:10D860007F4FC101E5CF19AD17FD4FC0FE0179967D
:10D870001F0110FD04C09E01235F3F4F1901612F5E
:10D88000012E000C770B880B990B0F94051EA70136
:10D8900096010F94641E4B015C01A30192016DA9D6
:10D8A0007EA98FA998AD0F94FE1D1DA21EA21FA2D6
:10D8B00018A6A50194011816B4F06D857E858F8594
:10D8C00098890F94DC246DA77EA78FA798ABB10130
:10D8D0006C5F7F4FAE014B5D5F4FCE018D960E9416
:10D8E00084681150C1CF69897A898B899C890F948A
:10D8F000DC246DA77EA78FA798ABAE014B5D5F4F71
:10D90000BE01635D7F4FC101EACF0F5F46CF27960F
:10D91000AEADBFAD27978C91882309F462CC8CE023
:10D92000EBEFFCE0DE01119601900D928A95E1F794
:10D930001DA61EA61FA618AA88E0FE013D96DE01C0
:10D94000959601900D928A95E1F75E01BDE2AB0ECE
:10D95000B11C7E01E5E2EE0EF11CA501BE01675D82
:10D960007F4FC7010E94846800E0DA2CCB2C3E2C4C
:10D970002F2C2796AEADBFAD27978C91081708F0D6
:10D9800054C0F12CE12C19AA1AAA1BAA1CAAB7018F
:10D990000F2C000C880B990B0F94051E2CE739ED0A
:10D9A00040E25FE30F94641E2B013C010F94D125EC
:10D9B0002C96EEADFFAD2C9780809180A280B38035
:10D9C000A50194010F94641E2DAD3EAD4FAD512FB6
:10D9D0000F94DC246DA77EA78FA798ABC301B2017B
:10D9E0000F947C279B01AC01C501B4010F94641E08
:10D9F0002DA939AD4AAD5CAD0F94DC246DA37EA397
:10DA00008FA398A7AE014F5C5F4F6D2D7C2D832DAA
:10DA1000922D0E948468FFEFEF1AFF0A2AE0E216B7
:10DA2000F10409F0B0CF0F5FA4CF1DA61EA61FA65C
:10DA300018AA88E0FE013D96DE01959601900D92B0
:10DA40008A95E1F7AE01435D5F4FBE01675D7F4F91
:10DA5000CE0185960E9484681DA21EA21FA218A650
:10DA6000BE016B5D7F4FCE0101960E9453F3B9CB8F
:10DA70001DA21EA21FA218A6B801F5CFCF92DF9259
:10DA8000EF92FF920F931F936B01FC01E080F180F6
:10DA900002811381EBEFFCE02481358146815781BF
:10DAA00060817181828193810E94CC671F910F9167
:10DAB000FF90EF90DF90CF9008958F929F92AF925A
:10DAC000BF92CF92DF92EF92FF920F931F93CF936B
:10DAD000DF93CDB7DEB72C970FB6F894DEBF0FBE3D
:10DAE000CDBF8B0140E050E068E472E44D835E837B
:10DAF0006F83788740E050E060EA70E449875A8796
:10DB00006B877C878130B9F1823009F459C020E0FD
:10DB100030E040E050E46091030D7091040D80917D
:10DB2000050D9091060D0F94DC244B017C0120E043
:10DB300030E048EC53E40F943C27181634F4812C61
:10DB4000912C88ECE82E93E4F92EF801A084B1849E
:10DB5000C284D3849401A701B501C6010F943C2768
:10DB6000181614F054016701C501D60189839A8300
:10DB7000AB83BC8348C0BE01675F7F4FC801089676
:10DB80000E943E6DB8016C5F7F4FAE014B5F5F4FEF
:10DB9000C8010E9484680E94B4292C960FB6F8949C
:10DBA000DEBF0FBECDBFDF91CF911F910F91FF90D0
:10DBB000EF90DF90CF90BF90AF909F908F9008959F
:10DBC000F80120853185428553856091030D709160
:10DBD000040D8091050D9091060D0F94DC246B01CE
:10DBE0007C0120E030E048EC53E40F94FE1D87FDFB
:10DBF00006C0C12CD12C28ECE22E23E4F22EC982DF
:10DC0000DA82EB82FC82BE01675F7F4FCE01019614
:10DC1000B7CF4F925F926F927F928F929F92AF9207
:10DC2000BF92CF92DF92EF92FF921F93CF93DF9339
:10DC300000D000D01F921F92CDB7DEB70E943344B0
:10DC4000D82E87FDB2C08AE50E94DB1D812C912C65
:10DC500020E2A22E21E4B22E882341F040E050E0E1
:10DC6000BA018AE50E9482224B015C011091F90CF5
:10DC7000ED2C0D2C000CFF081E151F0421F060E098
:10DC80008D2D0E941AC120E030E0A901C501B40128
:10DC90000F943C2718167CF580E090E0A0EAB0E4F1
:10DCA0008D839E83AF83B8872091030D3091040D3F
:10DCB0004091050D5091060DC501B4010F94DC246F
:10DCC0002B013C0120E030E048EC53E40F94FE1DB2
:10DCD00087FD06C0412C512C98EC692E93E4792ED7
:10DCE00049825A826B827C82BE016B5F7F4FCE017C
:10DCF00001960E943E6D84E50E94DB1D81116BC080
:10DD00008091F90C882321F060E080E00E941AC124
:10DD10008091E6089091E708A091E808B091E908A1
:10DD2000B05889839A83AB83BC83CE0101960E944D
:10DD30004AF120E030E0A901C501B4010F943C276D
:10DD400018165CF580E090E0A0EAB0E48D839E8335
:10DD5000AF83B887A50194016091030D7091040D04
:10DD60008091050D9091060D0F94DB246B017C01D1
:10DD700020E030E0A9010F943C2718161CF0C12CBC
:10DD8000D12C7601C982DA82EB82FC82BE016B5F04
:10DD90007F4FCE0101960E943E6D8091F90C811754
:10DDA00021F060E0812F0E941AC128960FB6F894E6
:10DDB000DEBF0FBECDBFDF91CF911F91FF90EF90DF
:10DDC000DF90CF90BF90AF909F908F907F906F909B
:10DDD0005F904F90089585E50E948D1D8823D1F0B6
:10DDE0000E9458226B017C0120E030E0A901C701AC
:10DDF000B6010F943C2787FF04C0F7FAF094F7F8B8
:10DE0000F094F7FAF094F7F8F094C982DA82EB8292
:10DE1000FC828BCFF70183E0EE0FFF1F8A95E1F7BD
:10DE2000EA51F74FC080D180E280F380DDCF0F93BD
:10DE30001F93CF93DF938B01CBEFDCE0E091F90CE4
:10DE400024E0E29FF0011124EA5EFD4F2081318140
:10DE500042815381FC0160817181828193810F94A1
:10DE6000D6252C853D854E855F850F94DC246C87F7
:10DE70007D878E879F87C8010E948A64DF91CF913A
:10DE80001F910F910C943666CF92DF92EF92FF9222
:10DE90000F931F93CF93DF9300D01F92CDB7DEB7C0
:10DEA0007C016B018A0161E083EC97E00E94773589
:10DEB00041E654E16AEC77E085E00E9408E8909141
:10DEC000A21181E0890F8093A21180918F1482FFAB
:10DED00006C08B7F80938F149E5F9093A2110E9447
:10DEE000373080E1EBEFFCE0AAEBB4E001900D925B
:10DEF0008A95E1F70E9436668091B90481110FC0BE
:10DF000081E08093B9048091550B8093B7041092FF
:10DF1000550B8091560B8093B8041092560B20E05D
:10DF200030E0A901F70160817181828193810F94B2
:10DF3000FE1D8823F1F08091520B81110CC080915D
:10DF40003A0290913B020197209153123091541262
:10DF50002817390774F080E090E0A0E7B2E48983E5
:10DF60009A83AB83BC83BE016F5F7F4FC7010E9462
:10DF7000176F87E00E948A24811103C0B6010E94B6
:10DF80005D6D20E030E0A901F8016081718182813E
:10DF900093810F94FE1D882319F0C8010E944AF155
:10DFA0000E94C12A81E00F900F900F900F90DF9197
:10DFB000CF911F910F91FF90EF90DF90CF90089538
:10DFC0009091FA0C9817B1F00E9436668091FA0C85
:10DFD000882341F08BEF9CE00E9417241092FA0CEA
:10DFE0000C947A2581E08093FA0C8BEF9CE00E94E0
:10DFF000C623F6CF08950F931F93A8E8BCE090E0E6
:10E0000080E0FC01E55BF34E45915591659174917B
:10E010004D935D936D937D93FC01E55CF34E4591CB
:10E0200055916591749150964D935D936D937C934A
:10E030005397FC01E55DF34E4591559165917491BF
:10E0400090964D935D936D937C9393970496803156
:10E050009105B9F680E29EE4A0E0B0E08093980CD0
:10E060009093990CA0939A0CB0939B0C80E090E84D
:10E07000ABE3B4E48093BC0C9093BD0CA093BE0CB6
:10E08000B093BF0C80E090E0AAE7B4E48093C00CAA
:10E090009093C10CA093C20CB093C30C80E090E0AD
:10E0A000A6E9B3E48093C40C9093C50CA093C60C6E
:10E0B000B093C70C1092C80C1092C90C1092CA0CE5
:10E0C0001092CB0C1092CC0C1092CD0C1092CE0C66
:10E0D0001092CF0C40E050E060E271E44093FF0802
:10E0E00050930009609301097093020980E090E069
:10E0F000A0EAB0E48093030990930409A093050972
:10E10000B09306090AE919E929E93EE300930709F2
:10E11000109308092093090930930A0980930B0989
:10E1200090930C09A0930D09B0930E091092740BF3
:10E130001092750B1092760B1092770B1092700B59
:10E140001092710B1092720B1092730B10926C0B59
:10E1500010926D0B10926E0B10926F0B80E090E09E
:10E16000A0EAB2E480934A0990934B09A0934C092A
:10E17000B0934D091092520910925309109254090C
:10E180001092550988EB9BE09093590980935809A8
:10E190008CED95E090935B0980935A0980E090E0C4
:10E1A000A0E0B0E480934E0990934F09A0935009EA
:10E1B000B093510924E131E0309357092093560977
:10E1C0002FEF30E030935F0920935E092AE030E0C2
:10E1D000309361092093600921E02093620900E0F7
:10E1E00010E82DE933E40093630910936409209348
:10E1F00065093093660940936709509368096093F5
:10E20000690970936A0980936B0990936C09A093D4
:10E210006D09B0936E0910927809109279091092E5
:10E220007A0910927B090E94AF341092FB08109279
:10E23000FC081092FD081092FE0880E00E94E06F3A
:10E240000E94F82880E090E0A8E9B1E48093581299
:10E2500090935912A0935A12B0935B128AE891EEF0
:10E26000AAE6BEE380935C1290935D12A0935E12C7
:10E27000B0935F1280E89AE6A9ECB3E48093601251
:10E2800090936112A0936212B093631283EC95E9AC
:10E29000ACE2B4E48093EE119093EF11A093F011EF
:10E2A000B093F11180E29BE1A2E9B1E48093F21115
:10E2B0009093F311A093F411B093F51187EF9CEDB7
:10E2C000ABECB5E48093F6119093F711A093F8119D
:10E2D000B093F9111092F6080E94D22810925F0BA9
:10E2E00080E090E0A0EEBFE38093570B9093580B33
:10E2F000A093590BB0935A0B80935B0B90935C0BDC
:10E30000A0935D0BB0935E0B1092040A1092030A67
:10E310000E949B2A10927009109271091092720942
:10E32000109273091092740910927509109276096F
:10E330001092770940E050E067ED73E44093E608FF
:10E340005093E7086093E8087093E90880E090E054
:10E35000A1EEB3E48093EA089093EB08A093EC0855
:10E36000B093ED084093EE085093EF086093F008E7
:10E370007093F1088093F2089093F308A093F40847
:10E38000B093F5080E94DB291F910F910C94AF34D4
:10E39000CF9381E080930F090E94274410920F09C8
:10E3A0008823E1F10E942744C82F87E599E10E9464
:10E3B000662F8AE00E942D2F0E94E426AB01BC014B
:10E3C0008EE399E10E9413378AE00E942D2F0E946C
:10E3D000E42620E030E048EC52E40F94641E0F94F1
:10E3E00048267093FE136093FD1385E08093F1132C
:10E3F00082E88093F41386E290E1A0E0B0E080939D
:10E40000F5139093F613A093F713B093F81381EAE2
:10E4100093E10E94B82B8C2FCF9108950E94FB6F3F
:10E420000E94C9440E94074484E799E10E94662F34
:10E43000C0E0F1CF2F923F924F925F926F927F9206
:10E440008F929F92AF92BF92CF92DF92EF92FF9204
:10E450000F931F93CF93DF93CDB7DEB76A970FB6B5
:10E46000F894DEBF0FBECDBF83E50E948D1D182F2F
:10E470003090FA0C882319F00E942022382E409008
:10E48000FB0C5090FC0C6090FD0C7090FE0C809189
:10E49000FF0C9091000DA091010DB091020D8B8B9E
:10E4A0009C8BAD8BBE8B8091030D9091040DA09140
:10E4B000050DB091060D8F8B988FA98FBA8F112300
:10E4C00029F0311003C080E00E94E06F86E50E94D1
:10E4D0008D1D8A8B0E941829882309F4C3C083E408
:10E4E0000E948D1D882309F49DC00E9458226B0153
:10E4F0007C01AEEEBAE0BF83AE83B987A887F5E0B2
:10E50000FD831D861E8628EC2F8702EC1A86212C9F
:10E5100088EC8B8792E49C87A885B985B98BA88BFA
:10E5200015E0E889F98981909190A190B190F98BDB
:10E53000E88B2A85322D4B855C85C501B4010F948B
:10E54000FE1D87FF04C08A86292CAB86BC862D85DC
:10E550003E854F85502FC501B4010F943C271816F6
:10E5600024F48D869E86AF860B2D1150D1F6FD8149
:10E57000F150FD8388859985449699878887F111A4
:10E58000CBCF2D853E854F85502F6A85722D8B858B
:10E590009C850F94DC2420E030E040E05FE30F94A2
:10E5A000641EA70196010F94DC244B015C012DEB46
:10E5B00037E346E855EB0F943C2787FD0AC02DEB67
:10E5C00037E346E855E3C501B4010F94FE1D181664
:10E5D0004CF580E00E94E06F10E0EE80FF8000E0EC
:10E5E000D7016D917D918D919D917D016D01B4E07B
:10E5F000CB1AD108A50194010F94DB24F6016083A6
:10E60000718382839383602F812F0E9415F00F5FA7
:10E61000053031F71F5F8E819F8144969F838E83E3
:10E620001530D9F6AA89AA2351F00E941829882307
:10E6300031F081EE9AE00E94662F0E9476368AE5DC
:10E640000E948D1D882351F00E94582269837A838D
:10E650008B839C83CE0101960E94CBEE832D0E947A
:10E66000E06F0BC0311003C09A89992341F30E94D7
:10E67000074487EF9AE00E94662F332051F0809183
:10E68000FA0C811106C00E941E4382EC9AE00E949F
:10E69000662F0E94074484EB9AE00E94662F8091C7
:10E6A000FA0C0E94F5360E94074487EA9AE00E941D
:10E6B000662FC090370CD090380CE090390CF09059
:10E6C0003A0C20E030E0A901C701B6010F943C27C5
:10E6D00018160CF053C042E0C701B6010E940BBDF2
:10E6E0008DE00E942D2F8AE00E942D2FA301920120
:10E6F0006091FB0C7091FC0C8091FD0C9091FE0CD4
:10E700000F94FE1D81111FC02B893C894D895E89A4
:10E710006091FF0C7091000D8091010D9091020DA0
:10E720000F94FE1D81110FC02F89388D498D5A8D90
:10E730006091030D7091040D8091050D9091060D6F
:10E740000F94FE1D81110E94B4296A960FB6F894A9
:10E75000DEBF0FBECDBFDF91CF911F910F91FF9014
:10E76000EF90DF90CF90BF90AF909F908F907F9071
:10E770006F905F904F903F902F90089582EA9AE0BB
:10E780000E94662FB3CF90919B1280919C12981398
:10E7900008C08091E50A9091E60A892B11F40C9447
:10E7A000EB1D80E00E94D04DEECF2F923F924F9212
:10E7B0005F926F927F928F929F92AF92BF92CF9211
:10E7C000DF92EF92FF920F931F93CF93DF93CDB71A
:10E7D000DEB7A8970FB6F894DEBF0FBECDBF85EDAC
:10E7E0009AE00E94A0248091530B83FD82C0209167
:10E7F000070D3091080D4091090D50910A0D60915F
:10E80000E10A7091E20A8091E30A9091E40A0F9480
:10E81000FE1D882309F46DC01091520B111165C0C3
:10E8200080913A0290913B020197209153123091CE
:10E830005412281739073CF40E94074488E895E1F0
:10E840000E94662F11E02091070D3091080D409134
:10E85000090D50910A0D6091E10A7091E20A8091D0
:10E86000E30A9091E40A0F94DB246B017C0120E021
:10E8700030E0A9010F943C2787FF04C0F7FAF09419
:10E88000F7F8F094E091F90C24E0E29FF0011124F4
:10E89000EA5EFD4F2081318142815381C701B6017B
:10E8A0000F94641E20E030E84BE354E40F943C27BF
:10E8B0001816ECF40E94074489E695E10E94662F41
:10E8C0008091E10A9091E20AA091E30AB091E40AF2
:10E8D0008093070D9093080DA093090DB0930A0D36
:10E8E00081EE9AE00E94476604C010E0ACCF11119F
:10E8F000E7CF2AE037ED43E25CE360914702709195
:10E9000048028091490290914A020F94641E6B0163
:10E910007C016091650270916602072E000C880BE5
:10E92000990B0F94051E9B01AC01C701B6010F9412
:10E93000641E698B7A8B8B8B9C8B8091FA0C88235D
:10E9400009F18090370C9090380CA090390CB09061
:10E950003A0CC090DD0AD090DE0AE090DF0AF09019
:10E96000E00A20E030E0A901C501B4010F94FE1DCA
:10E970008823E1F1A7019601C501B4010F943C275A
:10E980001816A4F1A12CB12C6501E090F90C8E01B0
:10E990000F5E1F4F21EE3AE04DED5AE069ED7AE04F
:10E9A00085ED9AE00E94266480E1E5EDFAE0ABEFA8
:10E9B000BCE001900D928A95E1F7A8960FB6F89405
:10E9C000DEBF0FBECDBFDF91CF911F910F91FF90A2
:10E9D000EF90DF90CF90BF90AF909F908F907F90FF
:10E9E0006F905F904F903F902F9008952091FB0C77
:10E9F0003091FC0C4091FD0C5091FE0C6091D50AB9
:10EA00007091D60A8091D70A9091D80A0F94DB248E
:10EA10006D8B7E8B8F8B988F2091FF0C3091000D2A
:10EA20004091010D5091020D6091D90A7091DA0A5E
:10EA30008091DB0A9091DC0A0F94DB24698F7A8F36
:10EA40008B8F9C8F2091030D3091040D4091050D0B
:10EA50005091060DC701B6010F94DB246D8F7E8F98
:10EA60008F8F98A32091070D3091080D4091090DCB
:10EA700050910A0D6091E10A7091E20A8091E30AD7
:10EA80009091E40A0F94DB246B017C0120E030E0DC
:10EA9000A9016D897E898F89988D0F94FE1D811142
:10EAA0000CC020E030E0A901698D7A8D8B8D9C8DA2
:10EAB0000F94FE1D882309F465CF2D893E894F8967
:10EAC000588DCA01B9010F94641E4B015C01298D58
:10EAD0003A8D4B8D5C8DCA01B9010F94641E9B0168
:10EAE000AC01C501B4010F94DC244B015C012D8DF8
:10EAF0003E8D4F8D58A1CA01B9010F94641E9B0130
:10EB0000AC01C501B4010F94DC244B015C01A701E9
:10EB10009601C701B6010F94641E9B01AC01C501AB
:10EB2000B4010F94DC240F948A274B015C012DEB78
:10EB300037E346E855E30F94FE1D87FF0FC020E042
:10EB400030E0A901C701B6010F943C2746015701E7
:10EB500087FF04C0B7FAB094B7F8B0942DEB37E351
:10EB600046E855E3C501B4010F94FE1D87FD1CCF97
:10EB700020E030E040EA51E4C501B4010F94D6250D
:10EB80000F944F261B01672B19F422242394312C58
:10EB9000B10190E080E00F94031E9B01AC0160E0A6
:10EBA00070E080E89FE30F94D6252B013C01AC0177
:10EBB0009B01C501B4010F94641E69A37AA38BA3C2
:10EBC0009CA3A30192016D897E898F89988D0F94F2
:10EBD000641E6D8B7E8B8F8B988FA3019201698D44
:10EBE0007A8D8B8D9C8D0F94641E698F7A8F8B8F9D
:10EBF0009C8FA30192016D8D7E8D8F8D98A10F94B6
:10EC0000641E6D8F7E8F8F8F98A3A3019201C70121
:10EC1000B6010F94641E6DA37EA38FA398A780E115
:10EC2000EBEFFCE08E010F5F1F4FD80101900D92BA
:10EC30008A95E1F70E9405F52B013C0128EC420E74
:10EC4000511C611C711CF02E912E81E0281A310894
:10EC500009F464C00E9405F58B019C010419150993
:10EC60002609370937FD5FC02B013C0128EC420E15
:10EC7000511C611C711C80E00E94D04D2D893E8981
:10EC80004F89588D69817A818B819C810F94DC2416
:10EC900069837A838B839C83298D3A8D4B8D5C8D20
:10ECA0006D817E818F8198850F94DC246D837E83B6
:10ECB0008F8398872D8D3E8D4F8D58A169857A85DC
:10ECC0008B859C850F94DC2469877A878B879C874A
:10ECD0002DA13EA14FA158A56D857E858F85988970
:10ECE0000F94DC246D877E878F87988BA9A0BAA0AC
:10ECF000CBA0DCA0E090F90C8E010F5E1F4F9E01AF
:10ED0000235F3F4FAE01475F5F4FBE016B5F7F4F99
:10ED10008F2D992D0E942664811197CFA9A0BAA0AA
:10ED2000CBA0DCA032CE0E94F0C7A8CF8F929F92DA
:10ED3000AF92BF92CF92DF92EF92FF92CF93DF9389
:10ED40008090470290904802A0904902B0904A02F9
:10ED5000FC01C080D180E280F38020E030E0A90196
:10ED6000C701B6010F94FE1D882341F0C0924702EF
:10ED7000D0924802E0924902F0924A02C0916502A4
:10ED8000D091660284E690E09093660280936502DB
:10ED9000E091F90C84E0E89FF0011124EA5EFD4F58
:10EDA000C080D180E280F38080E090E0A0E8BFE303
:10EDB00080839183A283B3830E94D573809247029C
:10EDC00090924802A0924902B0924A02D093660201
:10EDD000C0936502E091F90C84E0E89FF0011124F2
:10EDE000EA5EFD4FC082D182E282F382DF91CF9151
:10EDF000FF90EF90DF90CF90BF90AF909F908F905B
:10EE000008950F931F93CF93DF9300D01F92CDB738
:10EE1000DEB79C0105ED1AE090E1EBEFFCE0D801D4
:10EE200001900D929A95E1F7F9012081318142819B
:10EE30005381F80160857185828593850F94DC2468
:10EE4000F801608771878287938780E090E0A0EA6D
:10EE5000B0E489839A83AB83BC83CE0101960E9480
:10EE600096760F900F900F900F90DF91CF911F919A
:10EE70000F9108958F929F92AF92BF92CF92DF929F
:10EE8000EF92FF920F931F93CF93DF9300D000D0A8
:10EE90001F921F92CDB7DEB781E50E948D1D88239A
:10EEA00009F464C120E030E0A90160914E0970913D
:10EEB0004F0980915009909151090F943C271816E1
:10EEC0000CF041C18091520B81110DC080913A022A
:10EED00090913B02019720915512309156122817BC
:10EEE00039070CF430C180E1EBEFFCE0A5EDBAE0AE
:10EEF00001900D928A95E1F780916F098770F12C4E
:10EF0000873009F089C0F0906209FF2009F484C0BD
:10EF100020916B0930916C0940916D0950916E09F7
:10EF20006091030D7091040D8091050D9091060D77
:10EF30000F94DC246093030D7093040D8093050DF2
:10EF40009093060D8090610290906202A0906302FF
:10EF5000B0906402A50194010F943C27181644F464
:10EF60008092030D9092040DA092050DB092060DB3
:10EF700020E030E040E05FE36091B40C7091B50CAC
:10EF80008091B60C9091B70C0F94641E69837A83BC
:10EF90008B839C83CE0101960E948A640E94366610
:10EFA0008091630990916409A0916509B091660907
:10EFB0008093FB0C9093FC0CA093FD0CB093FE0C83
:10EFC0008091670990916809A0916909B0916A09D7
:10EFD0008093FF0C9093000DA093010DB093020D50
:10EFE000E090F90C80E090E0A8ECB2E489839A8389
:10EFF000AB83BC83A12CB12C65018E010F5F1F4F29
:10F0000027E03DE043E05DE06FEF7CE08BEF9CE0CC
:10F010000E9426640E9436666091560970915709D5
:10F02000072E000C880B990B0F94051E20E030E092
:10F0300040E752E40F94D6256D837E838F839887B3
:10F0400020914E0930914F0940915009509151093A
:10F0500060914A0970914B0980914C0990914D093A
:10F060000F94DC2469837A838B839C83BE016B5F5E
:10F070007F4FCE0101960E94176FFF2021F18091F2
:10F08000FF0C9091000DA091010DB091020D4091E7
:10F09000FB0C5091FC0C6091FD0C7091FE0C4093A8
:10F0A000D50A5093D60A6093D70A7093D80A8093F2
:10F0B000D90A9093DA0AA093DB0AB093DC0A84EBB6
:10F0C0009CE00E94967660915A0970915B09072E28
:10F0D000000C880B990B0F94051E20E030E040E7F0
:10F0E00052E40F94D6256D837E838F83988720E02A
:10F0F00030E0A9016091520970915309809154093F
:10F10000909155090F94DC2469837A838B839C83C7
:10F11000BE016B5F7F4FCE0101960E94176F8091F9
:10F12000E10A9091E20AA091E30AB091E40A809387
:10F13000070D9093080DA093090DB0930A0D87E079
:10F140009DE00E94476628960FB6F894DEBF0FBE7A
:10F15000CDBFDF91CF911F910F91FF90EF90DF9086
:10F16000CF90BF90AF909F908F90089583E50E94BD
:10F17000DB1D8823F1F00E9458226B017C0120E006
:10F1800030E0A9010F94FE1D87FD3FC120E030E86B
:10F190004BE354E4C701B6010F943C2718160CF456
:10F1A00038C1C0924A09D0924B09E0924C09F092C2
:10F1B0004D0982E40E94DB1D8823F9F00E94582249
:10F1C0006B017C0120E030E040E251EC0F94FE1D29
:10F1D00087FD27C120E030E040E251E4C701B601DD
:10F1E0000F943C2718160CF423C1C0925209D092F8
:10F1F0005309E0925409F092550985E40E94DB1D01
:10F200008823F1F00E9458226B017C0120E030E05D
:10F21000A9010F94FE1D87FD12C120E030E84BE3E9
:10F2200054E4C701B6010F943C2718160CF40BC127
:10F23000C0924E09D0924F09E0925009F0925109C4
:10F2400080E50E94DB1D882399F00E9458220F94CC
:10F250004826693185E1780714F068E175E16A3084
:10F26000710514F46AE070E07093570960935609D1
:10F2700082E50E94DB1D882399F00E9458220F949A
:10F280004826693185E1780714F068E175E16A3054
:10F29000710514F46AE070E070935909609358099D
:10F2A00085E50E94DB1D882399F00E9458220F9467
:10F2B0004826693185E1780714F068E175E16A3024
:10F2C000710514F46AE070E070935B0960935A0969
:10F2D00087E50E94DB1D882369F00E94582211E017
:10F2E00020E030E0A9010F94FE1D811101C010E063
:10F2F0001093620988E50E94DB1D8823D1F00E94EB
:10F3000058220F94482677FDA6C06C3381E0780719
:10F3100014F06BE371E0072E000C880B990B0F942F
:10F32000051E609363097093640980936509909347
:10F33000660989E50E94DB1D8823D1F00E945822CE
:10F340000F94482677FD8BC0653381E0780714F071
:10F3500064E371E0072E000C880B990B0F94051ED7
:10F3600060936709709368098093690990936A09AB
:10F370008AE50E94DB1D882351F00E945822609389
:10F380006B0970936C0980936D0990936E091092CC
:10F3900078098CE40E94DB1D882379F00E944522C5
:10F3A0008230910550F48093790991E02091F90C15
:10F3B000281708F090E090937A0981E40E948D1D4F
:10F3C000882321F00E94202280937A0984E50E94FC
:10F3D0008D1D882309F449C08091D3049091D404F1
:10F3E000892B09F446C00E94452282309105D8F548
:10F3F0002091F90C28171906B1F18F5F80937809D5
:10F400000E94B6C3109278099ECEC12CD12C7601F1
:10F41000C8CEC12C30E8D32E3BE3E32E34E4F32EE8
:10F42000C0CEC12CD12C20E2E22E21ECF22EDDCE7A
:10F43000C12CD12C90E2E92E91E4F92ED6CEC12C2C
:10F44000D12C7601F5CEC12C80E8D82E8BE3E82EA6
:10F4500084E4F82EEDCE60E070E0CB0162CF60E096
:10F4600070E0CB017DCF1092780980E00E94694264
:10F470006ACE0E94B6C367CE2F923F924F925F92A0
:10F480006F927F928F929F92AF92BF92CF92DF92B4
:10F49000EF92FF921F93CF93DF93CDB7DEB72C97F8
:10F4A0000FB6F894DEBF0FBECDBF7A011901DC01A3
:10F4B0002D913D914D915C912D833E834F835887D3
:10F4C000FB0140805180628073808090FB0C9090A3
:10F4D000FC0CA090FD0CB090FE0CA50194016D8178
:10F4E0007E818F8198850F94FE1D81110EC011E0E1
:10F4F000A30192016091FF0C7091000D8091010DAC
:10F500009091020D0F94FE1D811110E0D1012D91FB
:10F510003D914D915C9129873A874B875C87F70134
:10F52000C080D180E280F3802091010230910202FC
:10F530004091030250910402C701B6010F94FE1DD1
:10F54000882309F44EC0C0920102D0920202E092D8
:10F550000302F09204028091070D9091080DA09192
:10F56000090DB0910A0D4091FF0C5091000D609172
:10F57000010D7091020D8092D50A9092D60AA09248
:10F58000D70AB092D80A4093D90A5093DA0A609306
:10F59000DB0A7093DC0AC092DD0AD092DE0AE092A8
:10F5A000DF0AF092E00A8093E10A9093E20AA093C6
:10F5B000E30AB093E40A20E030E040E05FE36091CA
:10F5C000B40C7091B50C8091B60C9091B70C0F945F
:10F5D000641E69837A838B839C83CE0101960E948B
:10F5E00096762D813E814F8158852093D50A3093A0
:10F5F000D60A4093D70A5093D80A4092D90A50921B
:10F60000DA0A6092DB0A7092DC0AD1012D913D91F9
:10F610004D915C916091E10A7091E20A8091E30A58
:10F620009091E40A0F94DC246093E10A7093E20A5B
:10F630008093E30A9093E40A11112FC020E030E098
:10F64000A90169857A858B859C850F94FE1D8111A2
:10F6500033C060E070E088EC92E469837A838B8346
:10F660009C83CE0101960E9496762C960FB6F89454
:10F67000DEBF0FBECDBFDF91CF911F91FF90EF9006
:10F68000DF90CF90BF90AF909F908F907F906F90C2
:10F690005F904F903F902F9008952AEF3EE74AE207
:10F6A0005FE36091B80C7091B90C8091BA0C9091A5
:10F6B000BB0C0F94641ED1CF60E070E080EA91E44F
:10F6C000CCCF0F931F93CF93DF9300D000D01F9226
:10F6D0001F92CDB7DEB78B01FC0123A5211102C01B
:10F6E0000E9433F31D821E821F82188620E030E0C4
:10F6F00040E05FE36091030D7091040D8091050D72
:10F700009091060D0F94DC2469837A838B839C830C
:10F710009E012B5F3F4FAE014F5F5F4F6FEF7CE06D
:10F720008BEF9CE00E943C7A1D821E821F8218860D
:10F7300020E030E040E05FE3F8016085718582857C
:10F7400093850F94DC2469837A838B839C83B8012F
:10F750006C5F7F4F9E012B5F3F4FAE014F5F5F4F4E
:10F76000C8010E943C7A28960FB6F894DEBF0FBEFF
:10F77000CDBFDF91CF911F910F9108959B01AC01F7
:10F78000485F5F4FBC016C5F7F4F0C943C7A2F92B7
:10F790003F924F925F926F927F928F929F92AF9221
:10F7A000BF92CF92DF92EF92FF920F931F93CF936E
:10F7B000DF93CDB7DEB7A6970FB6F894DEBF0FBEC6
:10F7C000CDBF8C011B015A8749874090FB0C50909C
:10F7D000FC0C6090FD0C7090FE0C8090FF0C9090E3
:10F7E000000DA090010DB090020DDB018D919D9157
:10F7F0000D90BC91A02D8B8B9C8BAD8BBE8B9C01F7
:10F80000AD01C301B2010F94DB246B017C01D10176
:10F8100014968D919D910D90BC91A02D8F8B988FFA
:10F82000A98FBA8F9C01AD01C501B4010F94DB24EF
:10F830006B8F7C8F8D8F9E8FA985BA858D919D91C1
:10F840000D90BC91A02D8B879C87AD87BE879C01B6
:10F85000AD01C301B2010F94DB246F8F78A389A39C
:10F860009AA3A985BA8514968D919D910D90BC910E
:10F87000A02D8F87988BA98BBA8B9C01AD01C501F8
:10F88000B4010F94DB246BA37CA38DA39EA3A701DB
:10F890009601C701B6010F94641E6B017C012B8D8C
:10F8A0003C8D4D8D5E8DCA01B9010F94641E9B0184
:10F8B000AC01C701B6010F94DC244B015C012B891C
:10F8C0003C894D895E896B857C858D859E850F94ED
:10F8D000DB242B013C012F89388D498D5A8D6F8592
:10F8E000788989899A890F94DB246B017C01A301B3
:10F8F0009201C301B2010F94641E2B013C01A701C8
:10F900009601C701B6010F94641E9B01AC01C301AF
:10F91000B2010F94DC240F948A276B017C012F8D98
:10F9200038A149A15AA1CA01B9010F94641E2B0143
:10F930003C012BA13CA14DA15EA1CA01B9010F94CC
:10F94000641E9B01AC01C301B2010F94DC249B0136
:10F95000AC01C501B4010F943C271816B4F520E0A2
:10F9600030E0A901C701B6010F943C2787FF2AC0E8
:10F97000C701B601905820E030E040EA50E40F940F
:10F980003C27181614F5A10169857A85C8010E94E3
:10F99000C77BA6960FB6F894DEBF0FBECDBFDF9132
:10F9A000CF911F910F91FF90EF90DF90CF90BF907C
:10F9B000AF909F908F907F906F905F904F903F900F
:10F9C0002F900895C701B601D6CF20E030E040E087
:10F9D00050E4C501B4010F943C27181624F4B1017A
:10F9E000C8010E94617B19821A821B821C82BE019F
:10F9F0006F5F7F4FC1010E94BE7B2DEC3CEC4CEC55
:10FA00005CE3C701B6010F94641E9B01AC01F801D1
:10FA100060817181828193810F94641E6D837E83E6
:10FA20008F839887D8019B968C919B978823C9F0E8
:10FA30002AE939E949E95FE314966D917D918D9149
:10FA40009C9117970F94641E69837A838B839C83A0
:10FA5000BE016F5F7F4F85ED9AE00E94BE7BF8018B
:10FA600013A6BE016B5F7F4F89859A850E94BE7B7E
:10FA700090CF4F925F926F927F929F92AF92BF9280
:10FA8000CF92DF92EF92FF920F931F93CF93DF936A
:10FA9000CDB7DEB768970FB6F894DEBF0FBECDBF07
:10FAA000FB019080342F390D353008F026C1E180FC
:10FAB000022F0E0D053008F020C1EE2DF0E0E653C8
:10FAC000FB4F4080512C712C612C092C04C0769482
:10FAD0006794579447940A94D2F740FE0EC110E001
:10FAE000F801E653FB4F4080512C712C612CC32E42
:10FAF000D12C04C076946794579447943A95D2F7E2
:10FB000040FEFBC0F22E642F5C01660F770B072EC0
:10FB1000000C880B990B0F94051E2B013C01892DBD
:10FB200094E08902F0011124E059FB4EA3019201F7
:10FB300060817181828193810F94DC246D877E873F
:10FB40008F87988BF601EE0FFF1FEE0FFF1FE05916
:10FB5000FB4EA301920160817181828193810F9498
:10FB6000DB2469837A838B839C836F2D660F770BED
:10FB7000072E000C880B990B0F94051E2B013C01DE
:10FB80008E2D94E08902F0011124E45AFB4EA3016A
:10FB9000920160817181828193810F94DC24698B51
:10FBA0007A8B8B8B9C8B000F111F000F111FF8019C
:10FBB000E45AFB4EA301920160817181828193819D
:10FBC0000F94DB246D837E838F839887F501808576
:10FBD0009185A285B38589879A87AB87BC878D8BF2
:10FBE0009E8BAF8BB88F43E351E061E070E0CE01B4
:10FBF00041960E94AEC743E351E061E070E0CE0160
:10FC000005960E94AEC74AE351E061E070E0CE0184
:10FC10000D960E94AEC74AE351E061E070E0CE016C
:10FC200001960E94AEC7C988DA88EB88FC8827E174
:10FC300037EB41ED58EBC701B6010F943C2787FD28
:10FC40005CC023E030E04AE953E4C701B6010F94F9
:10FC5000FE1D18160CF451C0CD84DE84EF84F888A4
:10FC600027E137EB41ED58EBC701B6010F943C2774
:10FC700087FD43C023E030E84DE953E4C701B601F6
:10FC80000F94FE1D1816CCF1CD80DE80EF80F88435
:10FC900027E137EB41ED58EBC701B6010F943C2744
:10FCA00087FD2BC023E030E04AE953E4C701B601E9
:10FCB0000F94FE1D18160CF1C980DA80EB80FC80D1
:10FCC00027E137EB41ED58EBC701B6010F943C2714
:10FCD00087FD13C023E030E84DE953E4C701B601C6
:10FCE0000F94FE1D18164CF0AE014F5F5F4FBE0122
:10FCF000635F7F4FC5010E94C77B68960FB6F8947B
:10FD0000DEBF0FBECDBFDF91CF911F910F91FF904E
:10FD1000EF90DF90CF90BF90AF909F907F906F90CB
:10FD20005F904F9008952F923F924F925F926F9203
:10FD30007F928F929F92AF92BF92CF92DF92EF927B
:10FD4000FF920F931F93CF93DF93CDB7DEB7C058C9
:10FD5000D1090FB6F894DEBF0FBECDBF81E99AE09E
:10FD60000E94662F0F94041181116EC084E50E94D9
:10FD7000DB1D882329F00E94452260E00E941AC101
:10FD800080E090E0A0E8BFE389839A83AB83BC83E3
:10FD90008D839E83AF83B8878DEC9CECACE4BEE38F
:10FDA00089879A87AB87BC8780E090E0A0E2B1E4C6
:10FDB0008D879E87AF87B88B8CE390E09A8B898B79
:10FDC0008DEC90E09C8B8B8B8DEC9CECACECBEE3D3
:10FDD0008D8B9E8BAF8BB88F80E090E0A0EEBFE361
:10FDE000898F9A8FAB8FBC8F1BA61CA64AE959E955
:10FDF00069E97EE38FE40E9482226D8F7E8F8F8F70
:10FE000098A360E083E40E94302289A360E08BE441
:10FE10000E9430228AA382E40E94DB1D882381F1A4
:10FE20000E944522009761F19C0128523109253634
:10FE3000310520F16CE870E083E69AE00E943537E6
:10FE40008EE59AE00E94662FC058DF4F0FB6F894F7
:10FE5000DEBF0FBECDBFDF91CF911F910F91FF90FD
:10FE6000EF90DF90CF90BF90AF909F908F907F905A
:10FE70006F905F904F903F902F9008959A8B898B51
:10FE80008CE40E94DB1D8823E1F00E9458226B0164
:10FE90007C01C986DA86EB86FC8620E030E0A90189
:10FEA0000F943C2787FD0AC020E030E040E050E49A
:10FEB000C701B6010F94FE1D18161CF486E39AE0E4
:10FEC000C1CF81E50E948D1D882331F18091D3043B
:10FED0009091D404892BE9F00E9458226B017C0197
:10FEE000CD82DE82EF82F8862DEC3CEC4CE45DE3C3
:10FEF0000F943C2787FD0AC020E030E040E751E442
:10FF0000C701B6010F94FE1D181634F485E09AE07F
:10FF100099CF8AED99E096CF83E50E94DB1D882377
:10FF2000E9F00E9458226B017C01CD8ADE8AEF8ABB
:10FF3000F88E2DEC3CEC4CEC5DE30F943C2787FDF8
:10FF40000AC020E030E040E050E4C701B6010F9461
:10FF5000FE1D18161CF483EB99E074CF80E50E9417
:10FF60008D1D882341F18091D3049091D404892B75
:10FF700019F48BE799E066CF8BA58F5F8BA70E9462
:10FF800058226B017C01CD86DE86EF86F88A20E060
:10FF900030E0A9010F943C2787FD0AC020E030E043
:10FFA00048EC51E4C701B6010F94FE1D18161CF46D
:10FFB00083E599E047CF86E40E94DB1D8823E9F0C2
:10FFC0000E9458226B017C01C98EDA8EEB8EFC8E6A
:10FFD00020E030E040E85FE30F943C2787FD0AC053
:10FFE00020E030E040E850E4C701B6010F94FE1D68
:10FFF00018161CF48AE299E025CFC98CDA8CEB8CB8
:020000021000EC
:10000000FC8C8D889E88AF88B88CA7019601C701AB
:10001000B6010F94641E9B01AC0160E070E084E4C3
:1000200090E40F94D62529813A814B815C810F940D
:10003000641E2B013C01A5019401C501B4010F947C
:10004000641EA70196010F94641E2CEE31E548EB67
:100050005DE30F94D6259B01AC01C301B2010F945F
:10006000641E69837A838B839C8388E40E94DB1DF2
:10007000882379F00E944522009759F09C01255A67
:1000800031092838310518F08CEF98E0DBCE9C8BD5
:100090008B8B85E50E948D1D8823C9F00E9405F594
:1000A000611571058105910511F00F9484198091F6
:1000B000D3049091D404892B91F00E94582260932C
:1000C000CF047093D0048093D1049093D20482E53E
:1000D0000E948D1D811108C088EC98E0B3CE60E0CD
:1000E00070E088E492E4EBCF8091D3049091D40443
:1000F000892B61F00E944522E5969FAF8EAFE59770
:10010000181619064CF084E998E09CCE2AE130E0FC
:10011000E5963FAF2EAFE59789E50E94DB1D88236A
:1001200009F4BEC00E94582220913F0C3091400C2F
:100130004091410C5091420C0F94DB244B015C0127
:1001400088E50E94DB1D882309F4B3C00E94582271
:1001500020913B0C30913C0C40913D0C50913E0C59
:100160000F94DB246B017C01CBA2DCA2EDA2FEA2EA
:100170008FA298A6A9A6BAA627E137EB41ED58EBC6
:10018000C501B4010F943C2787FD9CC023E030E0FB
:100190004AE953E4C501B4010F94FE1D18160CF48E
:1001A00091C027E137EB41ED58EBC701B6010F9441
:1001B0003C2787FD87C023E030E84DE953E4C701C1
:1001C000B6010F94FE1D18160CF47CC084E40E9446
:1001D0008D1D91E089270E94E06F80E090E0A0EA09
:1001E000B0E48DA79EA7AFA7B8ABCE018D960E94B5
:1001F000D8F230915F0BEC963FAFEC9710925F0B0B
:100200000E943B1A89E498E00E94662F89899A89A6
:100210008A3191050CF059C08B899C890E94071E78
:1002200061E08091F90C0E949ABF811156C06FEF76
:100230008EE598E00E94AA358CA5811104C0CE01FC
:1002400001960E9433F380E090E0A0EAB0E480934E
:10025000DD0A9093DE0AA093DF0AB093E00A1DA6A0
:100260001EA61FA618AABE01635D7F4F85ED9AE00A
:100270000E94BE7BEC965FADEC9750935F0B0E94A3
:100280003B1A8AA18111E0CD1092EC111092EB1172
:100290000E9471C48091F90C90E00E94071ED4CD99
:1002A0008090FF0C9090000DA090010DB090020D79
:1002B00047CFC090FB0CD090FC0CE090FD0CF09070
:1002C000FE0C52CF8AE698E0BDCD0E94DA2081E094
:1002D0000E9422BE8111A0CFAACF1092070D1092CA
:1002E000080D1092090D10920A0D87E09DE00E9402
:1002F00047668BA5882309F452C020E030E040E730
:1003000051E46091B80C7091B90C8091BA0C909145
:10031000BB0C0F94D6256DA77EA78FA798AB80E165
:10032000EBEFFCE0A5EDBAE001900D928A95E1F7C4
:100330002D853E854F8558896091E10A7091E20ACA
:100340008091E30A9091E40A0F94DC246093E10A1F
:100350007093E20A8093E30A9093E40ACE018D96AB
:100360000E9496762D853E854F8558896091E10AD9
:100370007091E20A8091E30A9091E40A0F94DB24E1
:100380006093E10A7093E20A8093E30A9093E40A8F
:100390008CA5811104C0CE0101960E9433F3EAECD2
:1003A000F4E085E0DF011D928A95E9F780E1EBEF4B
:1003B000FCE0A5EDBAE001900D928A95E1F7898500
:1003C0009A85AB85BC858093DD0A9093DE0AA09365
:1003D000DF0AB093E00A1DA61EA61FA618AABE013A
:1003E000635D7F4F85ED9AE00E94BE7BBE01635E38
:1003F0007F4F85ED9AE00E94BE7B89A1882309F496
:10040000F5C32091FB0C3091FC0C4091FD0C5091F8
:10041000FE0CE0962CAF3DAF4EAF5FAFE097809102
:10042000FF0C9091000DA091010DB091020DAC96C2
:100430008CAF9DAFAEAFBFAFAC97A0E7B4E1A196D4
:10044000BFAFAEAFA197312C212CBFEF6C96BFAFE1
:100450006C97EFEFA496EFAFA497FFEFE396FFAF93
:10046000E3972FE4E6962FAFE69733ECE7963FAF9E
:10047000E79707E481E090E0A0E0B0E0022C04C040
:10048000880F991FAA1FBB1F0A94D2F7C458DF4FC9
:1004900088839983AA83BB83CC57D040AAECB4E06D
:1004A000E296BFAFAEAFE297ECE5F4E1A396FFAF03
:1004B000EEAFA39710E0C058DF4F2882C058D0405D
:1004C000E296AEADBFADE2978D91E296BFAFAEAF13
:1004D000E29790E0B0E0A0E0C458DF4F2881398176
:1004E0004A815B81CC57D04082239323A423B52338
:1004F000892B8A2B8B2B09F0E5C0A196AEADBFAD41
:10050000A197CD90DD90ED90FC90A396AEADBFADE0
:10051000A3972D913D914D915C91A8962CAF3DAF45
:100520004EAF5FAFA897A7019601E0966CAD7DAD89
:100530008EAD9FADE0970F94DB242B013C01A89674
:100540002CAD3DAD4EAD5FADA897AC966CAD7DAD1D
:100550008EAD9FADAC970F94DB244B015C01A301E2
:100560009201C301B2010F94641E2B013C01A5014D
:100570009401C501B4010F94641E9B01AC01C30139
:10058000B2010F94DC240F948A274B015C01A70170
:1005900096016BA17CA18DA19EA10F94DB246B0120
:1005A0007C01A8962CAD3DAD4EAD5FADA8976FA177
:1005B00078A589A59AA50F94DB242B013C01A701FE
:1005C0009601C701B6010F94641E6B017C01A30163
:1005D0009201C301B2010F94641E9B01AC01C701DB
:1005E000B6010F94DC240F948A2720E030E040E726
:1005F00051E40F94D625A50194010F94DC246B01DE
:100600007C018090CF049090D004A090D104B09051
:10061000D20420E030E040E85FE3C501B4010F946C
:100620003C271816F4F4C501B4010F9448264B0179
:100630005C0160E070E0CB01181419041A041B047B
:1006400034F40F943519A50194010F9464240F9488
:10065000051E9B01AC01B601C7010F94DC246B01A0
:100660007C019601A701E3966FADE397E6967FAD17
:10067000E697E7968FADE797902F0F943C271816D3
:100680000CF56C961FAF6C97C058DF4FB881C058FF
:10069000D040A496BFAFA497E896CFAEE897E9966E
:1006A000DFAEE997EA96EFAEEA97EB96FFAEEB97EF
:1006B000E396CFAEE397E696DFAEE697E796EFAE2A
:1006C000E7970F2D1F5FA396EEADFFADA39734966E
:1006D000A396FFAFEEAFA397153009F0F1CEFFEF71
:1006E0002F1A3F0AA1962EAD3FADA1972C5F3F4F29
:1006F000A1963FAF2EAFA19735E02316310409F044
:10070000B9CE6C964FAD6C97E42FF0E0E653FB4FFB
:10071000208181E090E0A0E0B0E0A4960FACA49727
:1007200004C0880F991FAA1FBB1F0A94D2F7822BFF
:100730008083A4965FADA49762965FAF629763963D
:100740004FAF6397E8968FADE897E9969FADE9972D
:10075000EA96AFADEA97EB96BFADEB9767968CAF95
:100760009DAFAEAFBFAF67975F3F09F423C24F3F66
:1007700009F420C284E04802F0011124E45AFB4E3F
:10078000108101813280238027E137EB41ED58EB66
:10079000612F702F832D922D0F943C2787FD0EC261
:1007A00023E030E04AE953E4612F702F832D922D2E
:1007B0000F94FE1D18160CF401C2A4969FADA497C9
:1007C000A4E09A02F0011124E059FB4EC080D180D0
:1007D000E280F38027E137EB41ED58EBB601C7012A
:1007E0000F943C2787FDEAC123E030E84DE953E44C
:1007F000B601C7010F94FE1D18160CF4DFC120E0EE
:1008000030E040EA50E4B601C7010F94DC24A09622
:100810006FAFA097A2967FAFA297A5968FAFA5972F
:10082000A9969FAFA997CB01A596AFADA597A9961D
:10083000BFADA99721968CAF9DAFAEAFBFAF21974B
:10084000812F902FA32DB22D25968CAF9DAFAEAFEB
:10085000BFAF2597A496BFADA497B11109C26C96FE
:10086000EFAD6C97E111D1C120E030E040EA50E4F7
:10087000612F702F832D922D0F94DC24A4966FAFDF
:10088000A497AD967FAFAD97E1968FAFE197E396D2
:100890009FAFE3976C96FFAD6C97FF2309F4AAC254
:1008A0006C963FAD6C97A096CFAEA097A296DFAEA8
:1008B000A297A596EFAEA597A996FFAEA99734305B
:1008C0000CF0CDC122ED822E23E5922E2BE7A22E35
:1008D00021E4B22E21964CAC5DAC6EAC7FAC21977E
:1008E00025962CAD3DAD4EAD5FAD25976F962CAFE7
:1008F0003DAF4EAF5FAF6F97A3019201B601C70145
:100900000F94DB242D966CAF7DAF8EAF9FAF2D97EC
:100910006F962CAD3DAD4EAD5FAD6F97612F702FD3
:10092000832D922D0F94DB2461966CAF7DAF8EAF3B
:100930009FAF6197A30192016091FB0C7091FC0C39
:100940008091FD0C9091FE0C0F94DB242B013C0157
:100950006F962CAD3DAD4EAD5FAD6F976091FF0CC6
:100960007091000D8091010D9091020D0F94DB2488
:100970006F966CAF7DAF8EAF9FAF6F97A0968FAD28
:10098000A097A2969FADA297A596AFADA597A99661
:10099000BFADA9978DA79EA7AFA7B8ABA4968FAD03
:1009A000A497AD969FADAD97E196AFADE197E39675
:1009B000BFADE39789AB9AABABABBCABC984DA8470
:1009C000EB84FC84CDAADEAAEFAAF8AE2DEC3CECB9
:1009D0004CEC5CE3C501B4010F94641E29813A819B
:1009E0004B815C810F94641E2091070D3091080D9E
:1009F0004091090D50910A0D0F94DC2469AF7AAF34
:100A00008BAF9CAFA3019201C301B2010F94641E8E
:100A10002B013C016F962CAD3DAD4EAD5FAD6F9798
:100A2000CA01B9010F94641E9B01AC01C301B2015C
:100A30000F94DC2420E030E040E050E40F943C27A9
:100A40001816ACF420E030E040E05FE3C701B601E7
:100A50000F94DC2429966CAF7DAF8EAF9FAF2997A2
:100A6000BE01635C7F4FCE0101960E94617B898548
:100A70009A85AB85BC8529968CAF9DAFAEAFBFAFD5
:100A800029976B961CAE1DAE1EAE1FAE6B97BE01B6
:100A9000695A7F4FCE01CD960E94BE7B8CA58823DC
:100AA000C1F02AE939E949E95FE36D817E818F81EF
:100AB00098850F94641E6B966CAF7DAF8EAF9FAF21
:100AC0006B97BE01695A7F4F85ED9AE00E94BE7B0D
:100AD0001CA6A090B00CB090B10CC090B20CD090FD
:100AE000B30CE090AC0CF090AD0C0091AE0C1091FA
:100AF000AF0C9701A801B501C6010F943C27181649
:100B000014F0750186018090470290904802A090F1
:100B10004902B0904A022DEC3CEC4CEC5DE3B7018D
:100B2000C8010F94641E609347027093480280933B
:100B3000490290934A0240E0BE01675B7F4FCE01BD
:100B40008D960F94030C80E1EBEFFCE0A5EDBAE08D
:100B500001900D928A95E1F78092470290924802A7
:100B6000A0924902B0924A0220E04FEFBE016F5AB4
:100B70007F4FCE0101960E94397D20E041E0BE0109
:100B80006F5A7F4FCE0101960E94397D2FEF40E0D2
:100B9000BE016F5A7F4FCE0101960E94397D21E040
:100BA00040E0BE016F5A7F4FCE0101960E94397D11
:100BB0000E94366680910B0D80930C0DE5964EAD2C
:100BC0005FADE59741505109E5965FAF4EAFE597B0
:100BD000452B09F42CCB62968FAD629787FD27CB0E
:100BE00063968FAD639787FF08CC21CB2BA13CA1E7
:100BF0004DA15EA1E0962CAF3DAF4EAF5FAFE09749
:100C00008FA198A5A9A5BAA512CCC601D701219696
:100C10008CAF9DAFAEAFBFAF219720E030E040EA90
:100C200050E4612F702F832D922D0F94DB24259695
:100C30006CAF7DAF8EAF9FAF25976C962FAD6C9745
:100C400024300CF411CEA4961FAFA497AD960FAF2D
:100C5000AD97E1963FAEE197E3962FAEE39792ED25
:100C6000892E93E5992E9BEFA92E90E4B92E32CED2
:100C7000A4964FADA49744300CF46EC06C965FAD53
:100C80006C975430BCF120E030E040EA50E4B6010B
:100C9000C7010F94DB2421966CAF7DAF8EAF9FAF61
:100CA000219720E030E040EA50E4612F702F832D3F
:100CB000922D0F94DB24A4966FAFA497AD967FAFCF
:100CC000AD97E1968FAFE197E3969FAFE3976C9670
:100CD0009FAD6C97A096CFAEA097A296DFAEA297DD
:100CE000A596EFAEA597A996FFAEA99794300CF004
:100CF000B6CFE8CDC601D70121968CAF9DAFAEAF80
:100D0000BFAF219720E030E040EA50E4612F702F20
:100D1000832D922D0F94DC2425966CAF7DAF8EAF82
:100D20009FAF25976C968FAD6C978111BACF20E05D
:100D300030E040EA50E4B601C7010F94DB24A096EE
:100D40006FAFA097A2967FAFA297A5968FAFA597FA
:100D5000A9969FAFA99777CF6C96AFAD6C97A1116D
:100D60002BC020E030E040E251E4A0966FADA097A8
:100D7000A2967FADA297A5968FADA597A9969FAD98
:100D8000A9970F94DB24A0966FAFA097A2967FAF90
:100D9000A297A5968FAFA597A9969FAFA997A4965E
:100DA0001FAFA497AD960FAFAD97E1963FAEE19719
:100DB000E3962FAEE39786CD6C96BFAD6C97B430BB
:100DC00034F120E030E040E251E4A0966FADA0970E
:100DD000A2967FADA297A5968FADA597A9969FAD38
:100DE000A9970F94DB2421966CAF7DAF8EAF9FAF98
:100DF0002197D5CFA096CFAEA097A296DFAEA297AF
:100E0000A596EFAEA597A996FFAEA99728CFA49671
:100E10001FAFA497AD960FAFAD97E1963FAEE197A8
:100E2000E3962FAEE39782ED882E83E5982E8BEF25
:100E3000A82E81E4B82E4ECD8F929F92AF92BF9292
:100E4000CF92DF92EF92FF920F931F93CF93DF9396
:100E500000D01F92CDB7DEB75C016B017A01122F73
:100E6000002309F443C00E94074489E198E00E94EE
:100E7000662F61E0812F0E942B319090E90483E07E
:100E80008093E90481E0809366120E940E3682E02E
:100E90008093671240E369E078E085EF97E00E9475
:100EA0001A3640E069E97DE08EEE97E00E941A363E
:100EB00060E081EE97E00E94773589EE97E00E942E
:100EC000662F8AE00E942D2F8BEF97E00E94AF20C3
:100ED00080916612882341F060E0812F0E942B31BF
:100EE00081E00E94D04DF4CF9092E90420E030E000
:100EF000A901F50160817181828193810F94FE1DAA
:100F0000882371F080E090E0A0ECB0E489839A83BC
:100F1000AB83BC83BE016F5F7F4FC5010E94176F1B
:100F200020E030E0A901F601608171818281938126
:100F30000F94FE1D882351F18090C00C9090C10C3D
:100F4000A090C20CB090C30C80E090E0A0E7B1E4A8
:100F50008093C00C9093C10CA093C20CB093C30CAF
:100F600080E090E0A0EAB1E489839A83AB83BC83FC
:100F7000BE016F5F7F4FC6010E94176F8092C00C49
:100F80009092C10CA092C20CB092C30C20E030E051
:100F9000A901F70160817181828193810F943C27BF
:100FA000181674F480E090E0A0E4B0E489839A839A
:100FB000AB83BC83BE016F5F7F4FC7010E94176F79
:100FC00029E93DE040ED57E06AED77E081E00E94DD
:100FD0003D360E940E3681E00F900F900F900F90DB
:100FE000DF91CF911F910F91FF90EF90DF90CF9005
:100FF000BF90AF909F908F900895CF93C82F80910E
:10100000530B83FD14C08091520B811110C080914D
:101010003A0290913B029C012150310940915512B6
:10102000509156124217530714F40E94071ECC2306
:1010300031F061E08091F90CCF910C949ABF8091CE
:10104000520B91E0892780934602809146028823C3
:1010500089F0809153129091541220915512309141
:101060005612821B930B97FF03C0919581959109AE
:10107000029744F4109246028091530B83FF06C0FE
:10108000C1E01AC080E00E94D04DDFCFC091520B6A
:10109000C11112C080913A0290913B0201972091B8
:1010A0005512309156122817390754F70E940744F9
:1010B00082EB97E00E94662F8C2FCF9108959F922C
:1010C000AF92BF92CF92DF92EF92FF920F931F9356
:1010D000CF93DF93CDB7DEB764970FB6F894DEBF3A
:1010E0000FBECDBF0E943344D82E87FDC6C08AE50F
:1010F0000E94DB1D882309F4D2C040E050E0BA0111
:101100008AE50E9482227B018C01B090F90C8D2D22
:101110000D2C000C990BB816190621F060E08D2DEE
:101120000E941AC12091030D3091040D4091050DCC
:101130005091060D60E070E088EC93E40F94DB249E
:10114000962EA72E6C019701A8010F943C27181624
:101150001CF0E92CFA2C860120E030E0A901B7014F
:10116000C8010F943C27181624F4E12CF12C00E060
:1011700010E0B701C8010F944826072E000C880B19
:10118000990B0F94051E6D837E838F83988720E0D3
:1011900030E0A9010F94FE1D882321F0CE010596B1
:1011A0000E94017780E090E0A0EAB1E489879A8705
:1011B000AB87BC871D861E861F86188A8CE40E941A
:1011C0008D1D882309F470C00E9458226B017C0198
:1011D00020E030E0A901C701B6010F943C2787FF4A
:1011E00004C0F7FAF094F7F8F094C98ADA8AEB8A27
:1011F000FC8A20915512309156122430310574F03A
:101200008091531290915412821B930B97FF03C04D
:1012100091958195910901E004970CF400E080E03C
:101220000E94FD87882359F022E0AE01475F5F4F9F
:10123000BE016F5E7F4FCE010D960E941C876D81AF
:101240007E818F8198858B019C01305809831A8398
:101250002B833C8320E030E0A9010F94FE1D8823FE
:1012600021F0CE0101960E9401778091F90C8B1537
:1012700021F060E08B2D0E941AC164960FB6F8949D
:10128000DEBF0FBECDBFDF91CF911F910F91FF90B9
:10129000EF90DF90CF90BF90AF909F900895E12C9A
:1012A000F12C00E211E431CFE091F90C88E0E89FE5
:1012B000F0011124EA51F74FC480D580E680F78011
:1012C00087CF7F928F929F92AF92BF92CF92DF9201
:1012D000EF92FF920F931F93CF93DF9300D000D034
:1012E0001F921F92CDB7DEB76C015B014A01722ECF
:1012F000780100913F090E94131E80915512909130
:1013000056128E159F051CF4C7010E94071E80E02F
:101310000E94FD87882331F0272DA401B501C60165
:101320000E941C871E141F0444F4C7010E94071E5C
:1013300060E08091F90C0E949ABF81E00E94FD87D5
:1013400080E090E0A0E7B2E489839A83AB83BC831A
:1013500080E090E0A0E8B0EC8D839E83AF83B887F7
:10136000BE016F5F7F4FCE0105960E94176F87E029
:101370000E948A24811158C08091030D9091040D20
:10138000A091050DB091060D4091BE045091BF048F
:101390006091C0047091C104C090BA04D090BB04A5
:1013A000E090BC04F090BD04C092D50AD092D60A59
:1013B000E092D70AF092D80A4093D90A5093DA0AF9
:1013C0006093DB0A7093DC0A8093DD0A9093DE0A57
:1013D000A093DF0AB093E00A80E090E0A8E4B2E4D2
:1013E00089839A83AB83BC83CE0101960E94967653
:1013F0008091C2049091C304A091C404B091C5042B
:101400008093DD0A9093DE0AA093DF0AB093E00A8E
:1014100080E090E0A0EAB0E489839A83AB83BC8348
:10142000CE0101960E949676C12CD12C80E7E82E41
:1014300082E4F82EC982DA82EB82FC8280E090E0BE
:10144000A0E8B0E48D839E83AF83B887BE016F5F51
:101450007F4FCE0105960E94176F20E030E0A90172
:101460006091C6047091C7048091C8049091C9042A
:101470000F94FE1D87FF0BC0C982DA82EB82FC82CB
:10148000BE016F5F7F4F86EC94E00E94176F8091E2
:10149000C6049091C704A091C804B091C904809378
:1014A000070D9093080DA093090DB0930A0D80933A
:1014B000E10A9093E20AA093E30AB093E40A81EE72
:1014C0009AE00E9447668091F60881110E9449EFD8
:1014D00061E088E398E00E9477358091A211815005
:1014E0008093A21141E654E160E478E085E00E9437
:1014F00008E88091A211882339F00E94E4AD809120
:10150000A21181508093A2118091B904882351F0D7
:101510001092B9048091B7048093550B8091B80460
:101520008093560B8091A311823011F40E94742F86
:101530000F94D51028960FB6F894DEBF0FBECDBF1E
:10154000DF91CF911F910F91FF90EF90DF90CF909F
:10155000BF90AF909F908F907F900895CF92DF9231
:10156000EF92FF92CF93DF936B017C01D42FC09158
:10157000E90483E08093E90481E080936612C1145A
:10158000D104E104F10431F00E9405F5C60ED71E26
:10159000E81EF91E80916612882389F0C114D104D7
:1015A000E104F10421F48D2F0E94D04DF3CF0E946D
:1015B00005F56C197D098E099F0997FDF4CF1092EE
:1015C0006612C093E904DF91CF91FF90EF90DF9016
:1015D000CF9008950F931F93CF93DF93C82F162FAB
:1015E0000E940744C11194C0C6E1D7E0CE010E9419
:1015F000662F61E0812F0E942B310E9405F5685310
:1016000070458F4F9F4F60933B0970933C098093C7
:101610003D0990933E0910923F090091E90483E04F
:101620008093E90430E020E049E95DE064EA77E096
:1016300082E00E943D3684EA97E00E94AF2081E07C
:101640008093661280916612882309F464C060E07A
:10165000812F0E942B3180913F09882309F454C0C7
:101660000E9407448AE897E00E94662F30E020E05D
:1016700044E757E06BE777E082E00E943D368BE776
:1016800097E00E94AF2041E060E070E0CB010E9453
:10169000AE8A30E020E050E040E067E677E085E0A9
:1016A0000E943D3687E697E00E94CB2C0E94131ED5
:1016B00080E00E94FD870E940744CE010E94662FB1
:1016C0000E9405F5685370458F4F9F4F60933B090B
:1016D00070933C0980933D0990933E0910923F0915
:1016E00030E020E049E95DE06BE577E082E00E94D0
:1016F0003D368AE497E00E94AF2081E08093661235
:1017000061E0812F0E942B3181E00E94D04D9ACF61
:10171000CBE2D7E06BCF0093E904DF91CF911F912B
:101720000F910895BF92CF92DF92EF92FF920F93A5
:101730001F93CF93DF93CDB7DEB7A0970FB6F89482
:10174000DEBF0FBECDBF0E94334487FDE0C0B09026
:10175000F90C282F082E000C330BB216130619F0C3
:1017600060E00E941AC185E40E948D1D882309F45F
:10177000DEC00E9458226B017C0120E030E0A9010C
:101780000F943C2787FF04C0F7FAF094F7F8F09421
:10179000F7FAF094F7F8F094C98ADA8AEB8AFC8AAF
:1017A0008CE0EEECF2E0DE01119601900D928A954C
:1017B000E1F78AE50E94DB1D882351F040E050E00C
:1017C000BA018AE50E94822269877A878B879C8783
:1017D00088E50E94DB1D882351F040E050E0BA010B
:1017E00088E50E94822269837A838B839C8389E5C2
:1017F0000E94DB1D882351F040E050E0BA0189E5EA
:101800000E9482226D837E838F83988785E50E9464
:101810008D1D882309F492C00E9458226B017C011F
:1018200020E030E0A901C701B6010F943C2787FFF3
:1018300004C0F7FAF094F7F8F094F7FAF094F7F898
:10184000F094CD8ADE8AEF8AF88E198E1A8E1B8E5E
:101850001C8E8CE40E948D1D882309F47CC00E949C
:1018600058226B017C0120E030E0A901C701B601DC
:101870000F943C2787FF04C0F7FAF094F7F8F09430
:10188000CD8EDE8EEF8EF8A262E070E082E40E94E0
:101890004922F82E8091A211811131C021E0AE01C0
:1018A0004B5E5F4FBE016F5F7F4FCE0141960E943E
:1018B000446F882321F16F2D81E00E94EA8A82E53E
:1018C0000E94DB1D882309F453C00E94452240E09A
:1018D00050E060EA71E44D875E876F87788B2091D6
:1018E000A211222361F08C012F2DAE01435F5F4FC7
:1018F000BE01635E7F4FCE0149960E94618980914F
:10190000F90C8B1521F060E08B2D0E941AC1A09676
:101910000FB6F894DEBF0FBECDBFDF91CF911F9100
:101920000F91FF90EF90DF90CF90BF900895C12C62
:10193000D12C80E8E82E80E4F82E2ACFE091F90C33
:1019400088E0E89FF0011124EA51F74FC080D18070
:10195000E280F38065CFE091F90C88E0E89FF00128
:101960001124EA51F74FC480D580E680F7807BCF01
:1019700090E080E0ACCFCF92DF92EF92FF920F9396
:101980001F93CF93DF93CDB7DEB76C970FB6F89464
:10199000DEBF0FBECDBF8CE40E948D1D882309F4ED
:1019A000B0C00E9458226B017C0120E030E0A90108
:1019B0000F943C2787FF04C0F7FAF094F7F8F094EF
:1019C000F7FAF094F7F8F094C98EDA8EEB8EFC8E6D
:1019D0008CE0EEECF2E0DE01119601900D928A951A
:1019E000E1F788E50E94DB1D8823A1F040E050E08C
:1019F000BA0188E50E94822220913B0C30913C0C78
:101A000040913D0C50913E0C0F94DB2469837A8306
:101A10008B839C8389E50E94DB1D8823A1F040E035
:101A200050E0BA0189E50E94822220913B0C30915E
:101A30003C0C40913D0C50913E0C0F94DB246D8387
:101A40007E838F8398878AE50E94DB1D882351F06F
:101A500040E050E0BA018AE50E94822269877A87D5
:101A60008B879C871D861E861F86188A8091A211EF
:101A7000811138C020E0AE01435F5F4FBE016F5F50
:101A80007F4FCE0149960E94446F882359F180917F
:101A9000F60881110E9449EF60E080E00E94EA8A26
:101AA000898D9A8DAB8DBC8DB0588D8B9E8BAF8BF5
:101AB000B88F198A1A8A1B8A1C8A1D861E861F8661
:101AC000188A8091A211882369F010E000E020E0DC
:101AD000AE014B5E5F4FBE016F5E7F4FCE010D9634
:101AE0000E9461896C960FB6F894DEBF0FBECDBF21
:101AF000DF91CF911F910F91FF90EF90DF90CF90EA
:101B00000895C12CD12C80E8E82E80E4F82E58CF1F
:101B10002F923F924F925F926F927F928F929F92FD
:101B2000AF92BF92CF92DF92EF92FF920F931F93EB
:101B3000CF93DF93CDB7DEB7E5970FB6F894DEBF4E
:101B40000FBECDBF8DAB2091E9042CAB21E02093DB
:101B5000E90480910B058D3409F4B8C4843511F47F
:101B60000C9409A2873409F091C1809109059091E4
:101B70000A058A31910509F432C208F079C184302E
:101B8000910508F030C12091480A8230910508F48F
:101B90008EC1213009F091C111E0029709F010E0E7
:101BA0000E94992219821A821B821C821D821E8227
:101BB0001F82188682E50E94DB1D882309F490C1EC
:101BC0000E9458226B017C0120E030E0A9010F94B3
:101BD000FE1D882309F4EAC04090FB0C5090FC0CD9
:101BE0006090FD0C7090FE0C8091FF0C9091000DA8
:101BF000A091010DB091020D8CA79DA7AEA7BFA724
:101C00008090D50A9090D60AA090D70AB090D80AB2
